:040000000C94C30C8D
:100004000C9400000C9400000C9400000C9400006C
:100014000C9400000C9400000C9417610C940000E4
:100024000C9400000C940C150C9400000C9400002B
:100034000C9400000C9400000C9400000C94C71461
:100044000C9400000C94CD5D0C9400000C94095E9B
:100054000C9400000C9400000C9400000C9400001C
:100064000C9400000C9400000C9400000C9400000C
:100074000C9400000C94725F0C9400000C94B56016
:100084000C9400000C940000000001000200040025
:10009400080010002000400080000001000200045D
:1000A4000008001000200040008000010204081035
:1000B40020408000B803C10B80100000BC03C10BBA
:1000C400821F0000C603C10B81030000CE03C10BD5
:1000D40001040300D803C20B01060500E203C40BAC
:1000E40001800000EE03CB0B020F0000F603C50BEA
:1000F400020F0000FE03C70B020FD0120604C90B47
:10010400011000001004190C011000001A04CA0B9D
:10011400000100002204CD0B010801002C04CE0BC9
:10012400030801003A04CF0B030700004204E50B67
:10013400017F3F004C04E40B010400005604D00B83
:10014400030400005E04E30B01641E006A04D10B87
:10015400000100007604D20B000100008204E20BCF
:10016400010200008E04D30B000100009C04D40B98
:10017400020F0000A804D60B020FE703B204180C08
:100184000163000010051A0C011000001A051B0C75
:1001940001020200BE04D80B03080100C404D90BF9
:1001A40003080000CA04DA0B03080000D004DB0BC8
:1001B40003080000D604DC0B03080000DC04DD0B9C
:1001C40003080000E204DE0B03080000E804E60B69
:1001D400040A2E00F004F00B040A2E00F804FA0BB3
:1001E400040A2E000005040C040A2E0008050E0C57
:1001F400040A2E0000000000FF0000002205000297
:100204002A0504043005080736050C0536058C0656
:100214003C0580094405100B4C05500C5605400361
:100224005E05140A6805180870051C010000000228
:10023400280060009800D00008014001210C5800FB
:100244002D0B2D002B0B2B004D0A4D00808182833A
:100254008400002188898A8B8C8D8E8F310B31200C
:1002640041424300320B322044454600330B3320D5
:10027400474849004D0A4D0000000000340B34206B
:100284004A4B4C00350B35204D4E4F00360B362073
:10029400505152002B0A2B0000000000370B37206E
:1002A40053545500380B382056575800390B392011
:1002B400595A2F002D0A2D0000000000430C430062
:1002C40000000000300B3020202E2C002C0A2C00C3
:1002D400000000003D0A43520000000000004A01F3
:1002E400460032002100004B004A01460032004D16
:1002F400000096004A0146003200540000E1004A22
:1003040001460032003D0000F000000032005000C1
:100314002D0000F000500032005000470000F000B3
:10032400A000320050004B0000F000F000320050FA
:10033400002B00005800B4000400380038002138B5
:1003440003006A6100008700C800640032003D4673
:1003540003006E65696E00000800C8006400320086
:10036400215603004B004A01460032004D000000B4
:1003740001000100E60063004D0000000000A00041
:100384001B00007105D700A0001A02007105690066
:100394000000180400730569001E011906007305A6
:1003A40050726F64756B74200000537061727465D1
:1003B400202000005F4944005F52733233324944C5
:1003C40000005F526F74617465005F5461737465FB
:1003D4006E5800005F54617374656E5900005F4489
:1003E400656661756C744B6579002A436F6465308A
:1003F40000002A436F64653100002A436F6465324C
:1004040000002A4D61784D6F64756C005F4572770A
:100414004D6F64756C002A546973636845005F4DC1
:10042400795465726D4E72005F4D617374657254D8
:1004340065726D7300005F454D6F646500005F4534
:1004440043726564577472005F5273304D6F646514
:1004540000005F5634756E6435005F50756C7365CB
:1004640054696D6500005F41736B43726564697420
:1004740000005F53656E64446562697400005F4305
:1004840072656469744D6F6465005F437265646985
:10049400744D6173746572002A5461626C6553749F
:1004A400617274002A5461626C65456E64002A4668
:1004B40069727374426F6E5000002A4A6F62310091
:1004C4002A4A6F6232002A4A6F6233002A4A6F62F4
:1004D40034002A4A6F6235002A4A6F6236002A4A7B
:1004E4006F6237005F4572726F7231005F457272DE
:1004F4006F7232005F4572726F7233005F457272C1
:100504006F7234005F4572726F7235005F467265B8
:100514006967616265005F4B6F6D6D6100005461D6
:100524007374657200004C69745A00004C656974F8
:10053400540050756C7300005461737420300000D3
:1005440073657269656C6C0073657269656C2032E1
:10055400000054617374203200005461737420707D
:1005640061720000466F6C676554000053776974CC
:1005740063680000706F7274696F6E696572656E8E
:1005840000002E666F6C67650000506F7274696FAF
:100594006E656E207369636865726E004368656694
:1005A4002D4D656E75004B206C697374656E00008B
:1005B4004B206C6F65736368656E00004B2064723A
:1005C40075636B656E0054206C697374656E00000E
:1005D40054206C6F65736368656E00005420647208
:1005E40075636B656E0053797374656D0000506FAD
:1005F4007274696F6E004B726564697465004B7246
:1006040065642E436C7200006D616E2E506F7274BF
:10061400696F6E00546573740000506172616D659A
:100624007465720050726F64756B746500004B657D
:100634006C6C6E65720056656E74696C6500436F10
:100644006C6F7273000030A00531AA0532B4053313
:10065400C00534CA0535D40536E00546EA0541F23D
:100664000543FA054402064A0C060000000030EA7D
:1006740005371806391E06382806423206453A065A
:100684006342060000004572726F72004F70742E50
:100694000000496D70756C73000054696D656F7569
:1006A40074008A062F0C000500009006320C00032B
:1006B40000009606300C000500009E06310C001464
:1006C40000002E202C3041424331444546324748F5
:1006D40049334A4B4C344D4E4F3550515236535496
:1006E400553756575838595A2F390500C11100004B
:1006F4000300D90B00000300C1110300170E03000F
:10070400D90B00000500E00800000A00C1110A002E
:10071400170E0A00D90B0A00C1110A00170E28008F
:10072400D90B0000000000000000000000000000E1
:10073400000000000000000000000000070C18206A
:1007440022204D994D40114048914720222018C045
:1007540007000000070C1F3FEE3F7277727FFF7F98
:10076400777F783FEE3F1FC00700000000000000C5
:100774000C183DEE3F3FEE3F1FC80F07000200007C
:100784000000000000000000000207080F1FCE3F19
:100794001FC80F070002000000000000000000074F
:1007A400080F0F880F376F7F7FFF7F3260070F803E
:1007B4000000000000000002000207080F1FCE3FE7
:1007C4003FEE3F1AC0070F80000000000000000049
:1007D400000000000006000F0F00060000000000EB
:1007E40000000000FFFFFFFFFFFFFFFFFFF9FFF026
:1007F400F0FFF9FFFFFFFFFFFFFFFFFF0000000016
:100804000000060009108810108810090006000076
:1008140000000000FFFFFFFFFFFFF9FFF6EF77EF97
:10082400EF77EFF6FFF9FFFFFFFFFFFF0000000087
:100834000E01006A1E33286161886133001E0000C6
:1008440000000000000000078C0C186618186C0CDF
:10085400078003030C0F03000300000002000303DE
:100864008C0302CC0202800202000E1E001E0C0049
:10087400000000000C000E0B08090CC40E0B4C0900
:1008840038C478784C3103CC0301800000000202A4
:1008940002271FCC18306770306C181FC227020063
:1008A400020000000000001000181C001E1F081F9A
:1008B4001F001E1C001810000000000000000000B3
:1008C40088010388070F881F0F88070388010080A9
:1008D4000000000000000207080F1FC0020200020F
:1008E4000200021FC80F07000200000000081919C7
:1008F40088191988191988191988191980001988EB
:1009040019000000000E1F36CC6666CC6636CC1E7D
:1009140006CC0606CC0606CC0600000000081F30F4
:10092400C03030081F30CC301F8C0000CC301F800A
:1009340000000000000000000000000000000000B3
:10094400000000000E1F1FEE1F0000000200070F32
:100954008C1F0200020200020200021FC80F0700DF
:10096400021FC00000000207080F1FC0020200029D
:100974000200020200020200020000000000020263
:1009840000020200020200020200021FC80F070058
:100994000200000000000000000001080101CE3F39
:1009A40001C8010100000000000000000000000078
:1009B400000004000C1C0E3F1C000C04000000008E
:1009C4000000000000000000000000000000000023
:1009D400400040400040400E7F0000000000000046
:1009E4000000088C1838EF7F38EC180880000000ED
:1009F4000000000000000000000000000207080FD3
:100A04001FCE3F7FF0000000000000000000000047
:100A14000000000F7F3FEC1F0F8007020000000062
:100A240000000000000000000000000000000000C2
:100A34000000000000000000000000000600060F97
:100A4400000F0F000F0F000606000600000006004E
:100A54000600000000000019881919881900000018
:100A64000000000000000000000000000006060670
:100A740066063FFC0C0CC819198C7F330033330015
:100A8400000000000600061F8C3F3600363F8C1F16
:100A940006CC063FC81F0600060000000000000048
:100AA4001338387E3801C80307000E1C0E3870EE68
:100AB400600000000000070D881919801B0E001E3D
:100AC4003E063333C8313BC61E0000000E000E0E36
:100AD400000606000C0000000000000000000000FA
:100AE400000000000380060E000C1C001C1C001CEF
:100AF4001C001C0C000E0608030000001C00060766
:100B04000003038803038803038803030007060024
:100B14001C000000000000000C3636C81F0F0C3FFC
:100B24000F081F36CC360000000000000000000053
:100B34000000060006060C3F3FC006060006000043
:100B440000000000000000000000000000000000A1
:100B540000000000000E0E000E06000C0000000055
:100B64000000000000000C3F3FC000000000000037
:100B74000000000000000000000000000000000071
:100B840000000000000E0E000E0000000001000036
:100B9400370000EC010380070E001C380070600071
:100BA400000000000F8E3F30676060FB61633366B6
:100BB4006C33787036303FE80F0000000300071FE5
:100BC400001F0300030300030300030300031FEEDD
:100BD4001F0000001FCE3F707360607E0001C803D9
:100BE40007000E1C00387FFF7F0000001FCE3F70FF
:100BF40073600037000FEC0F0063006037703FEC48
:100C04001F00000001CC0307CC0E1CCC3870CC6054
:100C14007FFF7F00CC0000CC000000007FFF7F60DE
:100C24000060600C7F3FE7000033006037703FECEA
:100C34001F00000003CC070E001C3800307FCE7F5D
:100C44007073606037703FEC1F0000007FFF7F000F
:100C5400660000CC000188010300030600060C00B6
:100C64000C0000000F8C1F38E630306E381FCE3F6A
:100C74007073606037703FEC1F0000001FCE3F7040
:100C840073606037703FFF1F006E0001C8031F00D0
:100C94001E0000000000000000000E000E0E000008
:100CA4000000000E000E0E00000000000000000016
:100CB40000000E000E0E00000000000E000E0E00DC
:100CC4000606000C00CC010380070E001C38003817
:100CD4001C000E07080301CC000000000000000007
:100CE4000000000E3F3FE000000E3F3FE000000028
:100CF400000000003000381C000E07080301CC017E
:100D04000380070E001C3800300000001F8C3F7069
:100D1400E66060EC0103800706000606000006009A
:100D2400060000001FCE3F306B676FBB6D6DBB6D5F
:100D34006DBE6F67C0703FCC0F0000000600060F49
:100D4400000F0F081919881930CC3F3FC660606640
:100D5400600000007F087F61CC6060CC617F8C7F85
:100D640060E660606E607FC87F0000000F8C1F38F3
:100D7400E630600060600060600060306E381FC85C
:100D84000F0000007F087F61CC6060666060666071
:100D940060666060CC617F807F0000007FEE7F60D2
:100DA40000606000607F887F6000606000607FEEAC
:100DB4007F0000007FEE7F6000606000607F887FBE
:100DC4006000606000606000600000000FCE1F38AB
:100DD400603060006063EE636066603066381FEE0A
:100DE4000F0000006066606066606066607FEE7F92
:100DF4006066606066606066600000001F881F06B1
:100E040000060600060600060600060600061F8801
:100E14001F00000000660000660000660000660017
:100E2400006660606C703FC81F000000606E606107
:100E3400C86367006E7C007C6E0067638C6160E64B
:100E4400600000006000606000606000606000603E
:100E54006000606000607FEE7F000000606E707074
:100E6400EE7979E66F6F66666666606066606066F6
:100E7400600000006066707066786C666C6666661A
:100E840063666361EE6060E6600000000F081F396E
:100E9400CC3060666060666060666030CC391F800C
:100EA4000F0000007F8C7F60E66060666060EC7F0E
:100EB4007F80606000606000600000000F081F39E0
:100EC400CC3060666060666060666333CC391FE670
:100ED4000F0000007F8C7F60E66060666060EC7FDE
:100EE4007F8067638C6160E6600000001F8C3F7048
:100EF400E6606000703F8C1F00E600606E703FC8C3
:100F04001F0000003FCC3F06000606000606000650
:100F14000600060600060600060000006066606023
:100F24006660606660606660606660606C303FC882
:100F34001F000000606660606C3030CC3019881986
:100F440019800F0F000F0600060000006066606045
:100F5400666060666060666666666F79EE7070E60D
:100F64006000000060666030CC3019800F06000617
:100F74000F081930CC306066600000006066603095
:100F8400CC301988190F000F06000606000606006B
:100F9400060000007FEE7F00CC00018003060006FF
:100FA4000C00183000307FEE7F0000001F881F18EF
:100FB40000181800181800181800181800181F88AE
:100FC4001F00000000004060007038001C0E000785
:100FD400038C0100E7000030000000001F881F019F
:100FE40088010188010188010188010188011F88A5
:100FF4001F0000000200070F8C1D38E770603000EE
:1010040000000000000000000000000000000000DC
:1010140000000000000000000000000000000000CC
:10102400007FFF7F0000070700070600060300009B
:1010340000000000000000000000000000000000AC
:101044000000000C1F3FE6001FEE3F6066607FEE6D
:101054003F00000060006060006060086F7FCE7039
:10106400606660606E607FC87F0000000000000062
:10107400000000081F3FC6706000606006703FC833
:101084001F00000000660000660000661F3FEE714E
:101094006066606066703FEE1F00000000000000A4
:1010A400000000081F3FC6707FEC7F6000703FC8DF
:1010B4001F00000007880F1C00181800187F007F0D
:1010C400180018180018180018000000000000008C
:1010D4000000000E1F3FE670606E703FE61F006E5A
:1010E400003FC83F60006060006060006F7F8C71EB
:1010F40060CC6060CC6060CC600000000000000642
:10110400000600000E0E00060600060600061F88F4
:101114001F0000000000000188010008030388018B
:101124000188010188010188191F800F30003030C7
:1011340000303008313380373E003E37083331CC3D
:10114400300000000E000E0600060600060600062B
:101154000600060600061F881F00000000000000AD
:1011640000000008597FCE7F66666666666666661E
:101174006600000000000000000000083F3FCE3081
:101184003066303066303066300000000000000009
:10119400000000081F3FCE70606660606E703FC83C
:1011A4001F00000000000000000000087F7FCE60E8
:1011B40060666070EC7F6F8060600060000000001B
:1011C4000000000E1F3FE67060666070EE3F1F6611
:1011D40000006600000000000000000C373FE63805
:1011E40030003030003030003000000000000000DB
:1011F400000000003F7F80607F083F0188017F80FE
:101204003F00000000001818001818007F7F001825
:101214001800181800181F880F00000000000000B4
:101224000000000660606660606660606E703FE6A5
:101234001F000000000000000000000660606C3029
:1012440030C81919800F0F000600000000000000CC
:1012540000000006666666666666666F6C3F39C89F
:1012640010000000000000000000000C6071C83B8A
:101274001F000E1F083B71CC60000000000000003E
:101284000000000C3030C81919800F0F000606004A
:101294000C0C0018000000000000000C7F7F80038D
:1012A40006000C1800307FCC7F00000003CC070E32
:1012B400000C0C000C1C00381C000C0C000C0E0C58
:1012C4000703C00006000606000606000600000626
:1012D4000600060600060600060000003C003E0765
:1012E4000003030003038C010380030300030700CE
:1012F4003E3C00000000001C6C36638000000000CF
:1013040000000000000000000000000000000000D9
:10131400000006000F198C306066607FEE7F0000CD
:101324000000000000001E0060077E0700F01EF0B1
:1013340060F77EF7FBDE1F00E007FF0700F81FF8E9
:10134400E0FFFFFF00000F00E002EF0200780F78DB
:10135400E07AEF7AF7BD1F00E007FF0700F81FF8F7
:10136400E0FFFFFF23000002000010000005000062
:10137400FE0500182800FE0400182400F90F00F8E8
:101384000F0070001F71802372802A73111574116D
:101394001C75151B76151A77181C78152105010084
:1013A400FF000000013F2B02001007210000010094
:1013B400072300100000FD3000073300113068FFE0
:1013C4000000E50080000100010001020004033078
:1013D400100400000802020900000A00000C0000CA
:1013E4000D00000F00001000001107001200001390
:1013F4000000FD500010B01B110700FD5000121E2C
:1014040001FD500013001F291F00FD5000200000A3
:10141400210000FE01002B0C00FE00002B200030F8
:101424000000310603320002350701360404370692
:10143400063805013907073C00063D07085000003F
:1014440051EF00520000533F01FE01006000A7FE6F
:1014540000006000276101006A0000800000810034
:1014640000820000830000840000850000901000CA
:10147400920007930700953F039700009800000728
:101484000100FD5000072100072300FD50000773F1
:1014940001FD0000000000000000F8000000FF0053
:1014A4000000FF0000007F80001E0F80007FE7C067
:1014B400007FFFE0003FFFE00007FFC00001FFC026
:1014C4000001FF800001FF0003FFFE0007FFFC0096
:1014D40007FFF00003FFF00003FFFE00001FFFC042
:1014E40001FFFFF001FFFFF801FFFFF8007FFFF8A5
:1014F4000007FE00003FFF00007FFF80007FFF80A9
:10150400007FC100001FE000001FF000001FF0007A
:10151400000FE0000007C0000007C0000007C00083
:101524000007800000030000000300000002000028
:1015340000000000000000000000E00000000000C7
:101544000003900000000000000E180000000000DE
:10155400003808000000000000C01800000000006F
:1015640003807000000000000C01C0000001800630
:10157400300700000003C00F401C00000006E01DFF
:10158400C0700000000C3039C1C000000018187190
:10159400C7180000001C0CE1DC7C0000000E07C32F
:1015A400F1C4000000070386070600000003800E54
:1015B4001C0200000001C01C300300000000E038E1
:1015C40018010080000070700FC183C0000038E073
:1015D40003E08E6006001DC00020FC200F000F8079
:1015E40000307030198007000010003030C0000057
:1015F400001800E060600000000803806030000014
:10160400000C0E003018000000043800180C000014
:101614000006E0000C060000000380000603000042
:101624000000000003018000000000000180C000F1
:10163400C0C060C030C030C030C030C030C030C066
:1016440030C030C030C030E030703018300C30045E
:101654003FFC3FFC2564002B003E3E006B65696E39
:10166400204B726564697400436F6C6F72546F75BC
:10167400636820567320312E35300049443D0020E4
:101684002047433D00202036346B004B653A004927
:101694006E3A0043616C6962726174696F6E004FE7
:1016A4004B00546F74616C20002D2D2D2D00546956
:1016B4006E79200054696E7920626164006B6569FB
:1016C4006E20454570726F6D004D4F44554C20534C
:1016D400544F5000446174612000696E69740000C5
:1016E400533F000066616C736368657220546973CC
:1016F40063682000546973636820766F6E204B2002
:10170400004665686C6572200056656E74696C20CD
:10171400616B7469760054696D656F757400435329
:1017240049204E722000436F646520006B65696E2A
:10173400204B72656469740066616C7363686572DA
:1017440020546973636800546973636820766F6E0C
:10175400204B005831393931303000504C5520205D
:101764003A00436F6465203A005469736368203A11
:10177400004D42005053004B656C6C6E6572200046
:101784004D31004F31005350004350004459006222
:10179400757379004D5000206765737065727274BB
:1017A400002564004162726563686E756E67004B64
:1017B400656C6C6E65722000546F74616C004D6FC3
:1017C40064756C2000202000433F0073656300496A
:1017D4006D7000504C553A20005370617274653A34
:1017E40020005072313A20005072323A200046757F
:1017F4006E6374203A20005479703A20003A2056DF
:101804003A2020302B2030003A003A20544F3A201E
:10181400003A2050733A200053703A004B204D6F29
:101824006465204A6F62204A6F62466C6167730088
:101834004B20004D6F646520004A6F6220200056E3
:101844002020204572722050676C20496D7020540E
:101854004F005620005061757365004B656C6C6ECB
:1018640065723A004D49004D42004D43004D500011
:101874004D4C0074657374202E2E004F4E0025309D
:101884003258002530345800253664002533642E40
:101894002530326400253564002564002532640057
:1018A40025336400444400004B230042530042218A
:1018B40000424600542300544F004952004D5A0040
:1018C40042510042520043530056530056430049CC
:1018D4004C00426600004B23005423004245004361
:1018E40045004241004453004342002350224153E7
:1018F4004349492D492F4F222C22312E3030222C9E
:10190400323030382D30312D30313B0023482245E0
:10191400636F222C22312E3030222C323030382D7D
:1019240030312D30313B0023532245636F222C226A
:10193400312E3030222C323030382D30312D3031B0
:101944003B00504F00504632333B50550025640055
:101954002B302B303B0025640025303258002E30CC
:1019640030004F4E00006D696B726F746F75636861
:10197400000001002D4E414E00000100DE0E7619DC
:101984000000F894EE27ECBBF1E0F5BFE5BFE0936F
:101994006C00F8E1F1BDE1BD8DE0A2E0BB27ED9361
:1019A4008A95E9F780E090E1A0E0B1E0ED9301973A
:1019B400E9F7EEE7F9E185919591009761F0A5913A
:1019C400B59105901590BF01F00105900D92019716
:1019D400E1F7FB01F0CFEFEFEDBFE0E1EEBFC0E0D8
:1019E400D3E00C947A160A9902C0E1E00895E0E08D
:1019F40008951A931FEFE2E00E94C16BE3EFE1BB8D
:101A040085E38A95F1F7E0EFE1BBE4E4E093740049
:101A14000E94CA6B0E942F66E03091F4E981EE0FB8
:101A2400E0520E94CF6B41F4EDB7FEB7FA93EA930C
:101A34001F930E94D46B1F910E9440660E94D86B32
:101A4400E0E0E09371000E94D86BE12F72C30E9422
:101A5400DD6B10E01430F0F400E00430C8F4A12F82
:101A6400ECE30E94E16B0E94E56B0E94EA6BE15B90
:101A7400FF4FFA93EA930E94EF6B0E94EF6BE02F03
:101A8400EE0FEE0FE10FEA930E94AC4B0F5FE5CF30
:101A94001F5FE0CFECE0E0930F04E0E0E09310047C
:101AA4000E94F46B0E9445490E94FA6B0E94F8421E
:101AB400E030D9F40E94016C0E94016CE6E9F0E088
:101AC4000E94066C0E94016C0E94016C0E94964662
:101AD4000E94106C0E944F410E94176C0E944F415B
:101AE400EEE1F0E00E941E6CE1CF0E94FB4241C493
:101AF400E881E03011F01C9A01C01C9832C00E94A9
:101B0400016C0E94016C0E94226CEFE3F0E00E94E1
:101B1400276C08951A93A0910403A43081F4E091F2
:101B24000F04E093100410E0183048F4ABE01A9F5F
:101B3400F001E052FD4F0E942D6C1F5FF5CF42C0B3
:101B4400A0910403A43039F4E881E0931004E0E0A8
:101B5400E0930F0406C0E881E0930F04E0E0E09313
:101B64001004219608951A93A0910403A43031F12E
:101B740010E0143018F50E94316C3196E491EA9328
:101B8400DFDFE0E0E09310040E943A6C3896FA93A9
:101B9400EA93EBE0F1E00E943D6C0E943D6CFA9305
:101BA400EA930E94316CE491EA930E94316C32967C
:101BB4000E94426C0E94B9431F5FDBCF0E94456CB8
:101BC4000E944A6C199108952A970E945C7D30E026
:101BD40010E000E047ED50E028E0E091190CE0301F
:101BE40019F020E149E650E03217F0F50E944E6CFE
:101BF400E13098F10E944E6CE03870F0EEE00E9403
:101C0400546CE8E5F6E1FA93EA930E944E6CEF70A7
:101C1400EF5F0E945C6C07C0ECE0EA9391DFE8E5BB
:101C2400EE83E0E0EF830E943A6C38960E94E56B05
:101C3400E7E3F0E00E94D67AE40FF51F0E943D6CC2
:101C4400FA93EA93EDE2F0E0FA93EA930E944E6C81
:101C5400EA930E94016C0E94666C1F5F143011F4B9
:101C640010E00F5F3F5FC0CF0E94456C0E94454962
:101C74000E94637D619608950E946C6CECE0EA9387
:101C84005FDF0E94F46BEBE0EA935ADF0E94706C12
:101C94000E94756CEAEAF0E00E947A6CE0913A0CDA
:101CA400F0913B0CE491EA93E0913A0CF0913B0CF7
:101CB40031960E94816C0E94B94301E00E94846CB9
:101CC4000E94876C11F00F5FF9CF0E94956C031787
:101CD40018F4E0E0E093C0050E94956C11E00E94C6
:101CE4009C6C0E94876C11F0153008F021C00E9492
:101CF400706C0E949F6CE0E4F0E00E94D67A349607
:101D0400FA93EA93E2EEF0E00E947A6C0E949C6CF3
:101D14000E94A26CE491EA930E949C6C0E94A26CC3
:101D240031960E94816C0E94B9433F5F1F5FD7CFF9
:101D34000E944A6C0E94657D36C427970E945C7D90
:101D440022E354E0A0910403A43011F426E453E008
:101D540010E0143010F00C94FA0E00E0051710F0A7
:101D64000C94F80EE12FEE0FEE0FE00F3E2F0E94C1
:101D74009C6C0E94AE6C3196E4910E94546C0E945B
:101D84009C6C0E94AE6C3296FA93EA930E94C068EF
:101D9400ED85E03039F4AF81A13210F4E0E0EF8357
:101DA400E0E0E887A02FBB27E22FE85FF0E00E9485
:101DB400D67A3896FA93EA930E949F6CEAE3F0E0AD
:101DC4000E94D67AE55BFF4F0E94B36C0E943D6C83
:101DD400FA93EA930E949C6C0E94AE6CE491EA939D
:101DE4000E94016C0E94666C0F5FB8CF1F5FB1CF79
:101DF4000E944A6C0E94637D2E96089522970E9449
:101E0400B86CA13059F40E94BD6CABE2B1E00E9401
:101E1400017B2E2F57E1E2ECF0E008C00E94BD6C7C
:101E24000E94C16C2E2F53E0E7EEF0E0EE83FF83B7
:101E34000E94C66CA0911908A13081F4E9ECF0E08D
:101E44000E94DD6C0E94E46C0E94E96CEBE2EA9370
:101E5400EBE5F6E10E94426C0E94B943E3E0F0E056
:101E64000E94DD6CEA85FB850E94EF6C0E94F26C97
:101E74000E94F66C3F5FE091C10BAFEE0E94E07AE6
:101E8400F0E0EE83FF8311E0E091C20B1E17B0F582
:101E940000E0E091C10B0E1778F50E94FC6C49F14B
:101EA4000E94036DE09310040E94846CAE81BF8194
:101EB4000E94D67A33960E94B36C0E949F6C0E9453
:101EC400D67ADF010E940D6D0E94106DEA85FB85B4
:101ED40034970E94EF6C0E94F26C0E94F66C3A9365
:101EE4000E94E220EF3F29F0ADE05A9FF0010E94EA
:101EF400156D3F5F0F5FCDCF1F5FC6CF0E94456C4E
:101F04000E944A6CC8C022970E945C7DE2E5F7E01B
:101F1400EE83FF8340E0443190F4AE81BF8111969B
:101F24000E941D6D1396EFEFEC93AE81BF81EC938D
:101F3400EE81FF813496EE83FF834F5FECCFE09117
:101F4400C10BA0EF0E94E07A2E2F0E94BD6CA0E48A
:101F5400B1E00E94017B5E2F0E94C66C21FE23C06B
:101F64000E94226D0E94226DEFEAF0E0FA93EA9358
:101F74000E94276D0E94F26C0E94F66C0E94FA6B1C
:101F8400E6EBF0E0FA93EA930E94226D0E94E46C7F
:101F94000E94276DEFE7EA93EDE5F6E1FA93EA9301
:101FA400E0E0F0E011C00E94226D0E94226DE8EE94
:101FB400F0E0FA93EA93E52F0E942D6DFA93EA93E9
:101FC4000E94F26CEAE8FBE0FA93EA930E94B943B8
:101FD4003F5F11E0E091C20B1E1710F00C94471004
:101FE40000E0E091C10B0E1710F00C9445100E9414
:101FF400FC6C11F40C944210A0919A0BE0E8EA23D3
:10200400E03821F0A091E20BA23019F40E94036D94
:102014000AC00E94306DE03011F4E0E001C0E8E055
:10202400E0930F04E7E0E0931004A02FBB27E22F16
:10203400F0E00E94D67A3396FA93EA930E940D6DEB
:102044000E949F6C0E94D67A33960E94EF6C0E9485
:10205400276D0E94F26C0E94F66C4E2FA0911E0810
:10206400E32F0E94356DEA0FFB1F43833A930E94CE
:10207400E220EF3F29F0ADE04A9FF0010E94156D88
:102084003F5F0F5FAECF1F5FA5CF0E94456C0E94DC
:102094004A6C0E94D9350E94637D28960895E1E038
:1020A400E0930D04E2E0E0930E04E0E0E09310041A
:1020B400ECE0E0930F04ECE5F3E00E942D6CEAE021
:1020C400E0930F04EAE4F3E00E942D6C0E9445497A
:1020D40008951A93A981A43029F4A0E021FCA1E079
:1020E400A03009F426C0E9810E943C6D0490E98186
:1020F4000E94426DE491A02DAE1BA2501A2F0E94A3
:10210400FA6BE4EBF0E0FA93EA93EB810E94426D00
:102114000E94897B3296FA93EA93EAE3F0E00E9404
:102124004A6DEFE7EA93EDE5F6E10E94426C0E9406
:10213400B9431881229608950E94DD6BE0E0EA938A
:102144000E94DD180E94306D0E2FE4E3F2E00E943D
:10215400897B33971E2F0E94016C0E94016C0E94A0
:10216400226C0E94516D0A930E94AC4B0E94EF6B4B
:102174000E94566D0E94B146E2E0E0930E04E091A5
:10218400980BEF70E09310040E945B6DEFE0E09316
:102194001004AA81A13051F40E94636D0E94756CF1
:1021A4000E949646E0E6F6E10E94686D21FE0DC0AD
:1021B400E4E0EA938EDFECE3F2E00E946C6DEEE380
:1021C400F2E00E946C6D0E946049A4DC80C0E8814A
:1021D4000E94426D0E946C6DEA810E943C6D0E94D7
:1021E4006C6D0E94EE46E881EA9373DFCAC11A93CC
:1021F4000A93EC81EA93EBDF1AEEEC810E943C6DCA
:102204000490EC810E94426DE491A02DAE1BA2507B
:102214000A2FAC81A43029F4A0E021FCA1E0A03075
:1022240009F409C01EEAAA81BB811B96E0E0EC9385
:10223400EC81EA934EDF0E94036DE0931004EC817D
:102244000E94716DFF93EF930E94226DEE810E94B4
:10225400426D0E94897B31960E944A6D0E94846C73
:10226400FA93EA93EC85E058EA930E94016C0E9489
:10227400776D0E94B943AF91BF91EC93EC810E94BA
:10228400426D0E946C6DEE810E943C6D0E946C6DEB
:102294000E94604919810881259608950E947C6DE9
:1022A4000E94C16C8F010E94016C0E94016C0E940B
:1022B400226C0E947F6D0E94636D0E949646EA81A3
:1022C400EA930E94DD180E945B6D0E94866D19815D
:1022D4000881239608950E947C6D0E94C16C8F0131
:1022E4000E94016C0E94016C0E94226C0E947F6D0E
:1022F4000E94636D0E949646EC81FD810E94686D88
:10230400AA81BB810E94527D24F4A030E0E1BE0783
:102314000CF006C0EA81FB81FA93EA930E945841CB
:10232400AA81BB81A130E0E1BE0724F0A030E1E145
:10233400BE070CF00AC0A6EEBBE0EA81FB81E150C7
:10234400F0410E94906D0E94986D0E94866D1981E3
:102354000881269608950E947C6D0E94C16C8F01AD
:102364000E94016C1A930A930E946049E0E0E09392
:102374003C0C099119910895E881EA930E94DD18B3
:102384000E94BE1FE03051F10E949E6D0E94016CBC
:102394000E94A26D0E945B6D0E94A66DE881EA9383
:1023A4000E942921E8830E94AA6D3B9734F00E9481
:1023B400AA6D0E94B56DE9E40BC0A3EEB6E00E94DD
:1023C400B96D0E94BC6D0E94C16D0E94C66DE3E7A9
:1023D400EA930E943446E2E0E0930E04D2C00E94E5
:1023E4002F68E0E0E0930F04A0910403A43019F4F3
:1023F400E8E6F3E002C0E4E7F3E0FA93EA930E942C
:10240400994308950E94BD460E942F680E948468E3
:10241400E1E0E0930D040E949E6DE6E0F0E00E948E
:10242400CA6DECE6F6E10E94686D0E94016CE7E07B
:10243400F0E00E94CA6DEFE7F6E10E94686D0E9429
:10244400CE6DEA930E946541E3E8F6E10E94686D6F
:10245400E0910403EA930E946541E9E8F6E10E94F1
:10246400686D08952A971A930A930E94016C0E943A
:10247400016C0E94226CE4E6F0E00E94276C00E00C
:1024840010E01530B0F4053020F40E94D36DE03034
:1024940009F40DC00E94016C0E94846C0E94CA6DF4
:1024A4000E94DA6D0E94D36D0E94DF6D0F5F1F5F83
:1024B400E8CF0E94E16D0E949646EFE8F6E10E94A3
:1024C400686DE0913108EA930E9465410E94706C46
:1024D4000E94636D0E949646E3E9F6E10E94686DEE
:1024E400E0912306EA93E5E0EA930E941B41E09120
:1024F400190CE03079F10E94706C0E94566D0E94B4
:102504009646E09128060E94E46D0E94226D0E9486
:102514009646E0912806E295EF70E695E695AE2F93
:10252400E0912906EE0FEE0FEA0F0E94E46D0E947F
:10253400756C0E949646E0912906E295EF70AE2FE5
:10254400E0912A06E295E07FEA0FEA93E6E0EA9357
:102554000E941B410E94706C0E94566D0E94964618
:10256400E0913F0CEA930E946B41198108817DC17F
:10257400E881E064E7B9369A349BFECF349AE4B13B
:10258400F5B121960895E881F981AA81BB81AE173E
:10259400BF071CF4EA1BFB0B06C0A881B981EA81C2
:1025A400FB81EA1BFB0B2496089528970E945E7D0D
:1025B400EFE0E0936100E1E0E09362000E94CA6B07
:1025C400E5E0E09361000E94CA6B0E94EA6DE0932B
:1025D4006F05F0937005E0917B05F0917C05E09325
:1025E4006D05F0936E05E1E0EA93C2DFE0937B05AD
:1025F400F0937C05EFE0E0936100E8E0E093620093
:102604000E94CA6BEAE0E09361000E94CA6B0E94D8
:10261400EF6DE0936B05F0936C05E0917905F09113
:102624007A05E0936905F0936A05E0E0EA93A0DF98
:10263400E0937905F0937A050E94EF6DA0916B0504
:10264400B0916C05EA0FFB1FA0917905B0917A0552
:102654000E94F46D8F010E94EA6DA0916F05B09104
:102664007005EA0FFB1FA0917B05B0917C050E94C9
:10267400F46D9F01E0916B05F0916C050E94FB6D78
:10268400FF93EF930E94EF6D0E94FB6DAF91BF919A
:10269400EA0FFB1FFF93EF93E0917905F0917A0520
:1026A4000E94FB6DAF91BF91EA0FFB1FE09375058C
:1026B400F0937605E0916F05F09170050E94016E2C
:1026C400FF93EF930E94EA6D0E94016EAF91BF9158
:1026D400EA0FFB1FFF93EF93E0917B05F0917C05DC
:1026E4000E94016EAF91BF91EA0FFB1FE093770543
:1026F400F0937805A0917505B0917605E4E1F0E0DA
:102704000E94A87A0E2EA0917705B0917805E4E195
:10271400F0E00E94A87AE02919F00E946945A3C05C
:10272400009371051093720520937305309374051B
:10273400A0916405A63428F4E0916405EF5FE0936A
:1027440064050E94076E989724F40E940C6E989773
:102754000CF00EC0A0916405AA3019F4E1E0E093F6
:102764006105A0916405A83219F4E2E0E0936105E3
:102774000E94076E999724F00E940C6E99970CF4AE
:1027840072C0E0916705EF5FE09367050E94116EE8
:102794000E94076E0E94166E0E941D6E0E94226E99
:1027A4000E94DB7A7F936F93FF93EF93A2E0B0E0F4
:1027B4000E94A47B0F010E94116EDF01F001EA1B4D
:1027C400FB0BAF91BF918F919F910E942B6E0E9442
:1027D4001D6E0E94306E0E940C6E0E94166E0E9446
:1027E400356EAC81BD818E819F81EFE3F1E060E0C5
:1027F40070E00E94DB7A7F936F93FF93EF93A6E0E0
:10280400B0E00E94A47B0F010E94306EDF01F00152
:10281400EA1BFB0BAF91BF918F919F910E942B6E8E
:102824000E94356EE0911204E03049F4E885F985A0
:10283400E0935905F0935A05EC81FD810AC0EC81BF
:10284400FD81E0935905F0935A050E94226E0E947F
:10285400707AE0935B05F0935C050E94106C0E9413
:10286400176C0E94F1440E94657D2C9608951A937A
:102874000E94BD46E2E0E0930E04E2E3F0E00E9431
:102884003D6C0E943A6EE7E9F6E10E94686DE4E16E
:10289400EA930E94C440E0E9F1E00E943E6EE4E164
:1028A400EA930E94C440A0916705A13010F0A89556
:1028B400FACF10E0143010F00C94B614E2E0E09378
:1028C4000D040E94426EDF010E946C6DFD01329680
:1028D4000E946C6D0E94B1460E94426E3496E4914F
:1028E400EA930E943446E1E0E0930D04A091670569
:1028F400AF3110F4A895FACFEAE0EA930E94C440FD
:102904000E94426EDF0135960E94897BBF01FD0162
:102914000E94486EDB010E94B47B0E944F6E0E94AD
:102924009F6CE8E2F0E00E94D67AE65AFF4F0E94DC
:102934003A6E0E94426E0E94486E0E94B56DA0914C
:102944006705AE3110F0A895FACF0E94426EDF0100
:102954000E946C6DFD0132960E946C6DE8E1F0E01E
:102964000E94066C1F5FA6CF0E944F6EEAEFF0E054
:102974000E943A6EE3EAF6E10E94686DE0EDF7E04A
:102984000E943E6E0E94BD464DC10E94546E0A9341
:10299400E4E6E2BF78940E94B34407DEE6B3AFEF07
:1029A400EA27E0933108A2E6BBE00E94636EE0915F
:1029B400620BE77031F4A0910A04E0E4EA27E093A3
:1029C4000A04E091620BEF7131F4A0910A04E3E888
:1029D400EA27E0930A040E94FD650E94CA21E2B33B
:1029E400EF700E2EA0911408B0911508EFE0F0E0FE
:1029F400AE27BF27EA23FB230E94897AE029E2BBA2
:102A0400E0911408E07111F41D9A01C01D98099118
:102A1400199115C00E94546EE6E0E4BDE0B1E29560
:102A2400EF70AE2FE0916300E071E15FEA231E2FA7
:102A34000E94516D0E94A1210E94D7651991E991CC
:102A4400EFBFF991E991B991A991999189917991FE
:102A54006991F9901990099018950E9401650E9456
:102A640087650E94F2500E94FA1E08951A93A89551
:102A74000E94CA42E13011F00C949915E091C60508
:102A8400E1501E2FA091C505A13021F40E94696E6A
:102A9400E03009F40CC0ADE01A9FF001E15FFC4F97
:102AA400BF01E081E260DB01EC930E94706EA091B3
:102AB400C505A23011F0A43089F40E94696EE09338
:102AC400DB050E94756E31F0FD01E15FFC4FE08192
:102AD400E27009F403C01A930E947E6EA091C505AA
:102AE400A33019F41A930E947A27A091C505A53042
:102AF40029F4E091C605EA930E94B127A091C50587
:102B0400A830A9F4E0E0EA93E091C605EF77EA93F0
:102B14000E94B0181E2F1F3F51F0E0E0EA930E947C
:102B2400C440E12FE058E093DB05E0932D06E091EB
:102B34000A04E078D1F0E0910A04EF77E0930A0404
:102B44000E948949E0910A04E07131F0E0910A049D
:102B5400E270EA930E949B45A0913208A13328F0C9
:102B6400E2E0EA930E94FB0C1E2FA0913C0CA130E2
:102B740039F4E0913D0CF0913E0C0E94826E09F410
:102B840001C0E9DB6ADF4EC01A930E94BD46E1E052
:102B9400F0E00E94426C0E94964610E00E948C6E07
:102BA4000E94016C0E94516D0E949646E09121089A
:102BB400E03049F4E6EAF6E10E94686D0E94926E04
:102BC4000E94C66D1E5FA0912108A130F0F0E09133
:102BD4002108E150EA930E940C19A091B30BAD3285
:102BE40029F40E949B6E0E944E7D79F0E3EBFBE09A
:102BF4000E94986DE6E0F0E0FA93EA930E94A86ED2
:102C04000E949B6E0E94C66D1E5FE0912108EF5FDB
:102C1400E09321081C3020F4A0912108AB3008F087
:102C240001C0BECF199108951A930E94BD46E9814F
:102C3400E03019F4E0E0E0931E08A981A230A9F481
:102C440010E0A0911E08A13010F01C3008F00DC057
:102C5400E0911E08E150E0931E080E94AC6E19F446
:102C64000E94BA6E09F01F5FECCF0E948C6E10E0D8
:102C74000E94016C0E94516D0E949646A0911E080C
:102C8400A03408F50E94AC6E19F40E94BA6ED1F01B
:102C9400E0911E08EA930E94DD180E945B6D0E9479
:102CA400016C0E94A86E0E94C56E0E94B56DE8E793
:102CB400EA930E9434460E94A66D0E94CA6E0E9446
:102CC400C66D1E5F05C0EDEAF6E10E94686D1E5FE9
:102CD400E0911E08EF5FE0931E081C3020F4A091E1
:102CE4001E08A13408F001C0C3CF188122960895AC
:102CF400E0E0E5BFE0936D00E0936C00EBBBEFEF29
:102D0400EABBE0E0E8BBE7BBE5BBEFEFE4BBE0EF29
:102D1400E2BBE1BBE0E2E3B9ECEBE2B9E0E0E09373
:102D24006200E0936100EFE0E0936500E0936400EB
:102D3400E0E0E0BFE7E0E3BFE4E6E2BFE0E0E1BFFC
:102D4400EFBDEEBDEDBDECBDE7BDE6BDEBBDEABD3F
:102D5400E9BDE8BDE0937900E0937800E3E0E5BDE8
:102D6400E6E0E4BDE0E0E3BDE0938B00EAE0E0935D
:102D74008A00E0E0E0938900E0938800E09381001A
:102D8400E0938000E2E1E0938700E4E3E0938600CF
:102D9400E0E0E0938500E0938400E0938300E09317
:102DA4008200E0936A00E0E3EABFE0E4E9BFE8BF41
:102DB400E1E4E7BFE0E0E0937D00EBB9E8EDEAB9D8
:102DC400E6E0E0939500E0E0E0939000E7E6E9B9FF
:102DD400E0E0E0939B00E8EDE0939A00E6E0E09306
:102DE4009D00E0E0E0939800E3E3E0939900E0E8DD
:102DF400E8B9E0E0E0BDE0E4E7B9E7E8E6B9E0B56A
:102E0400EF7EE0BDE0E2E0937000E0E0E09372006A
:102E1400E4E4E0937400EFE1E1BDEFE0E1BD0E9482
:102E2400AA5D0E94484B0E948C4578940E94484BAE
:102E34000E948C45E1E0EA930E947A0D0E94CE6DD7
:102E4400E53128F0A9E0B0E0E0E00E94BC7BDADAEA
:102E540021E030E0E0E0EA930E94FB0CE0933208CA
:102E6400EAE0F0E00E943E6E3F5FA0913208A43594
:102E740011F03A3008F001C0EDCF0E94636D0E945A
:102E8400706C0E949646A0913208A43581F4E1E06A
:102E9400EA930E94FB0CE0933208E2EBF6E10E9415
:102EA400686DE0913208EA930E94344607C0E0E07E
:102EB400E0933208E8EBF6E10E94686D94D0E030CC
:102EC40059F40E94636DE9E0F0E00E94CA6DE1EC00
:102ED400F6E10E94686D20E00E94116E0F01A2E0ED
:102EE400B0E00E94A47B0E161F0654F40E94306EBC
:102EF4000F01A6E0B0E00E94A47B0E161F060CF0A2
:102F0400B6DC203071F40E94636DEAE0F0E00E94C8
:102F1400CA6DEDECF6E10E94686DA8950E94D36E2F
:102F2400FCCF0E94C0360E94636DE9E0F0E00E948D
:102F3400CA6DE8EDF6E10E94686D0E94841BE030E2
:102F440019F0EEEDF6E102C0E3EAF6E1FA93EA9352
:102F54000E944B460E940F66E1E0EA930E94C4403F
:102F640000E010E00436E0E01E0724F40E948765C8
:102F7400E03009F007C0EAE0F0E00E943E6E0F5F27
:102F84001F4FF0CF0436E0E01E072CF0A091670538
:102F9400AF3108F06CDC6ADD0E941D320E94B61D60
:102FA400FACFFFCF0E94D66E17FD02C0103011F485
:102FB400E0E063C3E12F61C30E94D66E17FD10E009
:102FC4001A3008F41F5F0E94E36E57C30E94D66E46
:102FD40017FD02C0103011F4E0E04FC311500E94FD
:102FE400E36EE1E04AC31A930A9310E0E4E6F0E0EA
:102FF4000E943E6EA8950E942F66E03021F4E0EA1C
:103004000E94EE6E09F002C001E001C000E00E94DF
:1030140040661F5F003011F4153008F001C0E6CFA0
:10302400E02F0991199108950E94F36E43C40E9400
:10303400F36E0E94006F0895A881B9810E94527DA9
:1030440024F4A83EE3E0BE070CF005C00E94066F1E
:103054000E94A26613C3E0E011C3A881B9810E9453
:10306400527D24F4A83EE3E0BE070CF005C0EA81DB
:10307400E03011F4EFEFEA830E94066FED81EA93EA
:103084000E94CE6660C10E945E7D20E030E0283E52
:10309400E3E03E077CF4A8953A932A93CDDF1E2FF4
:1030A4001F3F29F0EFEFEA933A932A93D6DF2F5F7D
:1030B4003F4FEDCF0E94657D4FC01A930A93E0E025
:1030C400F0E0E093400CF093410CAA81A03468F442
:1030D4000E940F6FE55FFB4F8F010E94166F1A93DA
:1030E4000A93E0E4FCE00E94196FE091400CF09137
:1030F400410C27C11A931FEF1F5F1A93DEDFA981CA
:10310400BA81EA17FB0711F0113408F001C0F4CFBB
:10311400E12F188118C11A930A93A091C10BE09171
:10312400C20BEA9FF001A0911E08EA0F0E2F013492
:1031340008F00FE310911E08101758F41A93BDDF1E
:10314400AA81BB81EA17FB0711F4E12F03C01F5FBB
:10315400F3CFEFEF19810881249608950E945C7DD6
:1031640010E0103418F50E949F6CE8E2F0E00E9431
:10317400D67AE050FC4FAF01E0EAEA93FA01709688
:103184000E941D6FEC713E2FE0EAEA93FA013F962C
:103194000E941D6F0E2FEF81E31719F4EE81E017E3
:1031A40009F002C0E12F03C01F5FDBCFEFEF0E94E5
:1031B400637D289608951A930A93E091890BAA8156
:1031C400EA17C1F0A03468F40E940F6FE050FC4F7E
:1031D4008F010E94216F0E94196FEA81E093890B8D
:1031E40009C0EFEFE093890B0E942C6F0E94316FAE
:1031F400E093940BA6C01A930A930E940F6FE050B9
:10320400FC4F8F01AA81A03420F40E94216F0E94F8
:10321400006F97C01A930A93E091B20BAA81EA1740
:10322400A1F00E943B6F40F40E94476F0E94196F07
:10323400EA81E093B20B09C0EFEFE093B20B0E9476
:10324400526F0E94316FE093BD0B7BC01A930A93B7
:103254000E943B6F20F40E94476F0E94006F71C070
:103264001A930A93E091330CAA81EA1761F10E9440
:10327400576F18F50E94166F1A930A93E4E3FCE063
:103284000E94196FEA81E093330CE0E0E0932B068F
:10329400A091350CA13020F0A091350CA83008F095
:1032A4000BC0A8EDBBE0E091350C0E94616FAE0F3E
:1032B400BF1FEC91E0932B0606C0EFEFE093330CB5
:1032C400E0E0E093340C3DC01A930A930E94576FD8
:1032D40040F40E94166F1A930A93E4E3FCE00E9400
:1032E400006F2FC01A930A93E0912E0CAA81EA175B
:1032F400C1F00E94646F70F4E0EAEA930E94756C76
:103304001A930A93EFE2FCE00E94196FEA81E093BA
:103314002E0C07C0EFEFE0932E0C0E946E6F0E94FC
:1033240095680FC01A930A930E94646F50F4E0EA00
:10333400EA930E94756C1A930A93EFE2FCE00E94F0
:10334400006F19810881239608950E946E6F0E9470
:103354009568E881EF5FE093300CD2C124970E9416
:103364005C7D0E94756F0E949568AA85A03478F5EB
:10337400AB85A13010F0A63008F007C0EB850E94A1
:10338400616F0E947C6F0E948F6FEB85E030F9F4CF
:10339400E0E0EE83EF83E887E98740E050E020E057
:1033A40030E02530E0E03E0784F4F9010E947C6FB0
:1033B4000E948F6F0E94C56E4E0F5F1F0E94CA6EDF
:1033C4000E94946F2F5F3F4FECCF0E949F6F3FC1CD
:1033D4001A930A93AB81A13010F0A63008F01CC0F8
:1033E400EB810E94616F0E948D7A0E94897ADF01CD
:1033F400EA810E94B06FE8E0F0E00E94D67AE050E3
:10340400FA4E8F01E0EAEA930E94706C1A930A93D1
:10341400ECE1FCE00E94006F198108810C94F81E15
:103424000E945E7DEC810E94B46FE83109F459C0BA
:103434000E94B96F309729F00E94B96F0E94BE6F45
:10344400EC830E94B21F0E2F10E0101710F00C94A2
:10345400731A0E94C26F82DFAEE1BCE00E94636E09
:10346400A091200CB091210C8091220C9091230CFE
:103474000E94C76F0E946B7AE093200CF093210C9A
:103484006093220C7093230C0E94C26FA1DFE0EAC8
:10349400EA93EE810E94616FEE0FFF1FE050F04F40
:1034A4000E941D6FE270D9F4ED81E093240C0E9418
:1034B400B96F309751F40E94CE6D0E94CE6FEF5ECB
:1034C400F84DDF010E94D46F02C00E94B96FE093EF
:1034D400250CF093260C0E94D96F0E94DE6F1F5FAB
:1034E400B4CF0E94657D269608951A930A930E948C
:1034F400E46FECE2F0E00E94EB6F0E94EF6F0E9439
:10350400F46F10E01034D8F41A9355DEE0912208D9
:10351400EA931A9323DF0E94FD6FEA0FFB1F0F014A
:103524000E94FD6F0E940570DF01CB010E94CA6EEC
:103534000E946B7AD0010E94847B1F5FE3CFA0912D
:103544001908A330B9F500E00031A0F50E94846C9D
:103554000E940A7069F510E01A3050F5E02FE05D22
:10356400EA93E4EEF6E10E940F70E12FE05D0E9421
:103574001670E1F40E941B700E942270EA0FFB1F78
:10358400FF93EF930E9422700E9405707F936F93C4
:10359400FF93EF930E94F361AF91BF918F919F913D
:1035A4000E946B7AAF91BF910E94847B1F5FD4CF3E
:1035B4000F5FCACF10E01A3090F40E9422700E946C
:1035C4000570A0912908B0912A0880912B08909148
:1035D4002C080E946B7A0E94F46F1F5FECCF0C944E
:1035E400401F24970E945C7DEA85EA9366DD9F0173
:1035F400022E032A39F13A932A937CDD1E2F40E0F0
:1036040050E0E0E0EE83EF83E887E987AA851A17A4
:10361400B1F4012F003498F40A934FDD2E173F07BD
:1036240061F4EB85EA930A9399DE0E94C56E4E0F0E
:103634005F1F0E94CA6E0E94946F0F5FEBCF0E94BF
:103644009F6F05C0EB85EA93EB85EA9387DE0E94C2
:10365400637D2C9608951A93A895A981A63068F4E1
:103664000E94756F0E94956810E0103430F4E9816F
:10367400EA931A93ADDE1F5FF8CF1881229608955E
:103684001A9311E0163020F41A93E5DF1F5FFACF86
:1036940067C3E1E0E093340CE093350C31C0A895A6
:1036A4000E94526FEEEAF3E0FA93EA930E94706C80
:1036B4000E942970E093BB0B0E943270E093BC0B14
:1036C400E0E0E093BD0B1CC0A895E9E8FBE00E9494
:1036D4003970E9E2F0E00E94EB6F0E942C6FE4EA9B
:1036E400F3E0FA93EA930E94706C0E942970E093CD
:1036F400920B0E943270E093930BE0EBE093980BF3
:10370400219608950E945C7D0E943E70E03228F06C
:10371400AAE0B0E0E0E00E94BC7B00E085DCA09180
:10372400BE0BB091BF0BA633E2E1BE0741F110E03E
:103734001A3030F41A93B3DF1A9388DD1F5FF8CF81
:1037440010E0103430F41A93BFDF1A9354DD1F5F76
:10375400F8CF10E0103830F41A939BDF1A93B4DDDD
:103764001F5FF8CF8DDFA9E0B0E0E0E00E94BC7BF2
:10377400E6E3F2E1E093BE0BF093BF0B01E010E04F
:10378400183210F00C94171C0E9443709F010E9481
:103794004370AF010E944D703496E491E03011F013
:1037A400E13069F4D901AC910E944D703596E491F1
:1037B400EA1720F40E944D700E94547034C0E23025
:1037C40091F4DA010E947A7BE031A7E2FA0714F45B
:1037D400FF2342F40E944D7036960E94897BDA01E1
:1037E400ED93FC9320C0E33049F4D901AC91AF3F91
:1037F40021F40E944D700E94547015C0E43099F475
:10380400D901AC91AF3F79F400E00E944D70359638
:10381400E4910E1740F40E944D700E9454702F5F83
:103824003F4F0F5FF2CF1F5FABCF01DC10E01530CD
:1038340060F41A9357DDA0912F0CA63020F01A9350
:1038440084DD1A936FDD1F5FF2CFE02F0C94C82044
:10385400E881EF5FE883A881A43610F0E0E0E88314
:10386400E8810C9441210E94B96DA5E0B0E00E946A
:10387400D67A30960C944121A091370CBB27E09165
:10388400360CA6C0F9DF329774F00E945970E091AB
:10389400360C0E9460700E94006FE091360CEA932F
:1038A400D7DFE093360C08950E945970E091370CED
:1038B4000E946070FA93EA930E94EF660895E4E22E
:1038C400FCE00E9468700E945970E091370C0E94DD
:1038D40060700E94006FE091370CEA93B9DFE093C7
:1038E400370C08950E945E7DE0E0E093360CE0938F
:1038F400370C10E030E0343680F5A8950E945970FA
:103904003A93B1DFFA93EA93E4E2FCE00E94196F80
:1039140000E0A091240CA13010F0A03808F001C000
:1039240001E0E12FE03041F4013029F43093370C09
:103934003093360C11E00FC0E13031F4003019F44B
:103944003093360C12E007C0E23029F4013019F448
:103954003093370C13E03F5FCECF46C21A93A09149
:10396400CF0BA870B9F010E0E981FA810E949F6C36
:10397400AE17BF077CF4ED81E093240CEB81FC814E
:10398400E851FC4F0E946F70E0E0F0E00E94DE6FAF
:103994001F5FEACF18810C94CA20E881EF5FE883A7
:1039A400A881A43610F0E0E0E883E8810C9441217A
:1039B400E881E150E883A881A43610F0E3E6E883C7
:1039C400E8810C944121A091390CBB27E091380C7B
:1039D400F0E031960E947470EC59FF4FDF01E4E689
:1039E400F0E00E94337B08950E94B96DA5E0B0E039
:1039F4000E94D67AE050FE4F0C944121E9E2FCE0AB
:103A04000E946870E881EA93BBD10C9441211A9317
:103A14003ADBE1E0E093860BA3C1A89510E01436ED
:103A240080F41A93A6D1A091290CAF3F31F40E94DF
:103A34007970AF3FEFEFBE0711F01A93DFDF1F5F1E
:103A4400EECF0E947E70689420F88AC10E945E7D49
:103A54001091390CAD81AA23CAF5E091380CE11715
:103A640019F0AD81AA230AF030C01A9382D10E94C2
:103A74007970EE81FF81EA17FB0729F4E885A091AC
:103A8400290CEA1709F01EC00E948470EC81FD81A4
:103A94000E94757AEA17FB0744F40E9489700E9419
:103AA4009270E0E0EC83ED830BC00E948970EC839C
:103AB400FD83E0E0F0E00E949270E0E0E093290CE6
:103AC4001A935ED10E949770C8CF46C0E091380C1B
:103AD400E11729F0AC81BD810E94527D0CF01BC01E
:103AE4001A9347D10E947970EE81FF81EA17FB0790
:103AF40029F4E885A091290CEA1709F009C00E946D
:103B040089700E9492701A933BD1E0E0EC83ED83BC
:103B14000E949770DBCFAC81BD810E94527D1CF462
:103B240052DF33970CF418C0E885E093290CEE813A
:103B3400FF810E949C70EC81FD810E949270E09153
:103B4400380CEA931DD1E091380CEA9326DFE09318
:103B5400380CE0E0EC83ED83689420F8EC81FD817F
:103B64000E94657D299608951A93A091420CA03075
:103B740059F4E091450CF091460CFA93EA93E8EB82
:103B8400FBE00E94A17009F40BC0E1E0E093420C59
:103B9400E091380CE093440CE091380CE093430C32
:103BA400A091420CA13011F00C94341EE091390C18
:103BB400A091440CEA1711F40C94251EE091440CD6
:103BC400EA93F6DEE093440CEA93D3D0A091290C57
:103BD400A13010F0A03808F035C0E091430CEA930E
:103BE400E7DEE093430CA091440CEA1759F1EA9301
:103BF400C7D0E091E20BE030E9F410E01530D0F4E6
:103C0400ABE01A9FF001DF01E352FA4FE081E030AC
:103C140049F0FD01E452FA4FE081AE2FE091440CEB
:103C2400EA1709F005C00E94A770A091430CA08375
:103C34001F5FE4CFE9E2FCE00E946870E091440C6D
:103C4400EA939ED00FC0E091430CE093390CE0E07E
:103C5400E093420C689420F80E940968E093450CB4
:103C6400F093460C7DC01A93A8951091390CE091FD
:103C7400380CE117C1F00E94AD700E94527D64F4CB
:103C8400EB81A091290CEA1739F40E947970E9813B
:103C9400FA81EA17FB0709F003C0E12F1881A6C0D7
:103CA4000E949770E4CFEFEF1881A0C00E94847047
:103CB4000E94527D84F4E0912B06E87031F4E09187
:103CC4002F08A091290CEA1731F40E94B1700E94C8
:103CD400BE6FE03408F001C05CC10C949F21A8952C
:103CE400E091380CA881EA1761F0E8810E94B6706F
:103CF40019F0E8810C944121E881EA934EDEE883CF
:103D0400EFCFEFEF0C9441211A93A8951091390C41
:103D1400E091380CE117E1F00E94AD700E94527DF1
:103D24008CF4E0912B06E87031F4E0912F08A09117
:103D3400290CEA1739F40E947970E981FA81EA17AB
:103D4400FB0709F002C00C9486210E949770E0CF13
:103D5400EFEF0C9487211A931091390C1A93BFDF5B
:103D640019910895E881EA9318DEE883EA93B7DFAE
:103D740086C20E9459700E94BD700E94196F7FC252
:103D84000E9459700E94BD700E94006F78C20E9408
:103D94005E7D0E947E7010E030E0343628F5A895F0
:103DA4003A93E7DF00E0A091290CA03808F401E081
:103DB400E12FE03041F4013029F43093390C309391
:103DC400380C11E00FC0E13031F4003019F43093B5
:103DD400380C12E007C0E23029F4013019F43093B2
:103DE400390C13E03F5FD9CF0E94657D2496089576
:103DF4001A930A93A0911908A43009F43FC01091B2
:103E04002F080091510CE0913108E03059F0E09313
:103E14002F08689424F80E94C670E0E0E09330080C
:103E2400E0E520C0E0913008E03021F0E0932F0875
:103E3400E2E518C0E0E0E0932F08E093510CE09134
:103E4400C40BE03031F0E091C40BE150EA930E94DE
:103E54003219A091340CA17039F0E091C40BE093B5
:103E64002F08E4E4E093510CA0912F081A1721F4D1
:103E7400A091510C0A1711F0689423F80991199133
:103E840008950E94CC70EBE0EC93EC81D801169677
:103E9400EC93EB81D8011796EC93D8011896E0E0E7
:103EA400F0E0ED93FC93D80112960E94D970D801EA
:103EB40014960E94D9700E94DE70F2C00E94CC70E9
:103EC400ECE0EC930E94DE7021C21A9318E01131E9
:103ED40008F5E0911408F0911508A981BA81EA2740
:103EE400FB27BF010E94EA70E623F723309781F095
:103EF4000E94EA70A981BA81EA23FB23309731F04A
:103F04001A93E0E0EA931A93BCDF02C01A93D6DF57
:103F14001F5FDDCFFAC1A0911A0CA93030F0E091F7
:103F2400590CA091580CEA1709F414C0E091590CEB
:103F3400E03021F4E3E6EA93C1DF08C0E0911A0C13
:103F4400EA93E0E0EA93E3E6EA939BDFE091590C1D
:103F5400E093580C0895A0919A0BECE1EA2308959C
:103F6400A0919A0BA07411F0E2E00895A0919A0B2D
:103F7400A07809F0E2C10DC0A091890BAF3F09F40C
:103F8400DCC1E9DFE43009F4D8C1E5DFE03109F44C
:103F9400D4C1E1E008950895A881AF3F11F4E0E0B1
:103FA4006EC1D9DFE43011F4E1E069C1E0E067C13A
:103FB400A881A23019F4CFDFE83011F0E1E05FC14D
:103FC400E0E05DC1E881A3E2EA9FF001ED55F94F1D
:103FD400E081E13010F0E43108F002C0E1E04FC1CB
:103FE400E0E04DC1A881A13118F0E881E051E883F7
:103FF400E8810E94F5700E94FF70A091D00BA1305F
:1040040018F0A881A43009F006C0E6E9F0E00E94A7
:10401400897B0E94FF7033C1A881A13010F0A630C3
:1040240008F006C0E8810E940A71E15CF94F26C1DC
:10403400E0E025C1A881A13010F0A63008F006C048
:10404400E8810E940A71EC5BF94F18C1E0E017C1E6
:104054000E945E7DEC81EA93EDDFEF731E2F10303A
:10406400E1F0EC81EA93E6DFE0743E2FE12FE150CA
:10407400A1E00E94817AA0912306EA230E2F30301A
:1040840011F4003009F002C0E1E008C0303011F052
:10409400003009F402C0E1E001C0E0E00E94657D67
:1040A400259608950E945C7D00E00530A0F50A93F2
:1040B4000E9474190E940F71A7E10A9FF001EE5C3F
:1040C400F94F0E943970E4E1F0E00E94EB6FE09157
:1040D400300CDA015096EC93A0912F0CEFE3EA2315
:1040E400AE2FE091320CE295E07FEE0FEE0FEA0F77
:1040F400DA015596EC93E091300CE1503E2F3F3FAE
:1041040041F0E091310C0E94CE6FDA015196ED93AB
:10411400FC930F5FCACF10E01034C0F51A930E94CD
:10412400DD181A9339DFE13079F5E0919D0BEA93BC
:1041340073DFE1500E2F0F3F39F10E940F71E12F11
:10414400DA011396EC93E0919D0BDA011496EC934B
:10415400E091A30BF091A40BDA011696ED93FC9376
:104164000E94C76FA4E6B0E080E090E00E94DB7A92
:10417400DF01CB01E091A30BF091A40B0E942B6E05
:10418400DA011A96ED93FC931F5FC6CF0E94637DFC
:1041940026960895A0911908A23031F0A83021F094
:1041A400A73011F0A53009F40AC00E94E46FEFEFC4
:1041B400F0E00E94EB6F76DFE0E0E093A206089562
:1041C4001A93E981E058E98310E01530C0F4A3E2C2
:1041D4001A9FF001EB55F94FE081AE2FE981EA1700
:1041E40049F4F001EC55F94FE081AE2FE0912F082E
:1041F400EA1709F002C0E12F03C01F5FE6CFEFEF1B
:104204001881229608950E945E7DED81EA93D8DF9D
:104214001E2F1F3FC1F00E9416719F01D9011296F3
:10422400EC91EF77EC93EC81D9010E941C71EF5E65
:10423400FC4FBF01E081EF77DB010E941C71E15F5D
:10424400FC4FA1E0A083E12F0E94657DE2C40E949F
:10425400B96DED55F94FE081E03061F4E0914B0C1C
:10426400EF5FE0934B0C0E94B96DED55F94FA091AF
:104274004B0CA0830E94B96DED55F94FE081219656
:1042840008951A931FEFE091D40BF091D50BA981F7
:10429400BA81AE17BF073CF0E091D60BF091D70B73
:1042A400EA17FB070CF412C00E9423710E941E1827
:1042B4001E2F103031F01F3F21F0E0912F08E1173D
:1042C40029F4E1E0E093590CE0E01FC0E0E0E09362
:1042D400590C1AC01A930E942371D3DF1E2F103079
:1042E40099F01F3F39F4E8EEF6E1FA93EA93EB8193
:1042F400FC8106C0E8EFF6E1FA93EA930E94287184
:10430400FA93EA930E946D11E12F18812396089580
:10431400E0916505E03009F00895E0912C06E03065
:1043240009F008950AC0E0916605E03009F00895A7
:10433400E0912D06E03009F00895E0E008950E9430
:104344005E7DE0912606F0912706AC81BD81EA27C7
:10435400FB279F0110E0153090F4F901E17049F05A
:10436400A7E11A9FF001EF5CF94FDF01EC91EF5FD9
:10437400EC93D9010E942B719F011F5FECCFEC815C
:10438400FD81E0932606F09327060E94657D41C4D3
:1043940028970E945C7D3091260610E01530B8F510
:1043A400A7E11A9FF001EB5BF94F0081E12FA1E037
:1043B4000E94817A2E2FE22FE32391F0003810F02F
:1043C400003C08F001C00F5F003C31F4E22FA091E3
:1043D4002306EA2BE0932306003808F400E80FC014
:1043E400003408F40F5F003439F4EFEFE227A091B2
:1043F4002306EA23E0932306003808F000E0A7E14F
:104404001A9FF001EB5BF94F00831F5FC7CFE0E019
:10441400E0932C06E0E0F0E0E0931608F093170830
:10442400E091590CE03021F0E0911A0CEA93DADDC6
:10443400E0911D08EF5FE0931D08E091E30BA0916C
:104444001D08EA1751F4E091E30BF0E0A0E0B1E0BD
:104454000E949D7BEA1BE0931D08A0911908A130DE
:1044640019F0A93009F096C0A091620BB091630BCA
:10447400E4E1F0E00E94337B309719F4E1E0E0934B
:104484001F0846DFE03019F04EDFE07809F462C01F
:104494004ADFEF775E2F5A930E94DD180E940D6D5C
:1044A400ED55F94F5081503011F40C94AC2264DD79
:1044B400E13031F4E0911A08EA937ADDE03009F44E
:1044C40049C00E9430710E94B06FEC91EC71EC30E5
:1044D40021F4E0911D08E07851F40E943571EC91CB
:1044E400EA9380DD0E943A71EC91EA937BDD0E94AD
:1044F4003571AC91A63070F5A3EEB6E00E940D6D57
:104504000E94BC6D0E94636E0E943571EC91EA9327
:1045140083DD1E2F1130F0F00E943F710E94427122
:10452400CF010E943F710E94BC6D6D917C91E12F7F
:104534000E940A71EF5CF94F0E944771E60FF71F62
:10454400DC01ED93FC93E12F0E940A71EF5CF94FBB
:10455400A0E0A08310E01530E8F40E944A7113969D
:104564005C915F3FA9F05A9372DE5E2F0E945471F2
:104574000E943F710E944271BF010E943F710E94DC
:10458400BC6D0E945A71AE81BF811296E0E0EC933B
:104594001F5FE1CFA0911908A23039F0A83029F0AB
:1045A400A53019F0A73009F0E4C1E0E0E093200859
:1045B40000E0053010F00C94BB24A3E20A9FF00144
:1045C400ED55F94FEA87FB87AA85BB85AC91A030EE
:1045D40019F0A281A07809F0CAC1E0912008EF5F28
:1045E400E0932008AA85BB8513960E947A7B3097B6
:1045F40071F0AA85BB8513960E9467710E946D7144
:1046040029F4AA85BB8513960E94D970B0C180DEB7
:10461400E03021F00E946D7109F4A9C120E030E07E
:10462400333010F00C9468240E947571DF010E94ED
:104634009C6C0E94906DE887F987A181A27021F497
:10464400A481B581109709F40CC1E885F985A1818D
:10465400A47011F40C948E23A181A87021F40E94FB
:104664009D33E03009F457C00E947B71EBE0EC937A
:10467400A885B9850E948871A885B9851396EC919F
:10468400AC85BD851796EC93EC85FD8538960F01B6
:10469400E885F985A181E1E0EA230E948F71ED9319
:1046A400FC93A885B98514960E947A7BAC85BD8558
:1046B4001296ED93FC930E949271AC85BD8514967D
:1046C400ED93FC93A02FEAE0EA9FF001E30FEF5F84
:1046D4000E949871E885F985A085B185E2E0F0E053
:1046E4000E94D67AA885B9851896ED93FC930E940A
:1046F4009271309739F4A885B9851896E8EEF3E0FD
:10470400ED93FC93E885F985A181E8E0EA2BA8857F
:10471400B9851196EC936CC0E885F985A181A170E7
:1047240031F4A885B98514960E94677141C00E942E
:10473400A17172DCE1501E2F0E944A711296EC9115
:10474400E030F1F4AE81BF8153960E94636EEE8136
:10475400FF81A189B289109751F003881488AE8132
:10476400BF8151960E947A7BE015F1050CF007C0D9
:104774000E94A67111F00E94AB710E94B3710EC029
:10478400E885F98534960E94BB710E948F710E945E
:1047940074700E94C37153960E94D970E885F9859C
:1047A400A581AA232AF4A885B98514960E94D970F4
:1047B400A885B985EC91EC71EC3021F4E0911D08E9
:1047C400E078B1F4E885F985A481B5815E971CF49D
:1047D400A181A07209F404C0E885F985A28106C00C
:1047E4000E94A171FFDBE885F985A381AA93FADB16
:1047F4000E949271309781F0A885B98518960E941D
:1048040067710E949271309739F40E94A67111F079
:104814000E94AB710E94B3710E94A17119DCE03057
:1048240001F10E94A67159F00E94AB71AA85BB8563
:10483400EC91E150ADE0EA9FF0010E94156DAA856C
:10484400BB851296EC91E058AA85BB851296EC9331
:10485400E3E0E09324060E94A171ECDBEF73E093A4
:104864002506A885B98514960E947A7B309761F550
:104874002F5F323048F5A885B98516960E947A7B59
:10488400309789F0E885F985A681B7810E94CA71BD
:10489400AA85BB851396ED93FC93A885B9851696D6
:1048A4000E94D97011C00E947571DF01E32FEF5F80
:1048B400F0E00E94906DE887F987A181EDEFEA238B
:1048C400A885B9851196EC933F5FAACE233011F0E9
:1048D4000C94B9240E94A67111F00E94AB710E943D
:1048E4009D33E03069F00E947B71E8E0EC93AA8587
:1048F400BB850E948871AA85BB85EC910E94987142
:10490400AA85BB85E0E0EC93EA85FB85A581ECE113
:10491400EA23E83061F50E94CE6DAE2FEA85FB856F
:10492400E38DEA1741F4EA85FB85E48DE150EA93CF
:104934000E94DE171CC00E949D33E030C1F00E942B
:104944007B71E3E0EC93AC85BD85EFEFEC931896B7
:10495400EA85FB85E38D0E94CF71AC85BD851296F7
:10496400EA85FB85E48D0E94CF710E94D3710F5FAD
:1049740020CE0E94D97149F4A0911908A23021F0E7
:10498400A83011F0A53009F401C050C010E0153072
:1049940010F00C9418250E944A7113965C915F3FA5
:1049A40011F40C9416250E945471AE81BF81BD018F
:1049B4000E945A71EE81FF8138960E94BB710E9459
:1049C400DF710E94C3710E947A7BDF010E94527DD5
:1049D400B4F4EE81FF81A681B7810E94527D7CF4FC
:1049E400AE81BF810D901C90AE81BF8116960E944E
:1049F4007A7BD001AE1BBF0B0E94527D0CF014C019
:104A0400AE81BF81BD010D901C90EE81FF81A68116
:104A1400B781F001EA1BFB0BDB01ED93FC935A9386
:104A2400E5E0EA930E94E8421F5FB1CFE0911C08E1
:104A3400E03041F4E0911608F0911708E09314086F
:104A4400F09315080E94637D2E9608950E945E7D62
:104A5400A091C10BE091C20BE150EA9FF001EF5F1E
:104A64001E2F2FE330E000911E08A091180CA130F6
:104A740080F0E091180CE150A0911E08AE1728F0C8
:104A8400E091180CE1503E2F04C0E091180CE25064
:104A94002E2FEC81E03049F1EF3F51F4A0911E0834
:104AA400A11BA31720F0E0911E08E11B0E2F1DC0CF
:104AB400EE3F59F4E12FA0911E08AE0FA21720F487
:104AC400A0911E08EA0F0E2F10C0EC3F49F4A091EC
:104AD400180CA13020F0E091180CE1500E2F05C005
:104AE400AC81A1501A9FF0010E2FE0911E08E0172F
:104AF40051F00A930E94DD18A0918A0BAD3209F49B
:104B0400032F00931E080E94BD46A0911908A830E7
:104B140019F40E94850F02C00E94000F0E94657D57
:104B2400259608950E945C7D16DAE03111F40C9408
:104B3400082620E030E040E050E010E0133060F55B
:104B44000E94E3710E94BC6D0E947A7B309711F140
:104B54000E94E6710E94F5702E2B3F2B0E94E67195
:104B6400EA9376DAE03029F0E3E0E0932406E0E02B
:104B74004EC00E94ED710E94F5702E2B3F2B0E94B7
:104B8400ED71EA9365DAE03029F0E3E0E09324067E
:104B9400E0E03DC01F5FD2CF00E0053068F5A3E23E
:104BA4000A9FF001ED55F94FE081E03019F110E072
:104BB400133000F50E947571DF010E9428710E9474
:104BC400F471AE0FBF1F1296EC910E94F5704E2B3C
:104BD4005F2B0E947571DF010E9428710E94F4719D
:104BE400AE0FBF1F1396EC910E94F5704E2B5F2BF6
:104BF4001F5FDECF0F5FD1CFF901E423F523309798
:104C040029F0E1E0E0932406E0E001C0E1E00E9445
:104C1400637D269608951A93E0914F0CE03011F4C9
:104C24000C945426E091E40BE13059F4A0914F0C1C
:104C3400A13311F4EFE001C0E0E0EA930E94425E88
:104C440031C0E23059F4A0914F0CA13311F4E6E0E5
:104C540001C0E5E1EA930E94425E24C0E330B1F46E
:104C640010E0173040F40E942871E05CF64F0E9477
:104C7400FB711F5FF6CFA0914F0CA13311F4E1E358
:104C840001C0E0E3EA930E94425E0CC00E94FF71FF
:104C9400E9E4EA930E949762E0914F0C0E94067245
:104CA4000E940B7285C422970E945C7D30E0A09123
:104CB4001908A23029F0A83019F0A53009F014C160
:104CC400A985A03410F00C947527E0912F08E030EA
:104CD40009F40AC1E9850E94B46FE03131F4E1E3DB
:104CE400E0934F0C98DFE1E0FFC046D9E03009F4CF
:104CF400FBC010E0153058F40E941671E081AE2F0D
:104D0400E885EA1711F4E0E0EFC01F5FF3CF0ADF94
:104D1400E03011F40C94752710E00E941671EE83B4
:104D2400FF83AE81BF81EC91E03011F00C946E27CB
:104D340013960E94D97000E0033010F00C943E27C3
:104D4400A3E21A9FF001E855F94FDF010E94846C39
:104D54000E94906DAF01DA0116960E94D9700E94EC
:104D64001072DA011296EC930E941772DA0113960C
:104D7400EC93A0919A0BEEEFEA23DA01EC930E94F4
:104D84001E72DA011196EC93E6D8E43139F0FA0197
:104D9400A181E2E0EA2BDA011196EC930A9308D997
:104DA400E03011F40C942027FA01A281AA9334D99B
:104DB400E1502E2F2F3F81F0A7E12A9FF001EF5CF5
:104DC400F94FA0E0A083A7E12A9FF001EE5BF94F21
:104DD400A0E0B0E0A083B1830E9426720E94BC6D63
:104DE4000E947A7BDA011496ED93FC93013040F033
:104DF4000E9426720E94BC6D0E947A7B309709F053
:104E04000EC0AE81BF811596E02F0E94616F0E9493
:104E1400F471AE0FBF1F1196EC91E062EC93AE817A
:104E2400BF815A96EC91E062EC93023030F40E9418
:104E34002972DA0116960E94CF7104C0DA01149621
:104E44000E94D97088D8EC3019F4E0E0E0931D0892
:104E54000E9430720E94CE6FDA011896ED93FC9393
:104E6400FA01A281A63030F0A181E4E0EA2BDA0154
:104E74001196EC930F5F60CFA0911908A23011F046
:104E8400A53019F4A885AF3F08F007C0E0912F08BA
:104E9400EA93EA85EA930E94121AE885AE81BF81FB
:104EA400EC93E0912F08AE81BF811196EC93E985D4
:104EB400AE81BF811296EC93A885A43130F4E885C5
:104EC400E1500E943772A1E0A083AE81BF811696A3
:104ED400EC91ED7FEC9331E01F5F303011F415302D
:104EE40008F001C01ACFE32F0E94637D2A9608952B
:104EF4001A930A93A0911908A23011F0A53049F42D
:104F0400EA810E943772A0E0A083EA81EA930E94BA
:104F14007E6EA0911908A830F1F4EA810E943772DC
:104F2400A0E0A083EA81EA93E1E0EA930E941F47AC
:104F3400E091E20BE03069F4EA810E943D72E08185
:104F4400EF771E2FABE01A9FF001EA51FA4FA0E071
:104F5400A083689420F819810881239608956497A2
:104F64000E94B86CA23039F4E0912F08EA93EB8DDB
:104F7400EA930E94121AA0911908A83011F00C9417
:104F840027280FEF20E0253050F4A7E12A9FF001F5
:104F9400EE5CF94FE081AE2FEA8DEA1709F402C006
:104FA4002F5FF1CFA7E12A9FF001E15DF94FAF0137
:104FB400DA0115960C910F3F11F40C9427280E94E6
:104FC400437210810E94AD700E94527DECF4ACE2F9
:104FD400BCE00E9467710E9449720E948470A083A1
:104FE400B1831A930E94C21EABE00A9FF001E25201
:104FF400FA4F30810A93FE0137960E944F723A931A
:10500400FE0137960E9453720E945972F1F40E9475
:105014004372AFEFA083DA011396EFEFEC93DA015A
:105024001596EC930E9449720E945F72E0E0F0E0F2
:105034000E949270E0E0E093290C1A930E94C21E31
:105044000A930E94E910689420F80E94637D6B968D
:1050540008951A9310E01031B0F4A7E11A9FF001FB
:10506400EC5BF94FE081EF73AE2FE981EA1729F485
:105074001A930E942A20E03009F403C0E1E0188169
:10508400E0C01F5FE8CFE0E01881DBC01A93E09135
:10509400520CF091530CFA93EA93E4EFF1E00E947E
:1050A400A170F9F00E94647210E01530D0F4A09160
:1050B400560CAF5FE5E00E94307BE093560CEF5F47
:1050C400EA93C7DFE03059F0E3E0E0932406E0918F
:1050D400560CF0E0EF5FFF4EE093250669C21F5FB8
:1050E400E4CF66C21A93E0912306E0934E0CE8E7FE
:1050F400F0E0FA93EA93ECEDF0E0FA93EA930E947D
:10510400EE4610E01530D8F4E12FEF5FEA93A1DF0B
:10511400E03099F00E94016CE12FEA5FF0E00E9418
:10512400CA6DE5E0F7E10E94686DA6EEBBE00E945F
:1051340028710E94906D0E94986D1F5FE3CF38C262
:10514400A5DFE0912406E13029F4EDE0F7E10E94C7
:105154006B723CC0E23029F4EAE1F7E10E946B7221
:1051640035C0E33051F4E5E0F7E1FA93EA93E091D6
:105174002506F0E0E050F04F29C0E43019F4E2E2F3
:10518400F7E11FC0E53031F4E0912506EA930E946F
:10519400501120C0E63019F4EAE2F7E112C0E7301A
:1051A40029F4E0E3F7E10E946B7210C0E83029F4BF
:1051B400ECE3F7E10E946B7209C0E93059F4EBE4C7
:1051C400F7E1FA93EA93E0912506F0E0FA93EA9383
:1051D4000E946D11E0E0E09324060895A881B9814E
:1051E4001196E1E0EC930E94B170A881B981129606
:1051F400ED93FC930E94B21FA881B9811796EC939A
:105204000E94CE6DA881B98118960E94CF71E09159
:10521400C605A881B981EC93E091290CA881B981D4
:105224001696EC93E091890BA881B9811A96EC93B8
:10523400E091AC0BF091AD0BA881B9811496ED937C
:10524400FC932296089564970E945E7DA091E20BE0
:10525400A230E1F4EB8DEA930E94DD180E94B21FA4
:10526400ACE2BCE00E94CF71AAE2BCE0EB8D0E94EC
:10527400CF71E0912F08E093290C0E94B96F309709
:1052840021F00E94B96F0E949C7014C0AA8DAF3F98
:1052940009F4CAC0EA8DEA930E94BB1EAB8DAF3FEE
:1052A40029F40E94B1700E94BE6FEB8FEB8DEA93DC
:1052B4000E94DD180E94B21F0E2FA98DAF3F21F06E
:1052C4000E94BE1FE03009F001C0AEC00E9484708D
:1052D4000E94846CAE17BF071CF024DCE13009F097
:1052E400A3C0A091D10BA03021F4A091E20BA23075
:1052F40011F50E94CE6DE13041F00E949D33E03003
:1053040021F00E94B333E03009F002C00E947072B1
:105314000E94CE6DE13021F40E94A333E03009F401
:1053240009C00E947C72EE55F84FFA93EA9356DF57
:105334000E94827277C0EB8DEA93EA8DEA93B3DC24
:105344001E2F113011F00C94142AA091D30BA1300C
:1053540059F4E0912F08EA930E94B170FA93EA930A
:10536400EFEFFFEF0E9488720E9484700E94846CA9
:105374000E9474700E949270689420F8A091E20BCD
:10538400A03019F4A88DAF3F09F437C00E948C7285
:10539400EE51FA4F0E948470A083B183E88D0E947D
:1053A400716D3081E88DEA93FE0135960E944F724B
:1053B400E88D0E94716DE081EA93FE0135960E94AA
:1053C40053720E94AD1FE03131F00E948C72EA5199
:1053D400FA4FA1E005C00E948C72EA51FA4FA2E094
:1053E400A0830E948C72EC51FA4FFF93EF930E94BA
:1053F4000968AF91BF91ED93FC930E94597219F41F
:10540400E0E0E093290CEA8DEA930E94C21EE09149
:105414002F08EA930E94B96F0E949172FA93EA935B
:105424000E94B01CE1E001C0E0E00E94657D6C9642
:10543400089578DBE13041F40E949D33E03021F09F
:105444000E94B333E03009F007C00E94B96F0E9494
:105454009C700E94707226C32EC30E945E7D0E94BF
:1054640094721F3F11F40C94862AE0914F0CE030A3
:1054740011F00C94852A1A930E94DD18E5E0E0935C
:10548400240610932506A0911908A23031F40E9435
:105494009D720E946C21E03009F010C0A091500C64
:1054A400A13331F4E0912F08EA931A930E94121A5F
:1054B400E1E3E0934F0C0E94657DE2C2A0911908DC
:1054C400A830A1F40E94B96F0E94A1720E2F0A9312
:1054D4000E9413343E2F1A930A93EFEFEA933A9300
:1054E400B2DEE03019F00E94657DCAC2A0911908AD
:1054F400A53031F49EDFE03019F00E94657DC0C212
:10550400E0E3E0934F0C06C0E0E3E0934F0CE4E0EB
:10551400E09324060E94657DB3C2E09140090E9495
:10552400A57208951A93E6E0EA930E94425E0E94EF
:10553400FF71A0914009A83539F4E7E5F7E10E942D
:10554400B172E0E00E940B72A0914009A33509F505
:1055540010E0A0911908A83021F0A23011F0A53074
:1055640009F411E3E3E5EA930E9497621A930E9417
:105574009762E0E8EA930E949762E0E8EA930E9467
:105584009762E0E80E940672E0934F0CE0E00E940C
:105594000B72A0914009A93459F40E94B572E093AA
:1055A40025060E94BF72EC91E093500C56DF33DB6A
:1055B400199108950E945E7DA0913F09A53411F0D0
:1055C4000C94232B0E94C472E2E3F0E0E093490CB4
:1055D400F0934A0CA0914009A73741F4E4E4F9E0C0
:1055E4000E94CB720E94D0720E94A572A0914009C1
:1055F400A03310F0AA3308F023C02091270830917B
:105604002808E0E4F9E00E94CB72E2E0EA930E9409
:105614003D620E2F0E94D072E09325060E94D07244
:105624000E94D4720E9494720A931A930E94121ACE
:105634002093270830932808E2E5EA930E94425E0B
:105644001CC0E091470CF091480CFA93EA93E09166
:10565400490CF0914A0C0E94A17079F0E0E0E093CB
:105664003A09E5E4EA930E94425E0E94C472E8ECBF
:10567400F0E0E093490CF0934A0C0E94657D00C26F
:105684000E94D9720E94DF720E94016C0E94016C18
:105694000E949646A0911B08A23021F4EFE5F7E1A1
:1056A4000E94686DA0911B08A13021F4E6E6F7E1A1
:1056B4000E94686DE0911B08E03021F4EDE6F7E10B
:1056C4000E94686D0E94E9720E94426C0E94964694
:1056D4000E94EC720E94F172FA93EA93E0915F05E2
:1056E400F09160050E94F7720895E1E003C0E0E0E4
:1056F40001C0E2E0E0931B08C3DF08950E94AD1FE0
:10570400EC3109F0D8C1E091990BE33631F4A09162
:105714001908A23009F4EBDF17C0E23631F4A09186
:105724001908A23009F4E5DF0FC0A091C505A23025
:1057340011F0A63021F4E091990BEA9387D9A09156
:10574400C505A43009F4D1DFADC10E949E6D0E944D
:10575400016C0E94A26D0E94016C0E94016C0E9467
:105764009646E8E7F5E00E94686DE0911A080E9409
:10577400FB72E6E8F5E00E94686DE2E0E0930E0457
:1057840008950E94E46FE0ECF0E00E94EB6FE88182
:10579400E03009F406C0A0911A08AF5FE3E00E946C
:1057A400307BE0931A08E1E0E0934B0C0E94542014
:1057B40072C20E945E7D10E0103410F00C94282C0C
:1057C4000E942871ED55F94F30813F3FE9F11A935A
:1057D4000E94DD1800E00E94FF720E94BC6D0E94CE
:1057E4007A7B3B9794F00E9402730F010E94FF7230
:1057F4000E94BC6D0E9408730E940E730E94B06FD9
:10580400EC91EE7FD001EC9301E00E9413730E94AF
:10581400BC6D0E947A7B759794F00E9402730F010D
:105824000E9413730E94BC6D0E9408730E940E7341
:105834000E94B06FEC91E160D001EC9301E0013083
:1058440019F41A930E94FD181F5FB6CF0E94657D5C
:1058540017C11A930A9323FE03C00E9416733FD7FD
:105864000E94F842E030C1F1E0E00E941D7310385C
:1058740020F5113219F40E94167331D71D3439F40E
:105884000E9424730E94AD63E3E0E09318081B3286
:1058940071F40E942973EAE2EA93E8E7F7E1FA93E4
:1058A400EA93E0911A08E05DEA930E94AD631F3227
:1058B40019F4E1E0EA93CAD848DF103868F00E948E
:1058C4002F731A930E94292119DFE03011F410324A
:1058D40008F002C0E5E5F6E20E9495210E2F00389B
:1058E400C8F10F770034A8F5E0911F08E03031F0DB
:1058F4000A930E94BE11E0E0E0931F08E091570C68
:10590400E01739F10A930E94DD180E943571AC91B9
:10591400A83028F40E943A71AC91A830A8F0E02F86
:10592400EF5FE093A2060A930E9429210E94357139
:10593400EC91EA930E943A71EC91EA93E091A20609
:10594400EA930E94431F03C0E0E0E093A2060093A1
:10595400570C0EC0A091570CAF3F51F0E091A20636
:10596400E03019F0EA930E94601FEFEFE093570CC8
:10597400099119910895A881A03310F0AA3308F071
:105984001DC00E9433730E943873AAE0B0E00E94E5
:10599400D67ADF01E8810E943D73EA0FFB1FE09392
:1059A4002508F0932608E2E0E0930E040E94E972D1
:1059B4000E94426C0E94A26D0E94EC72A881A334E2
:1059C40051F40E94DF720E94E9720E94426C0E94AC
:1059D400A26D0E94EC725FC11A930A93A0E023FCAB
:1059E400A1E0A03019F0AA81A03009F016C0E89413
:1059F40023F8E7E0E09318080E94DD45A091310800
:105A0400A03019F40E94407309F407C0E7E0EA9358
:105A14000E94457364D6E89424F824FE24C00E94AE
:105A24004873EAE5F0E00E944F7319F0AA81A130AF
:105A3400C9F481D6E030B1F00E9455730FEF1FEF27
:105A44000E949D720E944321E03021F400912708B6
:105A540010912808EB81EA93E0912F08EA931A93B6
:105A64000A933DD60BC00E944873ECE2F1E00E9419
:105A74004F7321F40E945C73E0933008198108810C
:105A840024960895E091C70BF091C80B0E946073AF
:105A940011F4E2E00895E091C50BF091C60B0E9469
:105AA400607311F4E1E00895E091CB0BF091CC0B1D
:105AB4000E94607311F4E0E00895EFEF0895A0915F
:105AC4001908A23021F40E94BD460E94000FA09143
:105AD4001908A83009F462D6A0911908A53009F470
:105AE40049D1D9C0E2E0EA930E94C440E2E0E093E5
:105AF4000E04E881EA933FDFA881AF3721F4E091F7
:105B04002B06E37009F403C0E2E0E0931808A881CF
:105B1400A13239F0A33421F40E943373109709F0B1
:105B240004C0A0911908A23009F011C0A0911B086B
:105B3400A33009F4DEDDA0911B08A23019F4E1E0E2
:105B4400EA93BDDFE0911B08E03009F4D0DDA881C1
:105B5400AD3311F00C94092E0E94DD45E0911B0831
:105B6400E030B1F4E0912508F0912608FA93EA9325
:105B74000E946C21E03051F4E0912508F091260850
:105B84000E94D472E0E0EA939ADF01C0B0DD3FC026
:105B9400E13079F477DFEF3F41F0E3E00E94647392
:105BA4000E9424730E946A7303C0E1E0EA9387DFD2
:105BB4002EC0E230F1F40E943373A034E0E0BE075B
:105BC400B4F4E0912508EA930E947173E2E0E09353
:105BD4000E040E94016C0E94016C0E9496460E9471
:105BE4005B6D0E945110E3E0E0931B0801C081DD6E
:105BF4000EC0E33061F4E0912508EA930E94DD18B9
:105C0400E0912508EA93EEEFEA934DD872DDA8817E
:105C1400AD3409F46ADDA881A43521F4A0911908F2
:105C2400A23009F001C063DDA881AB3221F4EEEFAC
:105C3400EA930E942825A881AD3221F4EFEFEA937C
:105C44000E942825A881A73421F4E1E0EA930E9468
:105C54002825A881AB3421F4ECEFEA930E9428258F
:105C64001AC00E94CC200E94BD46E0E0E0931B08CD
:105C7400A881A13039F40E94407321F0A091CA0B8D
:105C8400A03009F402C033DD06C00E94000F0E9458
:105C94009D720E944321219608951A930A930E94AB
:105CA40075730E948D1F0E94F842E03091F10E94AA
:105CB4007E7378F10E942F7321DDE03051F50E944C
:105CC40086730E940521EF3F09F006C50E949D726C
:105CD4000E946C21E03021F40E94BE1FE13009F0E3
:105CE40018C00E94AD1FE83119F40E948B7309F0AB
:105CF40001C0F2C40E9486730E9455260E2F013003
:105D040021F4A091990BA03009F403C01A930E94C6
:105D14005011A0912E06AF3F61F110912E06EFEFC6
:105D2400E0932E061A930E94DD180E949D720E9431
:105D34006C21E03021F40E94BE1FE13009F019C04B
:105D44000E94AD1FE83119F40E948B7309F001C061
:105D5400C3C41A93EEEFEA930E9455260E2F013026
:105D640021F4A091990BA03009F403C01A930E9466
:105D74005011B2C40E94CC200E945420E89421F80F
:105D8400E0E0E0931E080E9492730E94BD460E94C8
:105D9400016C0E94016C0E949646E09132060E94BA
:105DA400DF6DE09133060E94DF6D0E94016C0E945A
:105DB400636D0E949646E0913F060E94DF6DE0917C
:105DC4003906F0913A060E94B56D08950E945E7DF1
:105DD4000E9475730E94F842E03049F00E947E737D
:105DE40030F00E942F738ADCE03009F422DBE0916A
:105DF400540CF091550C0E94826E11F40C94622F95
:105E04000E9492730E94016C0E94566D0E94A26DC2
:105E1400E0913706F09138060E94B56DE0913B069B
:105E2400F0913C060E94B56D00E0053010F00C9432
:105E3400622FA7E10A9FF001E15DF94F9F01F9018B
:105E4400A381AF3FD9F1D9011A960E94C16D7F9306
:105E54006F93FF93EF930E949973AF91BF918F91CA
:105E64009F910E94987A0E94DB7ADF01CB010E9405
:105E74009E73D9011C96ED93FC93F9010484158457
:105E8400D9011E960E947A7BE015F105B9F0F9015B
:105E940004841584A685B785F001EA1BFB0BE09307
:105EA400AC0BF093AD0BC5DAE13041F4D9011C968B
:105EB4000E947A7BD9011E96ED93FC930F5FB5CFB8
:105EC4000E94657D2AC40E945E7D0E9475730E94B3
:105ED4008D1F0E94F842E03011F40C94FB2F0E94B5
:105EE400FB420E2F0A93FEDD003820F0A091C60578
:105EF400A03808F429C00F770A930E94A5730E9462
:105F0400A1721E2FA091E20BA03011F41F3F09F4DF
:105F140016C030E0353098F4ABE03A9FF001E4521B
:105F2400FA4FE081E11749F43A9FF001E252FA4F47
:105F3400E081EF5FE093C605232F3F5FEBCF0A9329
:105F44000E9486732A9354C0A091E20BA03021F4DE
:105F5400003810F0053808F00AC00F770E94437229
:105F64001081EFEFEA930E9486730A936CD9A09193
:105F7400E20BA03011F0003808F43BC00F770A930D
:105F84000E94DD18BBDBE030A1F50E94A8730E94DB
:105F94000521EF3F19F00E94657DBFC30E94BE1F1B
:105FA400E13039F50E94B21FE03049F40E94A87331
:105FB4000E945526E03011F00E94AD731AC00E9471
:105FC400AD1FE83141F40E948B7321F00E94A87345
:105FD4000E9455260EC0A0911E08E02F0E94356D28
:105FE400AE0FBF1F1C910A930E948673EFEFEA93D2
:105FF4002AD9A0912E06AF3FF9F000912E06EFEFBB
:10600400E0932E060A930E94A5730E94A1721E2F8C
:106014000A931A93EEEFEA93EFEFEA9314D91F3F32
:1060240041F4A0919D0BA03021F4A091A00BA030CD
:1060340009F002C00E94AD7320FE0AC0E89420F863
:10604400E091E20BE03019F4FFD350D501C0AFD595
:1060540030E0353080F5ABE03A9FF001DF01EA51E2
:10606400FA4FE081E03049F0AC51BA4F0E94B3736B
:10607400E8EEF3E00E94A17099F4ABE03A9FF001DE
:10608400EA51FA4FE081E23051F43A9FF001EC51C9
:10609400FA4FDF010E947A7B0E94826E09F409C0E4
:1060A400ABE03A9FF001EA51FA4FA0E0A083689474
:1060B40020F83F5FCECF0E94657D2FC30E94B86C4D
:1060C400A33011F40C941932E0913A08ED3411F034
:1060D4000C944231E0913B08EA3511F00C94F7300E
:1060E40024FC83C0E0913C08E0532E2FE0913D084E
:1060F400E0533E2FEEE3F8E00E94CB720E94BF72A1
:10610400AC91AB3429F40E94B8730E94C9610E2F7C
:106114000E94BF72AC91A43529F40E94B8730E9406
:10612400C961AF01E091CD0BE31731F5E0E0E093F5
:106134004D0C0E9455734093270850932808A09152
:1061440030080A1759F0E7E0E09318080093300884
:1061540020934C0CE0E0E0932F080DC0A0914C0C70
:106164002A1721F0A0912E08A03009F004C0209332
:10617400180820934C0C35C0A0913008A03049F485
:10618400A091CE0B0E949C6CE255FF4FE491EA2350
:1061940009F40CC0E7E0E093180820934C0CE0E00D
:1061A400E0932F08E0913908E0934D0CE091390811
:1061B400A0914D0CEA17A9F440932708509328089E
:1061C400009330080E945573A0914C0C2A1721F0BB
:1061D400A0912E08A03009F004C020931808209341
:1061E4004C0C273011F40E94C670E0913B08E9344E
:1061F40039F4E7E00E9464730E945C73E0932F0813
:10620400E0913B08E23439F4E4E00E9464730E94B4
:106214005C73E0932F08E0913B08E03519F4E1E06A
:10622400E0931808E0913B08EC3449F4E4E0E0938F
:106234001808E0913C08E053EA930E941616E09196
:106244003B08E334E9F4A0913C08A13320F0A09189
:106254003C08A93308F014C00E94BB73E0912208E3
:10626400EA930E942D1BE0913908EA93E4E8F7E1F0
:10627400FA93EA930E94EF6F0E948D7B0E94A063C1
:10628400E0913A08E03521F4A0911908A13009F011
:1062940003C00E94297359DAE0913A08EF3459F4A3
:1062A400E0913B08EE3439F4E0913908EA93E7E8E9
:1062B400F7E10E94C173E0913A08E33569F5E09192
:1062C4003B08EF3349F5A0913C08A03320F0A0919E
:1062D4003D08A03308F420C00E94BB73E0913D0840
:1062E400E0531E2FA0912208A63010F41A3008F0B3
:1062F40013C0103011F40E94771AE0913908EA9320
:10630400EAE8F7E1FA93EA930E9422700E9405708A
:106314000E948D7B0E94A063E0913A08E33411F05F
:106324000C94E131E0913B08EF3311F00C94E1312E
:10633400E0913D08E03319F4EFEFE0932308A091D6
:106344003C08A033F8F00E94BB73A0912208A63049
:10635400C8F4E0912308EF5FE0932308E09122085A
:10636400EA93E0912308EA930E94F31AA0911E0C89
:10637400B0911F0C109721F4A0912308A03408F0C9
:1063840001C0E7CFE0912308EA930E94DD180E9440
:10639400C773EDE8F7E10E94B1720E94C56E0E94D6
:1063A400CC730E94D1730E94CA6E0E948D7B0E949E
:1063B400D1730E942C6F0E9421630E947063E0914C
:1063C4003A08E434A1F5E0913B08E43481F514E0A3
:1063D400E1E0E0933909103538F40E942871E85C53
:1063E400F74FE081E03208F41AC00E942871E85C9B
:1063F400F74FE081E33259F40E942871E75CF74FCC
:10640400E081E053EA930E94425E1F5F06C00E944F
:106414002871E85CF74F0E94FB711F5FDCCF0E947C
:10642400C773E0E9F7E10E94B1720E9470630E94B1
:10643400637D269608951A930A930E94D97111F4E4
:106444000C949932E0E0E093590CE0911808EF774E
:106454000E2F009318080E94BD460E94636DE4E06D
:10646400F0E0FA93EA930E949646013021F0A0915D
:106474001908A13009F00BC0EEE8F5E00E94686D40
:1064840098D9E4EFF1E00E941E6C0E94BD460730EB
:1064940049F40E94CC20E0E0E0931B080E94F11133
:1064A4000E947428043031F4E3E9F7E10E94686D36
:1064B4000E94B50D083019F40E94D7736FD10530CE
:1064C40019F40E94D77356DC013051F4E89423F890
:1064D400E0E0EA9356D90093190837D90E94000FD7
:1064E400093071F4E0E0EA934CD9E0E0E0931E084F
:1064F400E89423F80E94000F0E94E173E093590C82
:10650400023069F4E0E0E0931E08E0E0F0E00E946D
:10651400D472E89423F80E94E173EA93A2DB033077
:1065240011F40E947640009319080E948D1FA091D7
:106534001908A73011F00C944733E091520CF091F4
:10654400530C0E94826E21F0A0911B08A03009F028
:106554000AC00E946472E0914E0CA0912306EA17CF
:1065640011F00E9474280E94F842E030E9F0E2E061
:106574000E941D731A93FFD91D3409F4B6D81D3334
:1065840099F40E94DD457EDAEF3F41F0E3E0E093C9
:1065940018080E9424730E946A7306C0E7E8E09317
:1065A4001808E0E0E0931B08A0912F08A03031F018
:1065B400E0912F08A0912E08EA1709F457C0E09142
:1065C4002F08E150EA930E943219A091340CE1E0C3
:1065D400EA23E13021F4E0912B06EF7C09F429C091
:1065E400E0E0E0932E08E0914C0CE03019F0E093E9
:1065F40018081EC012E0E0912B06EC7009F018E0B8
:10660400E091C40BA0912F08EA1781F0E0912B06CA
:10661400E07439F011E0EAE2EA93E8E9F7E10E9474
:10662400C173E0912B06E07809F019E01093180883
:106634001DC00E94BD460E94F1110E94636DE4E0FA
:10664400F0E0FA93EA930E949646EBE4EA930E9400
:106654003446E0912F08EA930E946541EBE9F7E1A3
:106664000E94686DE0912F08E0932E08A0912F08F6
:10667400A03021F4A0912E08A03009F406C0E0E077
:10668400E0932E08E7E8E0931808A0911908A330D6
:1066940011F40E94733EA0911908A13009F4D9D8CD
:1066A400A0911908A23009F4F8DAA0911908A830C9
:1066B40009F409DCA0911908A53009F487DBA0913D
:1066C4001908A93049F4E0E0E0932008E0911908A2
:1066D400EA93E0E0EA9380D90991199108950E9420
:1066E400E873E652F84FA6E0A0830E94E873E752ED
:1066F400F84FAB81A0830E94E873E152F84FAA815E
:10670400A0830E94E873E552F84FA881B981A08361
:10671400B1830E94D3710E94F250249608950E947E
:10672400EE73A881B981AC91A53020F0A881B9811C
:10673400E0E0EC9387C0A0911308BB27E091120816
:1067440005C0A0911108BB27E0911008F0E0319634
:106754000E9474703596DF01E5E0F0E00E94337B1F
:1067640008951A9310911308E0911208E117A1F00B
:10677400ABE01A9FF001E652F84FE081E13011F0EE
:10678400E23011F4E1E04BC0EDB7FEB7FA93EA93BF
:106794001F93C5DF1F91E8CFE0E041C01A930E9428
:1067A400CC20ECEDF5E00E9439700E94E46C0E946C
:1067B400956810E0153068F40E94A770AFEFA083CD
:1067C400ABE01A9FF001EE51FA4F0E945F721F5F17
:1067D400F1CF10E0153048F4A7E11A9FF001EC5C0A
:1067E400F94FAFEFA0831F5FF5CFE0912B06E37065
:1067F40019F00E94407309F402C0689401C0E8943F
:1068040021F8EFEFE0932D08E091E20BE03029F45A
:106814001BD06CD1E89420F802C00E94850F199116
:1068240008951A9310E0153058F40E94A770E0817F
:10683400AE2FE981EA1711F4E12F03C01F5FF3CFF4
:10684400EFEF18812296089522970E945C7D00E064
:10685400053058F40E94F473A0E00E94FA73E152E8
:10686400FA4FA0E0A0830F5FF3CF00E00530C0F53E
:106874000E944372E081EF3F89F10E944372E081FC
:106884000E94B670B9F00E944972DF010E947A7BBF
:106894000E948470EA17FB0751F00E9449720E941B
:1068A4008470A083B1830E94FF73A1E0A0830E943F
:1068B400F47312C0ABE00A9FF001EA51FA4FE08191
:1068C400E03061F40E944372AFEFA0830E944972EA
:1068D4000E945F720E94FF73A1E0A0830F5FC6CF86
:1068E4000E94AD1E1E2F1F3F11F0E1E001C0E0E049
:1068F400E093590C1F3F11F40C94D23450E000E0A3
:10690400053048F40E944372E0811E1711F451E0EF
:1069140002C00F5FF5CF5030E1F500E00530C8F557
:106924000E944372E081EF3F91F50E94437210830D
:106934000E9449720E948470A083B183ABE00A9FD5
:10694400F001E052FA4FA091290C0E94FA73EF5122
:10695400FA4FFF93EF930E94B1700E94BE6FAF9104
:10696400BF91EC930E94FF73A1E0A0830E94F47393
:10697400A1E00E94FA73EC51FA4FFF93EF930E9447
:106984000968AF91BF91ED93FC9351E002C00F5F92
:10699400C5CF503029F01A930E94B41E1E2FAACFDF
:1069A40030E0353010F00C941835A7E13A9FF0012F
:1069B400E15DF94FEE83FF8350E000E0053048F5D8
:1069C400503029F5ABE00A9FF001EF51FA4F2081D6
:1069D4002A930E94DD180E94F473E081E13059F497
:1069E4002A930E94CE1FE13031F4A32FAF5FE091D0
:1069F4009D0BEA1709F00BC0E22FAE81BF811396FD
:106A0400EC93E02FAE81BF811596EC9351E00F5FBC
:106A1400D5CF503049F4AE81BF811396EFEFEC939C
:106A2400AE81BF811596EC933F5FBBCF0E94637D1F
:106A34000C94C0370E945E7DAC81BD81EBE4EC9385
:106A4400EC81FD813196FA93EA930E940574E05239
:106A5400FA4FE0810E945C6C00E00E940E74EC919D
:106A6400E03011F00F5FF9CF0E940E74E0E2EC9376
:106A74000F5F0E9414740E94106D0E940574EE5101
:106A8400FA4FDF010E94C16D0E941974EE81ABE0E0
:106A9400EA9FF001EF51FA4F10811A930E94DD181A
:106AA40000E00E940E74EC91E03011F00F5FF9CF1A
:106AB4000E940E74E8E7EC930F5F0E940E74E0E20C
:106AC400EC930F5F30E03A3060F40E941474EA0FE4
:106AD400FB1F0F01AAE8BBE00E9420740F5F3F5F19
:106AE400F2CF0E940E74EC930C94053864970E94C4
:106AF4005E7D00E010E0153040F40E94A770E08154
:106B0400EF3F09F40F5F1F5FF6CF053021F0A0912E
:106B14002D08A03009F406C0E0E0E0932D08EA93C4
:106B24000E949E1010E0153088F5ABE01A9FF0012A
:106B3400E152FA4FE081E03039F11A9FF001E3525B
:106B4400FA4FE081E030B1F01A93FE0135960E94CD
:106B54004F72ABE01A9FF001EF51FA4F30813A9334
:106B64000E94DD181A93FE013596FA93EA930E9467
:106B7400F9100AC01A930E94E910ABE01A9FF001C1
:106B8400E152FA4FA0E0A0831F5FCDCF053021F47E
:106B9400A0912D08A13009F406C0E1E0E0932D088E
:106BA400EA930E949E100E94657D689608950E9453
:106BB4005C7DA091E20BA23011F40C949F3930E07B
:106BC400343168F40E9427740E942A74DA01129600
:106BD400E0E0EC93DA01EFEFEC933F5FF1CF0E943A
:106BE400AD1E0E2F0F3F11F0E1E001C0E0E0E09395
:106BF400590C0F3FA1F10E94B170FA93EA930E94DD
:106C04008D181E2F1F3F31F1A0911E08E12FEA1BA2
:106C14003E2F3431F8F40E9427740E942A74FA013A
:106C240032960F01E081AE2F0E943074B0E0EA0F7B
:106C3400FB1FD001EC93FA01A281A43620F0DA0103
:106C44001296E3E6EC93DA01AC91AF3F19F4E02F2E
:106C5400DA01EC930A930E94B41E0E2FCACF0E944D
:106C64002F1530E0343110F00C94BE360E94277496
:106C74000E942A74FA01A381AF3F11F40C94BC362C
:106C84000E9435740E94B46FE83139F40E9435745F
:106C9400EA930E94D417E03009F408C00E943574C6
:106CA400EA930E94D417DA011296EC93A0919A0BFE
:106CB400A07839F4FA010280DA011196EC91E0151A
:106CC40009F458C0DA0113962C91ADE02A9FF00123
:106CD400EF5EFC4F0F01DA011296EC91D001EC93B8
:106CE4000E943574EA930E94E220EF3F29F0ADE060
:106CF4002A9FF0010E94156DDA011296EC91E030A2
:106D040089F00E943A74DF010E94306DEC93ADE08B
:106D14002A9FF001E25FFC4FDF01E091980BEF70D6
:106D2400EC9313C00E94306DE03021F40E943A7459
:106D3400A0E003C00E943A74A8E0A083ADE02A9FBB
:106D4400F001E25FFC4FA7E0A0830E943574EA9350
:106D54000E94E220EF3F19F0ECE0E0930F04DA0127
:106D64001296EC91DA011196EC932A93E1E0EA93FE
:106D74000E941F473F5F76CF0C949F39E7E0E09372
:106D840018080E941618A8950E94741CA8950E94C1
:106D9400C91EA895EFEFE093B20BE093890BE09343
:106DA400330CE0932E0CE0932E060E944074EC7F8B
:106DB40029F0A8E0B0E0E0E00E94BC7B08952497AD
:106DC4000E945E7D0E941342E8EAF7E10E94397056
:106DD4000E949F420E943B42E0912208E03061F011
:106DE400E3EBF7E10E9439700E949F42E091220890
:106DF4000E9445740E9449740E943B420E94771A83
:106E040000E00A30A0F40A930E940C190E94526F09
:106E1400EFE0EA930E947942E02FA3EAB6E00E94F1
:106E24004D740E9405700E9451740F5FEACF0E9456
:106E34004D42ECEBF7E1FA93EA93EFE0EA930E9418
:106E44009F420E94926E0E9451740E944F420E947F
:106E54003B4210E0103110F00C94BC370E94CE6D10
:106E6400E117E1F5E2ECF7E10E9439700E949F42DC
:106E74000E94516D0E944974E0E0E0931E08A091C5
:106E84001E08A03448F5E0912208EA93E0911E0818
:106E9400EA930E94F31A0E94C56E3097B9F0E0910C
:106EA4001E08EA930E94DD180E94C56EFA93EA93C5
:106EB4000E9457740E949F420E942C6FEAE0EA935A
:106EC4000E9479420E94CA6E0E945174E0911E0889
:106ED400EF5FE0931E08D3CF0E945C740E94287178
:106EE4000E940A7011F00C94BA37E2ECF7E10E94A8
:106EF40039700E949F420E94516D0E9449740E9401
:106F04006074E0E30E94167029F40E941B700E94D2
:106F1400C9619F0100240216030644F50E94B87358
:106F24000E94F3610E94356E0E94B8730E946874D7
:106F34003A932A930E9457740E949F420E946C7451
:106F4400EAE0EA930E947942EC81FD816E817F81BF
:106F54000E9451740E946074E1E30E94167029F447
:106F64000E941B700E94C9619F01D4CF0E945C746F
:106F74001F5F70CF0E9414420E94657D2896089579
:106F84000E945E7DAD81BE812C910E9471740E942D
:106F9400516D0E94846C0E94CA6DECE3EA930E94D6
:106FA4003446EC81EA930E9488462A93ED81EA9361
:106FB4000E940541EEE3EA930E9434460E94F17276
:106FC4000E9491720E94F7720E947674333409F41D
:106FD40031E2313320F0EC81E05DE31708F407C0BF
:106FE400E32F0E943D73E255FF4FE4912E273D337A
:106FF40011F0313209F401C0CACF3D3319F4AD8127
:10700400BE812C93E32F0E94657D279608950E94EC
:107014005C7D20E0AF81B8855C910E9471740E9410
:10702400516D0E94846C0E94CA6DE2E0EA930E9452
:1070340088465A930E9465410E94F1720E9491729F
:107044000E94F7720E947674303310F03A3308F0DD
:107054000EC0203009F450E021E0A52FEAE00E94A0
:10706400307BAAE0EA9FF001E30FE0535E2F3B324E
:1070740011F4533608F001C05F5F3D3211F4513012
:1070840008F401C05150333429F4203009F431E2BA
:1070940050E020E03D3319F4EE81E51708F005C017
:1070A400AF81B8855C9130E020E03D3311F031329E
:1070B40009F401C0B4CF3D3319F4AF81B8855C93B2
:1070C400D0C00E945C7D20E0AF81B8854D915C9179
:1070D4000E9471740E94516D0E94846C0E94CA6D5A
:1070E400AE81A23051F4E6E0EA930E948846FA01A8
:1070F4000E94CC730E94444108C0E5E0EA930E94D8
:1071040088465A934A930E944F410E94F1720E940A
:1071140091720E94F7720E947674303310F03A3301
:1071240008F01EC0203011F440E050E021E040316E
:10713400E7E25E0734F0DA01E0E1F7E20E94337B34
:10714400AF01493BEBE05E0724F0DA010E9438739B
:10715400AF01DA010E947B740E948074D097AD0164
:107164003B3221F44033E5E75E070CF002C04F5F89
:107174005F4F3D3221F40024041605060CF002C0D2
:1071840041505040333431F4203009F431E240E0CE
:1071940050E020E03D3311F0313209F401C09ACFC0
:1071A4003D3321F4AF81B8854D935C935AC00E945E
:1071B4005C7D0E94717420E050E04FEF0E94516D9D
:1071C4000E94846C0E9485740E948874E885EA9306
:1071D4000E946046E52FE10FF0E00E9491720E9448
:1071E400F7720E947674303310F03A3308F021C0FD
:1071F4003053431729F04F3F09F05F5F20E005C08B
:10720400A22FAF5FEA2FE3702E2FE52FAF81B88551
:107214000E948D740F01E32FA6ECB6E00E944D741A
:10722400AE0FBF1FE22F0E948D74E491D001EC9346
:10723400432F3B3219F4EE815E1708F002C05F5F02
:107244004FEF3D3211F4513008F402C051504FEF6A
:10725400EE815E1720F4313211F03D3309F401C0A0
:10726400ADCFE32F0E94637D299608951A930A9364
:10727400A0919A0BECEDEA231E2F00E00D3040F4B0
:107284000E9491740E949574E11711F00F5FF6CF7C
:107294000E949174EA0FFB1F0E94897B0E94686D13
:1072A400E02F3DC4AAE9BBE00E94B96DAE0FBF1F39
:1072B400EC91E17011F4E3E701C0E9E4EA930E9480
:1072C4003446219608950E945C7D0E9471740E9448
:1072D400516D0E94846C0E948574C8DF5E2F0E94E9
:1072E400F1720E9491720E94F7720E9476743D328C
:1072F40011F0363311F4503009F401C051503B32CF
:1073040011F0333311F45C3008F001C05F5FA091D9
:107314009A0BE1E0EA232E2FE52FA0E0B2E00E94D1
:107324004D740E949574E20FE0939A0B3D3311F073
:10733400313209F401C0CBCFE32F0E94637D26963E
:1073440008950E945E7D0E9471740E94516D0E9496
:10735400846C0E948574AAE9BBE0EC810E94B06F42
:10736400EC91E17019F4EFECF7E102C0E3EDF7E121
:10737400FA93EA930E944B460E94F1720E94917222
:107384000E94F7720E947674303310F03A3308F09A
:107394000FC0AAE9BBE00E94D46F0F01AAE9BBE0C9
:1073A400EC810E94B06FAC91E1E0EA27D001EC934C
:1073B4003D3311F0313209F401C0C7CFE32F0E94ED
:1073C400657D259608950E946C6CE1E0EA930E9425
:1073D4009F0E0E94016C0E94016C0E9496460E94BE
:1073E4002C6FEAE0EA93E3DEE13209F45FC40E9421
:1073F400016C0E94016C0E94A26DE7EDF7E10E940E
:10740400686DE5E9FBE00E9439705BDEE13209F466
:107414004DC40E94016C0E94016C0E94A26DEDEDAE
:10742400F7E10E94686DE091970BEF5F0E2FEDB7C7
:10743400FEB7FA93EA930F93EAE0EA93E8DD0F913B
:10744400E13209F433C400240216030624F4E02FC5
:10745400E150E093970B0E94016C0E94016C0E9422
:10746400A26DE6EEF7E10E94686DECEAFBE00E9493
:107474009A7409F41BC40E94016C0E94016C0E945E
:10748400A26DECEEF7E10E94686DEEEAFBE00E946B
:107494009A7409F40BC40E94016C0E94016C0E944E
:1074A400A26DE2EFF7E10E94686DE9E9FBE0FA936F
:1074B400EA93E3E60E94A37409F4F8C30E94016C02
:1074C4000E94016C0E94A26DEBEFF7E10E94686DCF
:1074D400FADEE13209F4EAC310E0133010F00C9440
:1074E4002A3B0E94016C0E94016C0E94A26DE12F54
:1074F4000E94FB72E1E0F8E10E94686D0E94A874AA
:107504000E949646ADE9BBE00E9428710E94106D6E
:10751400E0E10E94A37409F4C9C3E9E0F0E00E9429
:10752400426C0E949646A0EABBE00E9428710E9429
:10753400106DE0E10E94A37409F4B8C30E94016CC9
:107544000E94016C0E94A26DE12F0E94FB72ECE08C
:10755400F8E10E94686D1A93F4DEE13209F4A6C3DF
:107564000E94A8740E94AC7451F40E94E3710E94BA
:10757400B674E2E00E94BA7409F498C309C00E9488
:10758400E3710E94B674E0E00E94BA7409F48EC3F9
:107594000E94016C0E94016C0E94A26DE12F0E9466
:1075A400FB72EEE0F8E10E94686D0E94A8740E94EC
:1075B4009646A9EABBE0EE27A10FBE1F2C91332704
:1075C400EDB7FEB73197FA93EA933F932F93E0E038
:1075D400EA9377DD2F913F91E13209F467C3A9EA79
:1075E400BBE00E942871EA0FFB1F2083123070F564
:1075F4000E94016C0E94016C0E94A26DE12F0E9406
:10760400FB72E5E1F8E10E94686D0E94A8740E9493
:107614009646A0EBBBE0EE27A10FBE1F2C913327AB
:10762400EDB7FEB73197FA93EA933F932F93E0E0D7
:10763400EA9347DD2F913F91E13209F437C3A0EB80
:10764400BBE00E942871EA0FFB1F20831F5F45CF18
:107654002DC30E945E7D10E01A930E9471730E94F4
:10766400BF740E94016C0E9496460E94DA6D0E94CB
:10767400C3740E945B6D0E94B96F0E94B56D0E9435
:10768400016C0E94636D0E9496460E94C76F0E941F
:10769400C66DE7E0F0E0FA93EA930E94636D0E94FE
:1076A4009646E091AE0BF091AF0B0E94987A0E943F
:1076B400C66D0E94016C0E94566D0E949646ECE1D4
:1076C400F8E10E94686DE091970BEF5FEA930E94E6
:1076D4006541E7E0F0E0FA93EA930E94566D0E9458
:1076E4009646C4DD0E94A66DE091990BE03029F026
:1076F400E091990BEA930E94654100E00330D8F5CC
:107704000E94016CE02FED5FF0E00E94CA6D0E94C0
:107714001072EA930E946541EBE2EA930E943446B8
:107724000E941772EA930E9465410E94A66D0E940E
:107734001E7251F40E9426720E94BC6D0E94C16D9B
:107744000E94C774E3E709C00E9426720E94BC6DC0
:107754000E947A7B0E94B56DE9E4EA930E94344664
:107764000E94A66D0E943072EA930E946B410E94AF
:10777400CB740F5FC3CF0E94FB423E2F3B3211F408
:10778400103408F001C01F5F3D3211F4113008F4C9
:1077940001C011503D3439F41A930E94DD1813DEF0
:1077A4001A930E94FD18313209F056CF7FC20E940D
:1077B4005E7D10E00E94BD46012F0E94016C0E9474
:1077C400016C0E949646E0E2F8E10E94686D31E0A7
:1077D4003C3018F51038F8F40E94016C0E949C6C3F
:1077E4000E94CA6D1A930E9432190E94DA6D0E9497
:1077F400A66DA091340CE3E00E94CF74A091350CE7
:10780400E7E00E94CF74E0912B06EA93E8E0EA9364
:107814000E94054113953F5FDBCF0E94B50D0E9486
:10782400FB423E2F3D34E9F50E94D972102F1038E7
:10783400C0F51A930E9432190E94016C0E94016CD7
:107844000E94A26DE4E3F8E10E94686D0E94DA6D83
:107854000E94C3740E94E16D0E949646E7E3F8E13A
:107864000E94686DE4E3FCE0FA93EA93E3E00E948B
:10787400A37409F41BC20E94E16D0E94A26DEDE3A2
:10788400F8E10E94686DE5E3FCE0FA93EA93E7E02F
:107894000E94A37409F40AC21A930E9466191F5F16
:1078A400C6CF313211F0103808F001C083CFFEC1C9
:1078B4000E946C6C0E94BF740E94016C0E949646E8
:1078C400E3E4F8E10E94686D10E01530F0F41A93D7
:1078D4000E9474190E94016C0E94A86E0E94DA6DC5
:1078E4000E94C374E0912F0C0E94D474E091320C76
:1078F4000E94D474E091300C0E94D474E091310C55
:10790400EA930E946B411F5FE0CF0E94FB420E2F5F
:107914000D34E9F50E94D97210E01530C0F51A93C0
:107924000E9474190E94016C0E94016C0E94A26D55
:10793400E6E5F8E10E94686D0E94DA6D0E94C37466
:1079440030E03430F8F40E94E16D0E94A26D0E9490
:107954009C6C0E948B7AEA55F94F0E94897B0E94A5
:10796400686D0E949C6C0E948B7AEA55F94F0E94C4
:10797400D874FD013596E4910E94A37409F496C16C
:107984003F5FDFCF1A930E9494191F5FC6CF8EC149
:107994000E94DD6BE1E0EA930E949F0E00E0083252
:1079A40010F00C94913D0E94810D0E94016C0E9484
:1079B400016C0E9496460E94846C0E94DB740E94B3
:1079C400897B31960E94686D0E94A66D0E94846C2A
:1079D4000E94DB743496E491E038A9F40E94CE6DE1
:1079E4001E2FEDB7FEB7FA93EA931F93E0E1EA93F3
:1079F4000EDB1F91E13209F492C0E12FA9E0B0E05F
:107A04000E94BC7B88C0E238A9F40E943E701E2FFD
:107A1400EDB7FEB7FA93EA931F93E0E1EA93F7DA3E
:107A24001F91E13209F47BC0E12FAAE0B0E00E948B
:107A3400BC7B71C0E138E1F40E9440741E2FEDB7A5
:107A4400FEB7FA93EA931F93E3E0EA93E0DA1F9117
:107A5400E13209F464C00E94810D0E944074E11770
:107A640031F0E12FA8E0B0E00E94BC7BFFCF53C00F
:107A7400E03069F40E94846C0E94DB7432960E94A8
:107A84006C6DE1E00E94A37409F449C044C0E13084
:107A940069F40E94846C0E94DB740E94D874FD0116
:107AA4003596E4910E94A374D1F135C0E23061F4BB
:107AB4000E94846C0E94DB7432960E946C6DEFE02D
:107AC4000E94BA7461F127C0E33071F40E94846C9F
:107AD4000E94DB740E94D874FD013596E491EA9308
:107AE4004FDAE132E1F017C0E430A9F40E94846C6B
:107AF4000E94DB7432960E94897BE0935A0CF093C7
:107B04005B0C0E9491720E94DB743596E491EA93B7
:107B14004EDBE13221F00E9419180F5F40CF09912A
:107B240019910895E8810E94FB72EAEDF7E10E9441
:107B3400686D0C9411421A930E94D97210E01330AC
:107B440010F00C94F63D0E94016C0E94016C0E949E
:107B5400A26D1A93E7DFECE0F0E00E94426C0E9411
:107B640096461A939FDB0E94A8740E94AC7451F449
:107B74000E94E3710E94B674E2E00E94BA7409F4B0
:107B8400FFC209C00E94E3710E94B674E0E00E9443
:107B9400BA7409F4F5C2123028F50E94016C0E94EF
:107BA400016C0E94A26D1A93BDDFE9E5F8E10E9421
:107BB400686DECE0F0E00E94426C0E9496460E94E0
:107BC400CB74EAE0F0E00E94426C0E949646A0EB7F
:107BD400BBE00E9428710E94106DE3E60E94A3742A
:107BE40009F4CEC21F5FABCFCBC20E945E7D10E012
:107BF4001A930E9471730E94BF740E94016C0E94C8
:107C040096460E94DA6D0E94C3740E945B6D21E067
:107C140000E0033080F5E3E0F0E00E94B36C0E94E2
:107C2400CA6D0A937FDF0E941E7249F40E94267275
:107C34000E94BC6D0E94C16D0E94C77408C00E945E
:107C440026720E94BC6D0E947A7B0E94B56D0A93D5
:107C540029DB2F5F023068F4E7E0F0E00E94B36CA8
:107C64000E94CA6D0E9429720E94DF6D0E94CB742B
:107C74002F5F0F5FCECF0E94FB423E2F3B3211F4A9
:107C8400103408F001C01F5F3D3211F4113008F4C4
:107C940001C011503D3439F41A930E94DD184BDFB2
:107CA4001A930E94FD18313209F0A2CF0E94657D1B
:107CB400249608950E94D9720E94016C0E94016C5E
:107CC4000E949646EFE5F8E10E94686DE1E0E093DA
:107CD4002208E2E2F8E0FA93EA93E5E0EA9397D91E
:107CE400089522970E945C7D0E94FB420E2FE09132
:107CF4001B08E03011F00C9424400132D1F4EAE482
:107D0400F6E0A0913A0CB0913B0CEA17FB0761F442
:107D1400E7E0E0931808EAE2EA93E8E6F8E10E9473
:107D240039700E94AD63A8C0E0E0E093C0050E94F2
:107D3400E0740D3331F4E091C005F0E00E94A26CD0
:107D440004910D3441F4EAE2EA93EBE6F8E10E948F
:107D540039700E94AD63063449F4E2E7F6E0E0933B
:107D64003A0CF0933B0CE0E0E093C005003311F0D3
:107D74000B3229F4E091C005EF5FE093C0050D32AA
:107D840029F4E091C005E150E093C005013329F4E2
:107D940091DFED3311F40E94E774033321F48ADF99
:107DA400ED3309F40CD8063329F4E0E0E09322081B
:107DB4000E94E136043329F4E0E0E09322080E94B3
:107DC400E774A0912408A13010F40C94BA3F023354
:107DD40001F570DFED33E9F40E94F474D1F4E0911D
:107DE4002208EA930E942D1B30E0303190F40E9467
:107DF4009C6C0E940A7059F4E32FE05DEA93EEE66E
:107E0400F8E10E940F70E0E3EA930E94CF633F5FC2
:107E1400ECCF053331F5E0E0E09322080E94F474DE
:107E240001F511E01630E8F41A930E942D1B30E09E
:107E34003031A8F40E949C6C0E940A7071F4E32F04
:107E4400E05DEA93EEE6F8E1FA93EA93E12FE05D70
:107E5400EA93E0E3EA930E94CF633F5FE9CF1F5FB9
:107E6400E1CF013469F4EAE2EA93E1E7F8E10E9440
:107E7400C173E1E0E09318080E94637D2896089599
:107E84000A3409F4B2DE073311F00C94BA3F0E94AD
:107E9400BD46E0E0EA930E94E60DE1E0E0931C08B1
:107EA400E0E0F0E0E0931408F0931508EFE2F6E068
:107EB4000E943970E3E7F0E00E94EB6F0E940968CA
:107EC400EE83FF830E94FD74E8E2F0E00E94A1705B
:107ED400B9F00E9434120E940968EE83FF83A091D6
:107EE400190CA03021F00E949D33E03009F408C041
:107EF4000E94E873E652F84FAEE0A0830E94D3716B
:107F0400E5E0F0E00E941E6C40E050E00E94952104
:107F1400E03868F00E949521EF573E2F313010F081
:107F2400313108F004C0E32F0E94F570AF015A9379
:107F34004A930E94671F40931408509315080091B8
:107F4400DB05E0E0E093DB05013211F00B3209F4CC
:107F540001C0B8CF0B3221F4E1E0EA930E94E60DB0
:107F6400013209F0A3CFE0E0E0931C08E093DB05C5
:107F7400A0912408A23011F00C941D40093309F497
:107F840007DD053409F494DC033611F40E94290D4D
:107F9400083309F45EDB023409F409DC0334B1F577
:107FA4001091390C0E94BD4600E0E091380CE117B5
:107FB40011F00C3008F01DC00E94016C0E94846C0A
:107FC4000E94CA6D1A930E94BB1E1A937CD10E9410
:107FD400A66DE091290C0E94D474E0912C0C0E94AF
:107FE400D4740E94B1700E94B56D0E94977003957D
:107FF400DCCF0E94B50D0E94FB420E2F013221F00E
:10800400E091380CE11709F401C0CCCF043499F4A1
:108014000E94F47481F4A091D30BA03021F4A091B8
:10802400D10BA03031F00E9445730E94016C0E9474
:1080340022530E94091DE0911B08E03011F40E94B4
:108044003E0E49C0E130D1F4A0912108AB3010F4C8
:10805400013209F405C00E94C6150E94B50D0DC079
:10806400E0E0E0931E080E9402750E94C173E0E004
:108074000E940775E2E0E0931B082DC0E23059F539
:10808400013269F4E0E0E0931B080E94BD46EAE295
:10809400EA93EBE6F8E10E94C1730E943E0E0B32B4
:1080A40011F00D3359F40E940275FA93EA93E1E357
:1080B400EA930E94AD63E1E00E9407750D3259F422
:1080C4000E940275FA93EA93E2E3EA930E94AD6395
:1080D400E2E00E940775A0911808A33009F404CEC9
:1080E4000E94637D0C9467451A93E3E0E0931908BA
:1080F4000E94BD460E94016C0E94016C0E9496463B
:10810400E7E7F8E10E94686D0E94016C0E94636DCC
:108114000E949646E3E1F6E00E943970E0E1F0E067
:108124000E94EB6F10E0E091C90B1E1700F50E944E
:10813400CE6DE117D1F0E12FE05DEA93EFE7F8E1CE
:10814400FA93EA93E0E3EA93E0E00E94167049F4BC
:108154000E942871ED5EF94FA1E0A083E12FE05D5C
:1081640001C0EEE2EA930E9434461F5FDCCF0E9416
:10817400E074E0E0E093C005E0931B080E943E0E2B
:1081840019910895E881E03021F4E4EFF6E00E94CB
:108194000C75A881A13021F4EEEEF6E00E940C7576
:1081A400A881A23021F4EAEFF6E00E940C75A881C0
:1081B400A33021F4E8E0F7E00E940C75A881A43014
:1081C40021F4EEE0F7E00E940C7529C11A930A939A
:1081D400E0E0E0937D05E0937E0510E0143190F437
:1081E40000E0033068F4A3E01A9FF001EC57FA4F63
:1081F400DF01EE27A00FBE1FE0E2EC930F5FF1CF8B
:108204001F5FECCFE9C31A9311E0E981E11780F015
:108214000E942871E255FF4FE491AA81EA2319F0E4
:10822400E12FE05D01C0E0E2EA931CD51F5FEDCFD2
:108234002DC51A9311E0E981E11778F00E942871A5
:10824400E255FF4FE491AA81EA2311F0E1E301C072
:10825400E0E3EA9307D51F5FEECF18C52A97A091F4
:108264001B0CA13038F0EA85FB856C857D850E9466
:10827400C77407C00E9411750E9415750E9411757C
:10828400F9D426C12A970E9411750E941E750E9476
:1082940027750E941175EED41BC12A970E9411758F
:1082A4000E943A750E944175E5D41FC12A970E9425
:1082B4001175EDE9F8E10E9446750E94CC730E94A5
:1082C4004175D8D412C12A970E941175E0EAF8E1E9
:1082D40005C02A970E941175E4EAF8E1FA93EA933B
:1082E400EE850E945C6C0E941175C4D42B9608958F
:1082F4000E945E7D10E0E1E3E0933809E89431F8F0
:10830400EA930E945563E8EAF8E10E94B17200E042
:10831400E09182050E17E0F40E94846CEC57FA4F4A
:10832400E081E03258F4E3E2EA930E9497620E940B
:10833400846CEC57FA4FE081E05D05C00E94846CC8
:10834400EC57FA4FE081EA930E9497620F5FE0CF07
:108354000E944B759F010E9438153A932A93E8ECCA
:10836400F0E0FA93EA930E9415680E2FA0E031FC26
:10837400A1E0A03011F4003009F001C0ECCF31FECF
:1083840009C0E0E0E0938205E89431F8E1E00E945E
:10839400657DEFC41F5F123008F4ADCFE0E0E093D9
:1083A40082050E94657DE5C4E0918105E03021F4F9
:1083B400E881EA930E94425EA0918105A13069F4AC
:1083C400A0E09299A1E0A13021F4A8950E94D36E77
:1083D400F7CFE881EA930E94E260A0918105A23080
:1083E400F1F4E0918205F0E0EC57FA4FA881A08304
:1083F400E0918205EF5FE0938205E0918305EF5FF2
:10840400E0938305A03218F4EF5FE0938305A09115
:108414008305A83320F06CDFE0E0E0938305219628
:10842400089508950E945C740E945C7422D0EBE16C
:10843400EA93BADFE9E6EA93B7DFA0918105A130B8
:1084440061F4E8ECF0E00E943E6EE0919A00E0698D
:10845400E0939A00E9E1E0939900A0918105A230AC
:1084640021F446DFE0E0E0938305E0E0E09381055A
:108474000895EDE0EA9398DFEAE0EA9395DF089542
:108484001A9310E0E9811E1728F4EA81EA938CDF3D
:108494001F5FF8CFFBC3EDE201C0EDE3EA93E8E22E
:1084A400EA93EEDFE6DF08952A97A0911B0CA13032
:1084B40038F00E9411750E941E750E94277504C031
:1084C4000E9411750E941575FE010E9439700FD02B
:1084D4002E9608952A970E9411750E943A750E945B
:1084E4004F75FE010E94397002D02C9608951A939C
:1084F4000A9310E0EA81E03011F408E201C00A8135
:10850400AB81BC81EE27A10FBE1FAC91A03011F04E
:10851400101708F007C0AB81BC810E9454750E94FB
:108524005975EECFEA81E03039F0EA811E1720F464
:10853400E0E20E945975F9CF27C01A930A9310E01C
:10854400EA81E03011F408E201C00A81E12FAB8135
:10855400BC810E948D74E491E03011F0101708F092
:1085640009C0E12FAB81BC810E948D74E4910E940B
:108574005975ECCFEA81E03039F0EA811E1720F416
:10858400E0E20E945975F9CF198108812596089572
:10859400E091C405A091C305EA17B1F00E945E758D
:1085A4000E94BC6DEC91E093C6050E945E750E942A
:1085B4004271E181E093C505A091C4050E946475F0
:1085C400E093C405E1E00895E0E008950E94697530
:1085D400A981A0830E9469753196A881A083A09186
:1085E400C3050E946475E093C305BFC0E091DB0539
:1085F40008951A93E091DB05E03059F40E94381590
:108604000E94D97121F4A091DB05A03009F001C0CA
:10861400F5CF1091DB05E0E0E093DB050E94D97112
:1086240009F011E2E12FD6C30E945E7D0E94096821
:108634008F010E943815EC81FD81E00FF11FFF933B
:10864400EF930E940968AF91BF91AE1BBF0B9D01D0
:108654000024021603061CF40E94D97109F001C01B
:10866400E8CFE0E00E94657D269608951A93E9819B
:108674000E943D72A0E0A0830E946F75108117FFD5
:1086840005C0E12F0E947675A0E0A08316FF05C007
:10869400E12F0E947D75A0E0A0830E946F75A0E089
:1086A400A083E9810E943772A0E0A08318815DC095
:1086B4000E945E7D30E0EE81ADE0EA9FF001E05F74
:1086C400FC4F108116FF17C0E12FEF730E2F0E948D
:1086D400847511F03A3008F009C00E948C75DF01EE
:1086E4000E949C6C0E9492753F5FF1CF0E948C7532
:1086F4000E948074EC9317FF17C0E12FEF730E2FC5
:108704000E94847511F0343108F009C00E949875F4
:10871400DF010E949C6C0E9492753F5FF1CF0E9422
:1087240098750E948074EC930E94657D42C2E88132
:10873400F9810E946C6DEA81FB8132960E946C6D16
:10874400EC81FD8134960E946C6DEE81FF8136963A
:108754000E946C6DE885F9853896E491EA93E98581
:10876400FA8539960E94816C02D022960895A097CA
:108774000E945C7DEDA5FEA5A9A9BAA9EA0FFB1F7D
:10878400AF01E5E0F3E0EE83FF8310E01431C0F5C0
:10879400AE81BF81AC91A03049F1EE81FF81A3810C
:1087A400B481EFA5F8A9EA17FB0701F5EE81FF8173
:1087B400A181B281E9A9FAA9AE17BF07BCF0EE8185
:1087C400FF81A181B2814A175B0784F00E949E75E4
:1087D400AE0FBF1FE9A9FAA9AE17BF073CF00E946C
:1087E4009E75AE0FBF1F4A175B070CF402C01A93A5
:1087F4003DDFEE81FF813D96EE83FF831F5FC6CF91
:10880400E5E0F3E0EE83FF8310E0143110F00C9404
:10881400AE44AE81BF81EC91E03011F00C94A744DA
:10882400EAA5EC93E9A9FAA9AE81BF811196ED936B
:10883400FC93EFA5F8A9AE81BF811396ED93FC9349
:10884400EDA5FEA5AE81BF811596ED93FC93EBA536
:10885400AE81BF811796EC93E0910904A0910F04B7
:10886400EA27AE81BF811896EC93E0911004AE81A3
:10887400BF811996EC93E0911104AE81BF811A96E1
:10888400EC93AE81BF811B960E941D6D1C96E0E0A7
:10889400EC93E887E8A5F9A5309741F00E94A97503
:1088A4000E94AE75E4E1EA930E94F468EEA1FFA190
:1088B400309751F00E94A975E8A5F9A5FA93EA93B7
:1088C400E4E1EA930E94E068E0E0EC8F0E94A9757D
:1088D4000E94CB683E2F3B30C8F000E00E949875A0
:1088E400E081E03011F0053008F002C00F5FF6CFF0
:1088F4000E949875E081E03049F40E9498750E94C6
:10890400B375E058AE81BF811B96EC93E0E0EA8B2F
:108914003130C8F000E00E948C75E081E03011F045
:10892400043108F002C00F5FF6CF0E948C75E0811D
:10893400E03049F40E948C750E94B375E05CAE810E
:10894400BF811B96EC93E12F08C0EE81FF813D9619
:10895400EE83FF831F5F59CFEFEF0E94637DE396A1
:1089640008951A930A930E94BE753097A9F1E09175
:108974006205E03061F50E94BE75049000926205C4
:10898400E0916205E03031F4E0E0F0E00E940C7523
:10899400E0E01AC00E94C3750E94BE750E94897BE4
:1089A400F595E7958F01D801E0E0F1E00E94017BA5
:1089B400E0938700D801E0E0F1E00E94337BE0938C
:1089C40086000E94C375E0E4E0938B0005C0E0914B
:1089D4006205E150E09362050991199108950E949E
:1089E4005E7D00E025E033E010E01431B8F5D901F4
:1089F400EC91E03079F111960E947A7B0E94CB755C
:108A040024F5D90113960E947A7BAC81BD81EA17C3
:108A1400FB07DCF4F90101801280D90115960E944C
:108A24007A7BE00DF11DAE81BF81AE17BF076CF4F8
:108A3400F90103801480D9011796EC910E94DF712B
:108A4400AC81BD81AE17BF070CF004C0E12FEF5F0E
:108A54000E2F04C0235F3F4F1F5FC7CF003049F084
:108A6400E0916305E01721F0A0916305A03009F4BB
:108A740001C022C0A0916405A53079F40A93E1E015
:108A8400EA93A4DD0093630500936505D901EC9195
:108A9400E0936605E3E0E0936105A0916405AE31DF
:108AA40019F4E4E0E0936105A0916105A33018F0A6
:108AB400E5E0E093680507C0E0E0E0936405E09337
:108AC40061050E94D0750E94657D28960895E09105
:108AD4006305E03091F0A0916405A93220F4EA9393
:108AE400E2E0EA9373DDA0916405AD3330F0E091E8
:108AF4006305EA93E4E0EA9369DDE0E0E09361056D
:108B0400E09364050E94D075E0E0E0936305E09390
:108B14006705089530D15ADB0895EA81E0937F0513
:108B2400E881E0938005E0910A04E061E0930A049F
:108B340020C10E945C7DA0917F05A43120F4A09106
:108B44008005A33008F033C0E0917F05F0E0ACE08D
:108B5400B0E00E94D67A8F01E0918005F0E0A4E1B4
:108B6400B0E00E94D67A9F010E94D675ECE0F0E056
:108B74000E94DB75F0E00E94897A0E94276CEE81E6
:108B8400E030A9F0E0917F05A3E0EA9FF001EC5703
:108B9400FA4FDF01E09180050E94B06F4C91552798
:108BA4000E94D6754A93EFE0EA930E94544D0E94C6
:108BB400637D27960895E0910A04E07141F0E2E0B4
:108BC400EA93B7DFE0910A04EF7EE0930A04089584
:108BD4000E94E075AF3EE0E0BE0744F4A0910203BA
:108BE400B0910303AF33E1E0BE070CF039C00E943B
:108BF400E5750E94C26F0E94544DA0915D05B0912D
:108C04005E05549734F4A0915F05B0916005139705
:108C14000CF012C0E0915D05F0915E05A3E0B0E0B8
:108C24000E94AE7AEC57FA4FA0915F05B0916005AF
:108C3400EA0FFB1FA981A083E0910D04ACE0EA9F39
:108C4400F0010E94E0750E948D740E94F275E0911B
:108C54005D05F0915E053196E0935D05F0935E0548
:108C64000C94994AE881EA93E0911004EA93B0DF06
:108C74000C94684A1A9310E00E94F775E03031F0C2
:108C84000E94F775EA93EEDF1F5FF6CF18812396F3
:108C940008950E94FA750E94FF75E03021F00832B1
:108CA400E0E01E070CF007C00E94FF75EA93DADFCC
:108CB4000F5F1F4FF0CF198108815BC00E94FA75C6
:108CC400F801AB81BC810E94067621F0EA810E9402
:108CD4000B760CF009C0F801AB81BC810E941076C0
:108CE400C1DF0F5F1F4FECCF198108810EC30E94B3
:108CF4005E7D0E94E0750E94157631978F010E9477
:108D04001A760E94D6750E94227633C00E945E7D38
:108D1400AC810E9429760E2F11270E941A760E9498
:108D2400D6750E942276F1C2EA81FB81E0935D054B
:108D3400F0935E05E881F981E0935F05F0936005A7
:108D4400AA81BB81ECE0F0E00E94D67A0E94F27521
:108D5400A881B981E4E1F0E00E94D67A06C0EA81F4
:108D6400FB810E94F275E881F981E0930203F0939C
:108D74000303249608950E943176143120F41A9343
:108D840075DC1F5FFACF0E94016C0E94016C0E9487
:108D9400226CEFE3F1E00E94276C10E0153048F4F8
:108DA400A5E11A9FF001E051FB4FA0E0A0831F5FF3
:108DB400F5CF10E0143148F4ABE01A9FF001EC5EFB
:108DC400FB4FA0E0A0831F5FF5CFE0910A04EF7E84
:108DD400E0930A04199108950E943176143100F544
:108DE400ADE01A9FF001BF01E85FFC4FDF010E9474
:108DF4007A7B0F01DF01EB81FC81AE17BF075CF0CA
:108E0400E981FA81E015F10534F0FB01E05FFC4FE4
:108E1400E081E03009F402C01A9328DC1F5FDECF42
:108E24000E94016C0E9439760E94226CA985BA8541
:108E34000E943E760E94276C67C2A2970E945C7DC6
:108E4400E9A50E943D728F01D8011B96EC91E03098
:108E540009F415C2D8011B96EC91E9A3E07859F006
:108E6400FE013696FA93EA93EBA10E947675FA9383
:108E7400EA930E94B568E9A1E07459F0FE013696C0
:108E8400FA93EA93EBA10E947D75FA93EA930E9408
:108E9400B568FE013696FA93EA930E94CB68E8A37C
:108EA400E0910D04EB8FE0910E04EA8F0E948C6E2A
:108EB400D80111962D913C91D80113964D915C9156
:108EC400D80115960E947A7BEEA3FFA3D8011796CA
:108ED400EC91F0E0ECA3FDA3D8011896EC91EC8F93
:108EE400E0910E04A0E10E94E16BEAA3FBA30E94BF
:108EF40043760E94AE750E94AE75ECA1EA930E947F
:108F0400AC4BD8011996EC91EC8FE03011F4E8E009
:108F1400EC8F0E9443760E9448765A934A930E94AB
:108F24004F760E9453760E945A760E945D760E9484
:108F340043763A932A930E945D76EEA1FFA10E94A4
:108F440064765A934A930E9448760E945D76A8A557
:108F5400A130B1F43A932A93FA0131960E945A76D9
:108F6400FA013196FA93EA930E944F76F901319609
:108F74000E946976F9013196FA93EA930E945D762C
:108F8400A8A5A230F1F40E94537631970E945A7634
:108F9400EAA5FBA5E40FF51F3197FA93EA930E9423
:108FA4004F76EEA1FFA1E20FF31F31970E9469767D
:108FB400EAA5FBA5E20FF31F3197FA93EA930E9407
:108FC4005D76E8A5E03011F40C941149D8011996A6
:108FD400EC91EC8FE0910D04ACE00E946E760E945F
:108FE400017BED8FA8A1EA1710F40C944048E1E04E
:108FF400E0930E04E03021F0ECA1FDA1B5970CF450
:1090040002C00E947476AAA1BBA1ECA1FDA1EA1B37
:10901400FB0BDF010E942B71EAA3FBA3ABA1AA23E4
:109024001AF4E0E0EAA3EBA3A8A10E942976AEA17A
:10903400BFA1F0E00E947C76EE8FA8A5A13021F4B8
:109044000E947F760E948276A8A5A23031F40E9405
:109054007F760E9464760E948E76E0E0E9A30E9407
:109064009476AE0FBF1FEC91E03039F00E949476F5
:109074000E9410760E949976F2CFD1C0E1E0E0938D
:109084000E04E03031F0ECA1FDA1E734A0E0FA07D2
:109094000CF402C00E947476E8A1EF8FEAA1FBA150
:1090A400EE0FFF1FACA1BDA1AE1BBF0BE3E0F0E0D0
:1090B4000E94017BEAA3FBA3ABA1AA2322F4E1E073
:1090C400F0E0EAA3FBA3EF8DE150EF8FEF8DF0E02A
:1090D400DE011696AE0FBF1FAC91A03219F0AF8D12
:1090E400A13008F404C0EF8DE150EF8FEFCFAF8DC6
:1090F4000E942976AE2FEEA1FFA1B0E0EA17FB078C
:1091040014F3EF8DE03011F4ED8DEF8FAF8DECE0C3
:109114000E946E760E947C76EE8FA8A5A13021F481
:109124000E947F760E948276A8A5A23031F40E9424
:109134007F760E9464760E948E76E0E0E9A30E9426
:1091440094760E94067621F0EF8DA9A1AE1708F05F
:1091540007C00E9494760E9410760E949976EFCF01
:10916400AF8DE8A1EA1BAE2FED8DEA1768F0AF8D45
:10917400E8A1EA1BACE0EA9FF001A0910D040E9473
:109184006E760E947C7601C0E0E0EE8FA8A5A13047
:10919400A1F40E947F76E20FF31F31960E94DB75E3
:1091A400AFE00E94E16BE40FF51FDF01ECA1FDA12C
:1091B4000E94427131960E943A6EA8A5A23089F4A9
:1091C4000E947F76E20FF31F0E94DB75AFE00E94DE
:1091D400E16BE40FF51FDF01ECA1FDA10E94B67461
:1091E400BEDD0E949476AE0FBF1FAC91A03219F47D
:1091F400E9A1EF5FE9A30E9494760E94067639F014
:10920400AF8DE9A1EA1BAE2FED8DEA1708F407C074
:109214000E9494760E9410760E949976ECCFD80131
:109224001C96EC91E03029F10E948C6E0E944376EA
:1092340096DDF801A485A43698F4EFE0E0931004D9
:10924400F801A485AA3028F0A485AA930E94654158
:1092540006C0D8011C96EC91E05DEA9303DD09C0D9
:10926400ECE0E0931004E2E5EA93FCDCEDE4EA933D
:10927400F9DCEB8DE0930D04EA8DE0930E040E947B
:10928400637DAA9608951A9310E0E89427F81431A0
:1092940070F40E94696EE03011F00E94706E1F5FDE
:1092A400A895E12FE37011F40E942F15F0CFEFE0A1
:1092B400E09310040E942F150C94F14D1A9310E0C2
:1092C4001431F8F40E94756EB1F0A85FBC4F0E948F
:1092D4007A7BDF01EB81FC81EA17FB0764F4F00180
:1092E400E85FFC4FDF010E947A7BDF01E981FA81AC
:1092F400AE17BF070CF002C00E94706E1F5FA895E6
:10930400DFCFEFE0E09310041881259608951A93B7
:1093140010E0143190F40E94756E31F0FD01E15FAC
:10932400FC4FE081E17009F406C01A93E0910A044D
:10933400E170EA9382DD1F5FECCF0C94F14D2C9722
:109344000E945C7DAD89BE890E942B710E94A1762A
:10935400EB8BFC8BED89FE890E94A676EB89FC8958
:10936400E017F107FCF00E94D9762E2F33270E94D4
:10937400FD760E9404770E940B770E9410770E946A
:10938400FD76F801A98DBA8D0E94106D0E940B77AD
:10939400F8010E941A77EA8DEA930E940F4C0F5F3E
:1093A4001F4FDCCF48C02C970E945C7DAD89BE89DD
:1093B400E4E0F0E00E94017B0E94A176EB8BFC8B41
:1093C400ED89FE89EE0FFF1F0E94A676EB89FC89CA
:1093D400E017F10784F10E94D976AE2FED89FE895A
:1093E400B0E0EA0FFB1F9F010E94FD760E94047704
:1093F400E98DFA8DEE0FFF1F0E941A770E941077F5
:10940400ED89FE89EE0FFF1FA98DBA8DAE1BBF0B30
:10941400BA93AA93F801A98DBA8D0E94106D0E9487
:109424000B77F8010E941A77EA8DEA930E940F4C99
:109434000F5F1F4FCBCF0E94637D6B960895EA8127
:10944400F0E0EBBBF5BBF7E1F09365001F98E6E1B4
:10945400E0936500F09365001F9AE881F981EBBB06
:10946400F5BB1F98FFE1F0936500EEE1E093650022
:10947400F09365001F9A0C94644EE2E2EBBBE0E0CB
:10948400E5BBE7E1E09365001F98E6E1E093650042
:10949400E7E1E093650008951F9A0895A0910403FD
:1094A400A23021F4E881A8E4B3E10BC0A091040345
:1094B400A43021F4E881A8E4B3E103C0E881A8E280
:1094C400B3E1F0E00E9442710E94897B21960895E5
:1094D400E0910403E23011F4EEE40AC0E43039F41C
:1094E400E0E2EA93A981BA810E94157604C0E0E221
:1094F400EA93E981FA81FA93EA930E94214A17C018
:10950400E0910403E23011F4EFE40AC0E43039F4EA
:10951400E1E2EA93A981BA810E941E7704C0E1E2E4
:10952400EA93E981FA81FA93EA930E94214A229606
:109534000895E0910403E230B9F4E4E4EA930E946C
:109544002377AE0FBF1FFD01FE2FE0E0AF81B8858A
:109554000E94106D0E94214AE5E4EA930E94397644
:109564000E94214AE6E453C0E33089F4E7E3EA9336
:10957400FF81E0E00F010E942377EA0FFB1F0E94A6
:1095840028770E9439760E94214AE6E340C0E430FD
:1095940049F5E7E3EA93AF81B8850E941576DF01C8
:1095A400EB81FC81AE1BBF0BFD01FE2FE0E00F0140
:1095B400AF81B8850E9415760E942877AD81BE815F
:1095C4000E941E77DF01E981FA81AE1BBF0BBA93BB
:1095D400AA930E94214AE6E3EA93AD81BE810E94E8
:1095E4001E771CC0E0E5EA930E9488740E94214A19
:1095F400E1E5EA930E9423770E94106D0E94214ABC
:10960400E2E5EA930E9439760E94214AE3E5EA936F
:10961400E981FA81AD81BE81EA0FFB1FFA93EA93D7
:109624000E94214A28960895E0910403E33029F426
:10963400E3E0EA93E0E1F1E00BC0E43029F4E3E095
:10964400EA93E0E2F1E004C0E3E0EA93E0E3F0E16E
:10965400FA93EA930E94214A0895E0910403E330C7
:1096640029F4E3E0EA93E1E2F1E00BC0E43029F409
:10967400E3E0EA93E1E1F1E004C0E3E0EA93E8E344
:10968400F0E1FA93EA930E94214A08951A930A9307
:10969400EFE10E943177EBE10E943177EFE10E9424
:1096A4003177E8EFFFEFE0935C0CF0935D0CE4910D
:1096B400EF3F39F0E0915C0CF0915D0C0490009266
:1096C4000403E6ECF3E18F01A0910403A23019F442
:1096D400E8EAF3E18F01A0910403A43019F4E8E669
:1096E400F3E18F01F801E491ED3F39F4F80131968B
:1096F4000E946C6D0E945B7A19C0EE3F71F4F80110
:1097040031960E94897BDF01E0910403F0E0EA17BF
:10971400FB0711F00D5F1F4F09C0F801E491EA93B4
:10972400F80131960E946C6D0E94214A0D5F1F4F13
:10973400F801E491EF3FB1F60E94FA6BE1E0E093A7
:109744000E04E0930D04E4E1E09313046DDF09914A
:10975400199108950E943577AE85AA2362F0AD85EC
:10976400BE85A03FE0E0BE0734F4AB85BC85AF33D3
:10977400E1E0BE070CF050C00E943D77AE0FBF1F62
:10978400A03FE0E0BE0734F0AD85BE850E941576AB
:10979400E987FA87EF81F885AB85BC85AE0FBF1FDB
:1097A400A034E1E0BE0734F0AB85BC850E941E778F
:1097B400EF83F8870E94776D0E94776D0E94776D22
:1097C4000E94776DB6DE0E94776D0E9442774985CC
:1097D40054DE0BBB15BB2EE13FE100E010E0EF814E
:1097E400F885E017F10764F050E0451730F0209356
:1097F4006500309365005F5FF8CF0F5F1F4FEFCFB9
:109804004BDE0E94016C0E94016C0E94226CEFE30B
:10981400F1E0FA93EA938DDEC9C00E9435770E9485
:109824003D77EA17FB0741F0EF81F885AB85BC85EE
:10983400EA17FB0709F03EC00E944A771CF00E9419
:10984400517784F42D853E85ED85FE85E987FA8779
:109854002D873E872B853C85EB85FC85EF83F88738
:109864002B873C870E94776D0E9442770E943D7748
:10987400EA17FB0749F4F1DEEB85FC85ED87FE87EB
:10988400EF81F885E987FA87F8DD0BBB15BB2EE17C
:109894003FE10D851E85E985FA85E017F1073CF067
:1098A40020936500309365000F5F1F4FF4CFF4DD04
:1098B400BBDE7CC000930B0410930C040E94587709
:1098C4000E945F77FF93EF930E9463770E945F7714
:1098D400AF91BF91EA17FB0780F10E945177B4F46E
:1098E40020E030E00E946677E217F30774F00E94EC
:1098F40058770E946D770E9466770E9472770E9463
:109904007B7758D02F5F3F4FEDCF16C020E030E07B
:109914000E946377E217F3077CF00E9458770E9455
:109924006D770E9463770E947277F9010E948277B3
:1099340041D02F5F3F4FECCF39C00E944A77DCF40F
:1099440020E030E00E948677E217F3079CF00E9443
:1099540063770E946D770E948677D0010E94017B15
:10996400AF010E947B77FA010E94827723D02F5F98
:109974003F4FE8CF1BC020E030E00E945877E21749
:10998400F307A4F00E9463770E946D770E945877D2
:10999400D0010E94017BAF01F9010E948277FA0194
:1099A4000E94827707D02F5F3F4FE7CF0E94637DED
:1099B4002F960895EA81FB81FA93EA9389DD0E9448
:1099C4008D779EDDE2E2EA93E0910B04F0910C04C2
:1099D400FA93EA930E94214A249608950E945C7D9A
:1099E40000910D0410E0E0910E041E1710F00C9489
:1099F400534DE885F985FA93EA9382DD2C853D85FC
:109A04004A855B85022E032A11F40C944B4D37FFD3
:109A140036C05A934A935CDDE2E2EBBBE0E0E5BB7F
:109A2400E7E1E09365001F98F6E1F0936500E093A9
:109A34006500EE81EBBBEF81E5BBEFE1FEE1E09376
:109A44006500F0936500E093650001FF04C0F093A6
:109A54006500E093650036FF11C0F0936500E09364
:109A6400650001FF06C0F0936500E09365004F5F59
:109A74005F4F220F331F4F5F5F4FEDCF1F9A220FAF
:109A8400331F01FF02C04F5F5F4F4F5F5F4F0C9466
:109A9400044DE885F9853196E887F9871F5F0C94B2
:109AA400F54C38C022970E945C7DE885EA930E94B9
:109AB400504AEE83FF83E985A8E1EA9FF001E85D5F
:109AC400F84F8F0130E0383028F5F801E4915E2F2B
:109AD4000F5F1F4FF801E4914E2F407F0E94927751
:109AE4000E949777EA87FB87F801E4914E2F440F91
:109AF400440F440F440F0F5F1F4FF801E4915E2F92
:109B04000F5F1F4F0E9492770E949777EA87FB8727
:109B14003F5FD9CF0E94637D2E96089524970E94BB
:109B24005C7DEA85EA930E94504AEE83FF8300E05D
:109B340010E0EB850E940B76D4F5EF85F889E88771
:109B4400F98720E030E0EC850E94A4772CF5E989C0
:109B5400FA89449155273196E98BFA8B5A934A93A3
:109B6400EA85FB85FA93EA93E989FA89FA93EA93F9
:109B7400EC85FD85FA93EA930E94F04CE0910D0484
:109B8400EE0FEE0FEE0FA885B9850E948D74E8875D
:109B9400F9872F5F3F4FD7CFE0910E04AD85BE8587
:109BA4000E948D74ED87FE870F5F1F4FC2CF0E9406
:109BB400637D639608951A93EFEF0E940672E09313
:109BC400390910E00E942871E05CF54FE081EF3F15
:109BD40031F00E9428710E94A9771F5FF3CF199179
:109BE40008951A930A930091CF0BAA81A53411F416
:109BF400E0E066C0AA81A23539F4A0913508A1300D
:109C040019F40E94AC7709F405C00E94611CE0E0DD
:109C1400E0933508AA81AB3411F0A33599F4E02F11
:109C2400E470E43011F414E001C013E0E02FE270BA
:109C3400E23009F41C5FE02FE170E13009F41F5FAA
:109C4400E12F3EC0AA81A13511F0A13799F4E02F8C
:109C5400E470E43011F417E001C016E0E02FE27084
:109C6400E23009F41C5FE02FE170E13009F41F5F7A
:109C7400E12F26C0AA81A33421F0A13411F0A2342B
:109C840041F413E0E02FE170E13009F41F5FE12FAC
:109C940017C0AA81A73741F417E0E02FE170E13043
:109CA40009F41F5FE12F0CC0AA81A03441F415E030
:109CB400E02FE170E13009F41F5FE12F01C0EFEF05
:109CC400198108812396089524970E945C7D209130
:109CD400CF0BA0914009A53411F00C94304FE0E073
:109CE400E09335080E94FF71E0E0E0935D0BE091A2
:109CF400D30BE03089F5E0911008A0911108EA1720
:109D040039F00E94B277ED55F84FE081E13009F067
:109D140023C0E7E7EA930E9497620E94B277E8556E
:109D2400F84F0E944771FA93EA930E94B877EC5572
:109D3400F84FDF010E94B3730E94B877E755F84FDC
:109D44000E94BD77E2E0E09335080E94B277ED55BA
:109D5400F84FA2E0A0832FDFE0913508E03011F046
:109D64000C94304F0E94AC7711F40C940A4F0E946B
:109D7400561CE1E0E0933508E22FE870E83081F406
:109D84000E94C277E8EEF3E00E94017BDF010E94AB
:109D9400527D14F4E1E301C0E0E3EA930E94976288
:109DA400E22FE074E03411F413E001C012E0E0911A
:109DB400240C0E9445741A930E94F462E22FE4700A
:109DC400E43049F40E94C277E0E1F7E20E94337B79
:109DD400AF0114E006C00E94C2770E943873AF013D
:109DE40013E0E22FE071E03111F4415050405A93F6
:109DF4004A931A930E94F462E22FE072E03211F463
:109E040014E001C013E0E091270CF091280C17C076
:109E140018E0E22FE470E43009F41F5FE22FE870E9
:109E2400E83009F41F5FE22FE072E03209F41F5FAB
:109E3400E22FE074E03409F41F5FE0E0F0E0FA930D
:109E4400EA931A930E94F462E22FE170E13029F45C
:109E5400E0915D0BEA930E949762ADDEA091400908
:109E6400A73729F4E2E0E0933508E03009F473C041
:109E74000E94FF710E94C7770E94B5721E2F0E9434
:109E8400D072AF01E1E0EA930E943D620E2FE091AF
:109E94001008A0911108EA1739F00E94B277ED5525
:109EA400F84FE081E23009F053C00E94B277EC55DC
:109EB400F84FDF010E947A7B4E175F0711F00C9474
:109EC400A64F0E94B277E655F84F008011800E9499
:109ED400CE6D0E948F71EA17FB0769F10E94B27779
:109EE400E655F84FDF010E947A7B0E94CD770E94ED
:109EF400B277E655F84FDF010E947A7BEC59F44FB4
:109F0400E0810E94D5770E94DC770E94516D0E9407
:109F1400DF77EFEAF8E10E94B172003029F05A933A
:109F24004A930E94CA6202C00E94E5770E94E977C0
:109F34000E94706309C0003039F00E94ED7720F46C
:109F44000E94A8730E945526E1E1F8E00E94F4778C
:109F5400E0E0E0933508A0914009A33421F40E9485
:109F64009D33E03009F40BC00E94FF710E94C77753
:109F74000E9445730E94016C63D30E94091DA09145
:109F84004009A13411F0A23421F40E94FF710E940F
:109F9400C777A0914009A03421F40E949D33E0309A
:109FA40009F420C00E94B572E887F987E2E0EA93D9
:109FB4000E943D621E2F0E94F8770E942F180E9473
:109FC400E8730E94FE77E152F84F10830E94E87311
:109FD400E652F84FA7E0A0830E94D3710E94FF715C
:109FE4000E94C777A0914009AB3439F0A33529F01A
:109FF400A13519F0A13709F076C00E949D33E030F5
:10A0040011F40C946F500E94FF710E940578E1E4F2
:10A01400F9E00E94CB72E22FE270E23029F4E4E02E
:10A02400EA930E943D6202C0E1E0F0E0E887F9872C
:10A03400A0914009A13511F0A13721F40E94D072FA
:10A044001E2F02C01091E50BE22FE470E43011F4EE
:10A05400E4E001C0E3E0EA930E943D62AF01A09115
:10A064004009A33511F0A13731F4E885F9850E9440
:10A07400757AE887F9870E94ED7720F0A091D30BD9
:10A08400A13011F51A935A934A93EB85FC85FA9300
:10A09400EA930E94281D0E945F77EE83FF83AE81BE
:10A0A400BF810E94527D84F40E94FF71E6E6EA9328
:10A0B4000E949762EE81FF813197EE83FF83AE8128
:10A0C400BF810E94527D94F31A935A934A93EB856D
:10A0D400FC850E9488726FDD06C00E9445730E9451
:10A0E400016C0E94281D0E94637D2A9608950E9497
:10A0F4000978E89422F80E94C773E2E7EA930E9481
:10A104009762E0913B08EA930E949762EFE0EA933A
:10A114000E949762A0913808AA3219F41A9365D361
:10A124001AC0A0913B080E942871EC59F44FE081B9
:10A13400EA1721F4E0913B08E03349F40E949F6C54
:10A14400AC59B44FE0913B08EC931A934ED322FCE4
:10A1540002C00E947063C0C20E940978E0913B086B
:10A16400E053AE2F0E942871EB58F44FE081EA17B8
:10A1740041F51A933AD3A0913608A23019F40E94FB
:10A18400117809F402C00E941778A0913608A33010
:10A1940019F40E94117809F402C00E941778E0E0D3
:10A1A400E0933608E093600C0E942871EB58F44F5A
:10A1B400BF01E081EF5FAE2FEAE00E94307BDB015C
:10A1C400EC938AC2E881E03019F40E94E57706C076
:10A1D400E881E8500E9445740E94CA62219608955D
:10A1E4000E945C7D25FC28C20E94117811F40C9415
:10A1F40072520E941A78E752F84F9F01D9011196C2
:10A20400EC91E43071F50E9420780E9423780E943A
:10A214002A78F901A681A03021F4A281B381109794
:10A2240009F007C0E2EBF8E10E94B1720E94E977FD
:10A2340015C00E94DC770E942E780E94DF77E5EB40
:10A24400F8E10E94B1720E9432780E943878F901D4
:10A25400A085B185BA93AA930E94CA620E943E78EF
:10A26400EBC1E730C9F40E9420780E9423780E9451
:10A274002A78E8EBF8E10E94B1720E9432780E94D9
:10A28400DF77EBEBF8E10E94B1720E942E780E9416
:10A29400CA620E943E78D0C1E93089F40E942078D5
:10A2A4000E9423780E942A78EEEBF8E10E94B172B2
:10A2B4000E9445780E94DF770E943E78BDC1E63057
:10A2C40029F5EAE2EA930E945563E1ECF8E10E9481
:10A2D400B172D901EC910E944878E091CD0B0E94B3
:10A2E4004878EBE4EA930E9497620E942E780E94D9
:10A2F400CA62E4E5EA930E9497620E9432780E945F
:10A30400CA620E9470630E94177896C1E530C9F44E
:10A314000E9499730E94CD77D901EC910E94D57760
:10A324000E94DC770E942E780E94DF77EFEAF8E142
:10A334000E94B1720E9432780E94CA620E943E78E2
:10A344007BC1E83039F50E9420780E9423780E946E
:10A354002A78E4ECF8E10E94B172F901A681AA938B
:10A364000E94A573309719F00E94B96F04C0D901F7
:10A374001696EC91F0E0FA93EA930E94CA620E9466
:10A38400E9770E947063D9011196E0E0EC930E9492
:10A39400177852C1E130C9F5A0911908A53029F404
:10A3A400E091CD0BE65F1E2F01C011E0E12F0E946A
:10A3B4004C780E9428710E9451780E9454780E941F
:10A3C400DC770E942E780E94DF77E7ECF8E10E94A8
:10A3D400B1720E9432780E943878D9011796EC91B4
:10A3E4000E9445740E94CA62A0911908A53041F4E4
:10A3F4000E945878A481B581BA93AA930E942C63D1
:10A404000E944B750E945E7817C1E330B1F40E943C
:10A414009973F0960E9469780E9499730E9451780A
:10A424000E945478EAECF8E10E94B1720E943278FA
:10A434000E946D780E945E78FFC0EB3069F50E943F
:10A4440070780E9473780E945478EDECF8E10E94D1
:10A45400B172F901A681AA93B5DE0E945878A7814A
:10A46400AA93B0DE0E945878A085B185BA93AA93C6
:10A474000E9438780E9432780E943878F901A481C9
:10A48400B581BA93AA930E9438780E9445780E94B5
:10A494006D780E945E78D0C0EC3089F40E947078A8
:10A4A4000E9473780E945478E0EDF8E10E94B17242
:10A4B4000E9445780E946D780E945E78BDC0EE309F
:10A4C40079F40E9470780E9473780E945478E3EDC6
:10A4D400F8E10E94B1720E944B750E945E78ACC094
:10A4E4000E94AC7761F0A0913608A03041F4A091AD
:10A4F400D20BA13021F40E94CE6DE13009F426C0C4
:10A50400A091850BA03059F0E091870BF091880B56
:10A51400FA93EA93E8EEF3E00E944F73B9F4E1E3AF
:10A524000E946978E091760BE05D0E94D5770E94E5
:10A53400CE6DEA930ED1E09336080E944B75E093FA
:10A544005E0CF0935F0CE0E0E093850BA09136087D
:10A55400A03059F0E0915E0CF0915F0CFA93EA930D
:10A56400E4E6F0E00E944F7309F025C0A09136089C
:10A57400A23019F40E94117809F402C00E941778DD
:10A58400A0913608A33019F40E94117809F410C080
:10A59400A091600CA33030F00E941778E0E0E093C3
:10A5A400600C06C00E941A78E652F84FA8E0A08317
:10A5B400E0E0E0933608A091860BA130E9F5E09144
:10A5C400390CA091380CEA1791F1EAE20E946978FB
:10A5D400E091740BE05D0E94D577E091390CEA9329
:10A5E4000E94BB1E0E94DC77E091290C0E944574F6
:10A5F4000E94DF77E6EDF8E10E94B1720E94B1702B
:10A60400FA93EA930E9438780E9430740E94777813
:10A614000E947063E091390CEA930E94001DE0915E
:10A62400390CEA930E94CF1CE093390C05C0E0E09A
:10A63400E093860B689420F80E94637D2696089523
:10A644001A930A930E949D33E030D9F00E94E87374
:10A65400E752F84F8F01EC81FD81D8011296ED93FA
:10A66400FC93EA81FB81D8011896ED93FC93EE816B
:10A67400D8011696EC93D8011196E4E0EC930E946D
:10A68400D3711981088127960895E091420BEA93CA
:10A694000E949762E091430BEA930E9497620895A7
:10A6A400F4DF0E948D770E947A780E947A780E9463
:10A6B400DF7799C01A930E94C9611E2F103021F0D0
:10A6C400E12FE150E093400BE0DFE091400BEF5FBE
:10A6D4000E9445740E94DF77199108950E945E7D5F
:10A6E40031E00E94817828F00E94BF72AC91A433BB
:10A6F40008F02AC030E00E94BF72EC91E270E69547
:10A704001E2F0E94BF72EC91E1700E2FA0915A0B84
:10A714001A1729F4E1E0EA27E0935A0B31E0A091FB
:10A724005B0B0A1729F0E1E0EA27E0935B0B31E0C9
:10A73400E0915B0BEE0FE05DA0915A0BEA0FEA93F8
:10A744000E9497620E94B873E32F0E94657D24964D
:10A7540008951A9310E00E94AC7711F40C94F1530D
:10A764000E94561CEAEDF8E10E94B172E091240CBB
:10A774000E9445740E94DF77EDEDF8E10E94B1720A
:10A78400E091270CF091280C0E9477780E94C27700
:10A79400A031E7E2BE074CF4E0EEF8E10E94B172AA
:10A7A400E091250CF091260C13C0E3EEF8E10E9431
:10A7B400B172E9810E94CE6F0E94C277EA0FFB1F3B
:10A7C4000E946F70E091250CF091260CE051F74245
:10A7D400FA93EA930E94CA620E94E97711E00E9408
:10A7E4008578E12F18812296089524970E945C7D34
:10A7F4000E9485780E947261E13010F40C94CB566B
:10A80400E091420BEB3441F4E091430BE33219F451
:10A814000E94C9611E2FBAC2E435A9F4E091430B2A
:10A82400E33221F40E94C961EE83FF83E091430B7C
:10A83400EF3441F40E94C9611E2F1A930E94887458
:10A844000E942F18A3C2E23411F00C946A55E091CF
:10A85400430BE13251F4AA85AF3F29F40E944573BA
:10A864000E94016CEDDE0E94091DE091430BE1346E
:10A87400E1F40E94C9611E2F113071F4A0913608D1
:10A88400A13019F40E94AC7709F402C00E94611C43
:10A89400E0E0E093850B09C0E1E0E093850B0E94C2
:10A8A4000968E093870BF093880BE091430BE53440
:10A8B400A9F4E6EEF8E10E94B1720E943E1CF397FF
:10A8C4003CF00E94C9610E946F700E948C7801C0A4
:10A8D400E0E3EA930E9497620E94E977E091430BD8
:10A8E400E634D9F40E94987819F40E94C961AF0142
:10A8F400E885F9850E94BE6F0E2F003420F0A091E8
:10A90400D30BA13021F40E94A4780E94281DAA85AB
:10A91400AF3F19F40E94A47893DEE091430BE23533
:10A9240011F00C9427550E94987819F40E94C9617B
:10A93400AF0130E0A091D30BA03021F40E94CE6D82
:10A94400E13009F027C00E94A333E03011F10E94E6
:10A954007C72EC55F84FA885B985A083B1830E9419
:10A964007C72E655F84FDF01EA850E94CF710E94A0
:10A974007C72E855F84F10830E947C72E755F84FBB
:10A9840040830E947C72ED55F84FA1E0A0830E94A1
:10A99400827259C00E949D33E23010F40C94255504
:10A9A4000E94F8770E94351E3E2F3F3F29F00E94F7
:10A9B4008470A417B5070CF412C00E943074E41B11
:10A9C400F50B0E9492700E94597219F4E0E0E09332
:10A9D400290C3A930E94C21E689420F803C0E0E058
:10A9E400E887E9870E94E873E752F84FDF01EA85B8
:10A9F400F0E0EC59F44FE081EC930E94E8730E947C
:10AA0400FE77EF51F84FDF01EA850E94CF710E9473
:10AA1400E873E152F84F10830E94E873E652F84F4E
:10AA2400A5E0A0830E94D371E885F985309759F099
:10AA34000E94F877FA010E94757A0E9488720E9437
:10AA4400A4780E94B01C689422F8E091430BE3358B
:10AA5400F1F50E94C961E887F9870E941A78DF013D
:10AA6400E652F84FE081E23081F4FD01EF51F84FF6
:10AA7400008011800E94CE6D0E948F71EA17FB073F
:10AA840021F4A0913608A23009F01FC00E941A7860
:10AA9400E552F84FDF010E947A7BDF01E885F985F2
:10AAA400EA17FB0779F40E941A78DF01ED51F84F99
:10AAB400E081EA93FD01E752F84FE081EA930E94B6
:10AAC400552603C0E7E0E0932406689422F85EC1AB
:10AAD400E43411F00C94D355E091430BE33559F46D
:10AAE400E9EEF8E10E94B1720E94675E0E94487824
:10AAF400E1E0E0933909E091430BE03511F00C9467
:10AB0400D2550E94A878E03011F40C94D25520E07C
:10AB14000E94AC7840F00E94BF72AC91A23219F04E
:10AB24000E94B07809F43CC0E22FE03061F40E9446
:10AB3400BF72AC91A33211F421E004C00E94B47836
:10AB44000E94425E2AC0E13051F40E94BF72AC916F
:10AB5400A43211F422E001C020E010E01EC0E23073
:10AB640011F0E330D1F40E94B4780E94E167EF3F22
:10AB740099F0E12FE295E07FEF930E94B4780E9470
:10AB8400E167AF91EA0F1E2F2F5F243021F41A934F
:10AB94000E94425E20E001C020E00E94B873B8CF5A
:10ABA400F5C0E33411F00C943B56E091430BE534CB
:10ABB400B9F4E6EEF8E10E94B1720E943E1CF397EC
:10ABC4004CF00E94C961E05FF84D0E946F700E94D2
:10ABD4008C7801C0E0E3EA930E9497620E94E977CF
:10ABE400E091430BE634A9F441E050E00E94C961CE
:10ABF4000E2F0E94B878E13019F40E94C961AF01A8
:10AC04001A930E94846CE05FF84D0E9469760E945A
:10AC1400281DE091430BE33591F40E94BC780E9417
:10AC2400B46FE83131F4E091890BEA930E94DE17A6
:10AC340006C0E885EA93EFEFEA930E945526E09177
:10AC4400430BE134A9F4ECEEF8E10E94B1720E94E6
:10AC5400BC78EA930E94DD180E949425E03011F03C
:10AC6400E1E301C0E0E3EA930E9497620E94E9777E
:10AC74008DC0E63511F00C94A056E091430BE334FB
:10AC840011F00C949F560E94C9611E2F113010F4CC
:10AC94000C949F56A0911908A13091F50E94B878A0
:10ACA400E03021F0A091A2061A1709F028C0115033
:10ACB4000E94C961AF011A930E9429213E2F0E946C
:10ACC400FF720E9442710F010E94FF720E94BC6DCC
:10ACD4000E94C3780E94B878E03071F00E94C96184
:10ACE400AF010E9413730E9442710F010E941373FB
:10ACF4000E94BC6D0E94C3781A930E94BE111DC0AD
:10AD04001630D8F41150A12FEAE00E94E07AA3E2B1
:10AD1400EA9FF001E855F94FBF01A12FEAE00E9434
:10AD2400307BF0E0BB01AAE0B0E00E94AE7ADB0128
:10AD3400AE0FBF1F14960E94D97028C0E93431F5B4
:10AD4400E091430BE03551F40E94C9611E2FE0E00D
:10AD5400EA931A930E94B018E0932E06E091430BF5
:10AD6400EC34A1F40E948D61E09328060E94B87827
:10AD7400E03021F00E948D61E09329060E94B878AA
:10AD8400E03021F00E948D61E0932A060E942E613A
:10AD940031CD0E94637D2B960895A091580BA03568
:10ADA40021F4A091590BA03408F005C0E091590B8F
:10ADB400EA930E94FD18A091580BA33521F4A091A9
:10ADC400590BAA3008F005C0E091590BEA930E9490
:10ADD4002819A091580BAB3421F4A091590BA03839
:10ADE40008F005C0E091590BEA930E946619A091FE
:10ADF400580BA63521F4A091590BA03108F005C0D9
:10AE0400E091590BEA930E949419A091580BA43530
:10AE140011F40E9419189CD60895E3EAF6E0FA9317
:10AE2400EA93E091420BEA93E0E8F0E00E94EB6FD2
:10AE340008950E94CB78A0E0A083E091400BE093BA
:10AE4400590BE091420BE093580B08950E945C7DEE
:10AE54000E947261E13010F40C94225AE091580B74
:10AE6400A091420BEA1709F098DFE091420BE3321C
:10AE740039F5E091430BEC3431F4CFDFE4E0E093B7
:10AE840018080E94D178E091430BE435C1F4C5DF82
:10AE9400E091630CE03029F0EF77A9E0B0E00E9484
:10AEA400BC7BE091640CE03029F0EF77AAE0B0E0DD
:10AEB4000E94BC7B0E94D178E7E0E093180802C0AE
:10AEC400EB34E1F5E091430BE13211F4A6DF35C038
:10AED400E53211F462DF31C0E33299F40E94D7788D
:10AEE40021F00E94E2780E9432190E94CB78E0811E
:10AEF400EB3429F4E0E0E093340CE093350C99DF73
:10AF04001CC0E134D1F40E94C9619F012093340C28
:10AF14000E94E87891F00E94C9619F01A091340CCD
:10AF2400F901E270F070EA2BE093340C0E94E878A7
:10AF340021F00E94C961E093350C7FC2E33581F5AD
:10AF4400E091430BE13211F468DF29C0E33299F454
:10AF54000E94D77821F00E94E2780E940C190E9486
:10AF6400CB78E081E33529F4E091400BEA930E9429
:10AF7400511B5FDF14C0EE3491F40E94687410E03A
:10AF84001A3068F4A3EBBBE0EE27A10FBE1F0E94AA
:10AF94002871EC5BF44FE081EC931F5FF1CF4DC25D
:10AFA400E63511F00C941E58E091430BE13211F494
:10AFB40034DF41C0E33299F40E94D77821F00E9433
:10AFC400E2780E9474190E94CB78E081E63529F476
:10AFD400E091400BEA930E94A7192BDF2CC0E635C1
:10AFE40031F40E94C9619F012093300C24C0E534E0
:10AFF40071F40E94C9619F0120932F0C0E94E8788C
:10B0040029F00E94C9619F012093320C14C0E435D9
:10B0140091F440E050E00E94C9619F01022E032A8E
:10B0240011F042E050E00E94E87819F00E94C961F2
:10B03400AF014093310C01C2E43511F00C94D8589F
:10B04400E091430BE33231F40E94C9613197E093FC
:10B05400400BABC0E03511F00C94D75810E00E94BF
:10B06400AC7850F00E94BF72AC91AD3329F00E94CD
:10B07400B07811F01E3008F005C00E9428710E94BB
:10B08400EE78EDCF0E9428710E94F778EDE30E94DC
:10B09400FC7811F00C94D758E4E5E093580B10E0D9
:10B0A4000E944D703496E491EF3F11F40C94D758FC
:10B0B4000E946C740E944D700E946C6D0E94A36883
:10B0C400E03011F00C94D5580E944D703496E49100
:10B0D400E03851F40E94C961E058FF4FE093630CDB
:10B0E400E0E8E093640C5FC0E23839F40E94C9617F
:10B0F400E058FF4FE093640C56C0E13839F40E94E5
:10B10400C961A8E0B0E00E94BC7B4DC0E03011F002
:10B11400E13051F40E944370FF93EF930E94C961A0
:10B12400AF91BF91EC933FC0E23059F40E94437059
:10B13400FF93EF930E94C961AF91BF91ED93FC938C
:10B1440032C0E33051F40E944370FF93EF930E94A6
:10B15400A861AF91BF91EC9326C0E43021F50E9421
:10B164004D703596E491EA930E9477620E94437091
:10B17400E093610CF093620C00E00E944D703596F0
:10B18400E4910E1780F40E94846CEC5BF44FE08130
:10B19400A091610CB091620CEC93A1E6BCE00E941A
:10B1A400636E0F5FEACF1F5F7BCF47C1E03511F0BD
:10B1B4000C941F5AE091430BE33299F40E94D77820
:10B1C40021F00E94E2780E94DD180E94CB78E08191
:10B1D400E03529F4E091400BEA930E94661B29DED6
:10B1E4002CC1E13211F419DE28C1E134D1F40E94FA
:10B1F400C9611E2F00E00D3098F40E949174EA0F8B
:10B20400FB1F3396E491E11749F40E9491740E9464
:10B214009574A0919A0BEA2BE0939A0B0F5FEBCFF6
:10B224000CC1E63559F5E0E0E093410BADE9BBE034
:10B234000E940179FF93EF930E94C961AF91BF917E
:10B24400EC93EBE2EA930E943E61E03059F0A0EA0D
:10B25400BBE00E940179FF93EF930E94C961AF9113
:10B26400BF91EC930E940479A091410BA33018F490
:10B274000E94E87809F401C0D9CFDFC0ED34D1F4DD
:10B28400E0E0E093410BA9EABBE00E940179FF935F
:10B29400EF930E94C961AF91BF91EC930E9404792E
:10B2A400A091410BA33018F40E94E87809F401C07E
:10B2B400EACFC3C0E735D1F4E0E0E093410BA0EB63
:10B2C400BBE00E940179FF93EF930E94C961AF91A3
:10B2D400BF91EC930E940479A091410BA23018F421
:10B2E4000E94E87809F401C0EACFA7C0E434C9F5A4
:10B2F400E0E0E093410B0E94C9619F01E2E0EA9320
:10B304000E944B61AF01E3E70E94FC7859F40E946C
:10B314000A79BF01D9010E94CA71E40FF51FDB014C
:10B32400ED93FC93E9E40E94FC7879F40E940A7995
:10B3340020833183AAE9BBE00E9401790F010E94B6
:10B344001179EC91E160D001EC930E940479A09111
:10B35400410BA33018F40E94E87809F401C0CBCF64
:10B364006CC0EE3499F40E94687410E01A3068F4EA
:10B37400AAE8BBE0EE27A10FBE1F0E942871EC5B78
:10B38400F44FE081EC931F5FF1CF57C0E33449F4ED
:10B394000E94A8780E94C961E093950BF093960BE4
:10B3A4004CC0E33589F40E94C9619F010024021650
:10B3B400030624F42B30E0E03E070CF004C0F9014E
:10B3C4003197E093970B39C0E53529F40E94C961A0
:10B3D400E093990B32C0EF3491F40E94C9611E2F9F
:10B3E400ECE2EA930E943E61E12FE295E07FEF9365
:10B3F4000E94C961AF91EA0FE093980B1EC0E0353B
:10B40400E1F4E0E0E093410BACEABBE00E94177981
:10B414000E944271FF93EF930E945762AF91BF91D4
:10B42400ED93FC930E940479A091410BA23018F48F
:10B434000E94E87809F401C0E7CF0E942E6108CD8C
:10B44400E0E0E093430A0E94637D269608950E94FB
:10B454005E7D0E947261E13010F40C94DB5CE0913B
:10B46400420BE332A9F4E091430BE03519F4EFEE1B
:10B47400F8E109C0E83419F4E0E1F9E104C0E33586
:10B4840031F4EBE2F9E1FA93EA930E94A8628EC2E6
:10B49400E43511F00C94E65AE091430BE43229F4BC
:10B4A400E8E2F0E00E941B798EC0E33211F402D985
:10B4B4008AC0E03511F00C94E55AE7D8A091400B0E
:10B4C400A83210F00C94E55A0E941F790E946C6D0A
:10B4D4000E94A862EDE3EA930E9497620E941F799A
:10B4E4003496E491E03839F40E94CE6D0E9445749C
:10B4F4000E94CA6268C0E23839F40E943E700E9419
:10B5040045740E94CA625FC0E13839F40E944074F5
:10B514000E9445740E94CA6256C0E03011F0E130C6
:10B5240051F40E941F7932960E94897B0E944771D0
:10B534000E94237948C0E23059F40E941F79329660
:10B544000E94897BDF010E94B3730E94CA623BC0E0
:10B55400E33051F40E941F7932960E94897BE08186
:10B56400EA930E94D8622FC0E43069F50E941F79E3
:10B5740032960E94897BE093610CF093620C10E098
:10B584000E941F793596E4911E1790F40E94287149
:10B59400EC5BF44F0F01A091610CB091620CEC9143
:10B5A400D001EC93A1E6BCE00E94636E1F5FE8CF7C
:10B5B4000E941F793596E491F0E00E94F7780E948A
:10B5C4006C740E942163F2C1E33579F5E091400B7C
:10B5D400EA930E940C19E091430BE43229F4EAE067
:10B5E400F0E00E941B7920C0E33211F463D81CC040
:10B5F400EE34D1F44AD810E01A3068F40E9428716D
:10B60400EC5BF44F0F01A3EBBBE00E945475D00137
:10B61400EC931F5FF1CFE0E0E0934E0B0E946C745B
:10B624000E9421630E94E977C1C1E635D9F5E09112
:10B63400400BEA930E947419E091430BE43229F41D
:10B64400E5E0F0E00E941B792CC0E33211F432D81B
:10B6540028C0E53451F419D8E0912F0C0E944574A8
:10B664000E942779E091320C19C0E63529F40E9432
:10B674004753E091300C12C0E43599F40E944753CB
:10B68400E091310CE03011F0E1E301C0E0E3EA9332
:10B694000E9497620E942D79E091310CF0E00E94A3
:10B6A400777884C1E03511F00C94A55CE091400BEF
:10B6B400EA930E94DD18E091430BE43229F4E0E4BC
:10B6C400F0E00E941B793EC1E33219F40E945C53FE
:10B6D40039C1E13411F00C94B15B0E94475312E07C
:10B6E400A0919A0BECEDEA233E2F00E00D3078F4A4
:10B6F4000E9491740E949574E31739F40E94917426
:10B70400EA0FFB1F3396149102C00F5FEFCF0E9424
:10B71400516D0E94DF77E091980BE03089F0E6E408
:10B72400F9E10E94B1720E94306D0E9445740E943A
:10B734002779E091980BEF700E9445740E94DF779F
:10B74400E091990BE03051F0E9E4F9E10E94B17223
:10B75400E091990B0E9445740E94DF77F3C0E434B2
:10B7640079F50E943179A091410BA33040F5E09125
:10B77400410BE03011F00E942D790E941179EC9177
:10B78400E17061F4A3EABBE00E9417790E94BC6DEA
:10B794000E94B3730E942C63E3E70BC0A3EABBE0EF
:10B7A4000E9417790E94BC6D0E94B3730E94CA6202
:10B7B400E9E4EA930E9497620E940479D4CFBEC060
:10B7C400ED34C9F40E943179A091410BA33090F477
:10B7D400E091410BE03011F00E942D79A9EABBE021
:10B7E4000E943779EC910E9445740E94CA620E94BB
:10B7F4000479EACFA3C0E735C9F40E943179A09156
:10B80400410BA23090F4E091410BE03011F00E9422
:10B814002D79A0EBBBE00E943779EC910E9445742E
:10B824000E94CA620E940479EACF88C0E63531F5E5
:10B834000E943179A091410BA330F8F4E091410BBF
:10B84400E03011F00E942D79ADE9BBE00E94377918
:10B85400EC910E9445740E94CA62EBE2EA930E9452
:10B864009762A0EABBE00E943779EC910E9445748C
:10B874000E94CA620E940479DDCF60C0EE34D1F424
:10B884000E94475310E01A3068F40E942871EC5B60
:10B89400F44F0F01AAE8BBE00E945475D001EC9369
:10B8A4001F5FF1CFE0E0E0934E0B0E946C740E94A6
:10B8B400216344C0E33499F40E9447530E946C749A
:10B8C400E1E5F9E1FA93EA930E94B96F0E94CC731F
:10B8D4000E944F750E946C740E9421632FC0E03552
:10B8E400A9F40E944753E091AC0BF091AD0BFA938D
:10B8F400EA930E9444630E942D79E091AE0BF0918B
:10B90400AF0BFA93EA930E94446318C0E33531F411
:10B914000E944753E091970BEF5F0DC0EF3491F411
:10B924000E9447530E94306D0E9445740E942779FB
:10B93400E091980BEF70F0E00E942379EBE3EA9337
:10B944000E94976233C0EB3489F5E091400BEA938F
:10B954000E943219E091430BE43229F4E0E8F0E06C
:10B964000E941B7923C0E33219F40E945C531EC069
:10B97400E134E1F40E944753A091340CE1E0EA235E
:10B984000E9445740E942779A091340CE3E0EA23D5
:10B994000E9445740E942779E091350C0E944574F9
:10B9A4000E94CA62E4E5F9E10E94B1720E942E612C
:10B9B40050CD0E9485780E94657D249608951A933F
:10B9C4000E94FF71E0E4F9E00E94CB720E94857846
:10B9D4000E943B79E181E43471F40E943B79028056
:10B9E4000E94CE6DE05DE01529F00E943B79E28172
:10B9F400EA3209F401C057C00E9440790E943B79A1
:10BA0400E1810E9444790E943B79E2810E94447959
:10BA14000E94BF721C910E943B7933960E94CB72A4
:10BA2400E12FE23131F40E944A79E6E0EC930EDA38
:10BA34003AC0E13131F40E944A79E2E1EC9307DD46
:10BA440032C0EF30A9F40E944A79EEE0EC930E94F0
:10BA54007053E13039F4A0913508A03019F00E94F8
:10BA6400AC7709F402C00E94611C0E9450791BC08B
:10BA7400EE30C9F40E944A79EFE0EC930E947053CF
:10BA8400E13089F4A0913508A03019F00E94AC7718
:10BA940009F402C00E94611CE0E0E0933508EFEF76
:10BAA400EA930E94F75363C21A930E94C7730E94D9
:10BAB4001B70EAE7EA930E9497620E94BF72119793
:10BAC4001C91E12FE23131F4E6E0EA930E9497629F
:10BAD400BDD937C0E13131F4E2E1EA930E949762C3
:10BAE400B6DC2FC0EF3099F40E9454780E94705352
:10BAF400E13039F4A0913508A03019F00E94AC77F8
:10BB040009F402C00E94611C0E9450791AC0EE30F0
:10BB1400C1F4EFE0EA930E9497620E947053E1300F
:10BB240081F4A0913508A03019F00E94AC7709F493
:10BB340002C00E94611CE0E0E0933508EA930E9491
:10BB4400F753A0913808AA3211F00E9470630FC213
:10BB5400EFEFE093580BE093590B0895AC81A033B9
:10BB640010F0AA3308F006C00E945779E0530E94EF
:10BB74005F7999C4AC81A13410F0A73408F006C0F1
:10BB84000E945779E7530E945F798DC4A881B981D7
:10BB9400E0E0EC9388C4AA93EA93FA93EFB7EA93AC
:10BBA4001A930A931BB10CB1E0919D0CF0E0E55996
:10BBB400F34F0083A0919D0CAF5FA0939D0CA23323
:10BBC40019F4E0E0E0939D0C09911991F3C21A93E2
:10BBD400E0919E0CA0919D0CEA17D1F3F0E0E55999
:10BBE400F34F1081A0919E0CAF5FA0939E0CA233E3
:10BBF40019F4E0E0E0939E0CB9C1A0919D0CAE5CF9
:10BC0400E0919E0CAE1BE2E30E94307B08950A9201
:10BC14001A92FA926A937A938A939A93AA93BA930A
:10BC2400EA93FA93EFB7EA930E94647949F0A091FA
:10BC34003909A03021F00E94F50CE13009F401C06B
:10BC440011C0E091040DF0E0E156F34FE081ECB94E
:10BC5400A091040DAF5FA093040DA43619F4E0E0A5
:10BC6400E093040DE991EFBFF991E991B991A9919C
:10BC74009991899179916991F99019900990189500
:10BC84001A930E94647959F45D9B09C0A091390903
:10BC9400A13021F40E94F50CE03009F013C010919A
:10BCA400030D0E942871E156F34FA981A0831F5F01
:10BCB400143609F410E0E091040DE117E1F3109358
:10BCC400030D02C0E981ECB9A1C20E94647921F498
:10BCD4000E94F50CE13009F001C019C350C10E9463
:10BCE4005E7D8BDFE03011F40C946F5F70DF1E2FEC
:10BCF400A091680CA53618F0E0E0E0933A09309181
:10BD04003A09E0913A09E03011F00C94D65EA09122
:10BD1400E40BA13021F0A091E40BA23031F4E12F27
:10BD2400EF77E0934009EBE4CEC01A3521F4E1E06B
:10BD3400E0933A09CAC0123049F4E4E1E0933A09C5
:10BD4400E0E0E0933B09E0933D09BFC0A091E40B20
:10BD5400A33069F4173729F01A3310F4103308F4B8
:10BD640002C0E7E001C0E0E0E0933C0905C01A939B
:10BD74000E94F34DE0933C09A0913C09AF3F99F038
:10BD840010934009E1E0E0933B0910933D09E091F1
:10BD94003C09E03011F4E5E404C0EAE0E0933A0938
:10BDA400E0E0E0933F0991C0E13069F4103039F4E8
:10BDB400E2E0E0933A09E0E0E0933F0903C0E0E009
:10BDC400E0933A0982C0E23059F410933C0910938D
:10BDD4003D09E0E0E0933B09E3E0E0933A0975C0F4
:10BDE400E330F1F40E946A790E947079EA0F0E94AC
:10BDF4007A79A9F4E0913D09E03071F4E4E0E0934C
:10BE04003A09E0913B090E94616F0E9483790E9484
:10BE14006A79A0E0A08303C0E0E0E0933A0955C04A
:10BE2400E43049F41D3019F4EAE5E0933F09E0E019
:10BE3400E0933A094AC0EA3079F40E946A790E9490
:10BE44007079EA270E947A7931F4E0E0E0933A09C4
:10BE5400E5E4E0933F0939C0E431B9F40E946A791A
:10BE64001083E12FA0913D09EA27E0933D09E09179
:10BE74003B09EF5FE0933B09E0E0E093670C13308C
:10BE840019F4E5E1E0933A0920C0E53111F0E63117
:10BE940059F41A93E7E6FCE0FA93EA93EAE3F9E04B
:10BEA400FA93EA935BDE11C0E73179F4E0E0E093C2
:10BEB4003A09173131F4E091670CA0913D09EA1772
:10BEC40009F003C0E3E4E0933F09A0913A093A176B
:10BED40019F0E0E0E093680C04CF0E94657D44C44F
:10BEE400AA93BA93EA93FA93EFB7EA931A930A934D
:10BEF40010919B0000919C00E12FEC71A9F4E0915A
:10BF0400CD0DF091CE0DEB5FF24F0083ADECBDE0B3
:10BF14000E94636EE83CA0E0FA0731F4E0E0F0E050
:10BF2400E093CD0DF093CE0D09911991E991EFBFF6
:10BF3400F991E991B991A99118951A930E94887978
:10BF44000E948D79D9F30E948879EB5FF24F1081BA
:10BF5400AFECBDE00E94636EE83CA0E0FA0731F468
:10BF6400E0E0F0E0E093CF0DF093D00DE12F1991D4
:10BF740008950E9488790E948D7909F0C8C1E0E093
:10BF840008950E945E7DF5DFE03021F0A091660CFB
:10BF9400A03009F0E5C0D1DF1E2FA091D90DA53640
:10BFA40018F0E0E0E093D30D3091D30DE091D30D80
:10BFB400E03059F4113019F4E4E0E093D30D1A356C
:10BFC40019F4EAE0E093D30DC3C0E430C1F4E0E037
:10BFD400E093D30D1A3229F00E94CE6DE05DE11793
:10BFE40069F4109338081093D40DE5E0E093D30D71
:10BFF400E0E0E093660CE1E0E093D60DA9C0E53003
:10C00400A9F4E0E0E093D30D0E94CE6DE05DE1176A
:10C0140061F00E9494790E949D79E091D60DEF5FC2
:10C02400E093D60DE6E0E093D30D92C0E63091F4B0
:10C03400E091D60D0E949D790E949479EF5FE09380
:10C04400D60DE0E0E093D70D133019F4E7E0E09368
:10C05400D30D7EC0E73011F0E83059F41A93E7EDC0
:10C06400FDE0FA93EA93E3EDFDE0FA93EA9376DDDB
:10C074006FC0E93081F4E0E0E093D30D173131F47F
:10C08400E091D70DA091D40DEA1709F003C0E4E5BF
:10C09400E093660C5DC0EA3041F4103011F4EBE03B
:10C0A40001C0E0E0E093D30D53C0EB3071F4E0E065
:10C0B400E093D60D1093D50D1093D40DECE0E093DE
:10C0C400D30DE0E0E093660C43C0EC30A1F5E091C1
:10C0D400D60DF0E0E05CF64F10830E949479EF5F98
:10C0E400E093D60DE091D50DE150E093D50DA091EC
:10C0F400D50DA03021F4A091D40DA03009F00EC0CC
:10C10400EDE0E093D30DE091D60D0E94616F0E94A3
:10C114008379E091D60DF0E00E948379A091D50D4A
:10C12400A03021F4A091D40DA03009F403C0E0E0C4
:10C13400E093D30D0DC0ED3059F4E0E0E093D30D5E
:10C144001D3031F4EAE5E093660CEFEFE093650C03
:10C15400E091D30DE31719F0E0E0E093D90D13CF8C
:10C164000E94657D01C3AA93EA93FA93EFB7EA9319
:10C17400E091DB0EA091DA0EEA1791F0E091370816
:10C18400E03019F0E89426F80AC00E94A279F0E0A1
:10C19400E030A1E0FA0719F4E0E0E093DB0E03C01D
:10C1A400E89425F826F8E091650CE03019F0E0E019
:10C1B400E093D30DE991EFBFF991E991A991189515
:10C1C4001A93E091DB0EA091DA0EEA1721F4E091C4
:10C1D4009B00E072C1F4E091DA0EF0E0E652F24F17
:10C1E400A981A0831091DA0E1F5F0E949F6CA0307A
:10C1F400E1E0BE0709F410E0E091DB0EE117E1F3A2
:10C204001093DA0E03C0E981E0939C001881229612
:10C214000895E0E0E093DB0EA091DA0EA13020F067
:10C224000E94A279689426F80895AA93BA93EA938F
:10C23400EFB7EA93E091650CE03041F4E0E0E0937D
:10C24400DB0E0E94CE6DEF5FE0933708E991EFBFFC
:10C25400E991B991A99118950E94AC7818F00E94BF
:10C26400B07809F403C00E94B873F6CF0E94B07886
:10C2740011F40E94B87308950E94BF72AC91E881D2
:10C28400EA1729F40E94B8733197E1E05DC1E0E058
:10C294005BC10E945E7D00E010E0EEE20E94FC784B
:10C2A400E9F420E030E0EC810E94A477BCF4D801EA
:10C2B4000E947B748F010E94817818F00E94B079EB
:10C2C40008F009C00E94BF72EC910E943D730E0FEA
:10C2D4001F1F0E94B8732F5F3F4FE5CFF801E1C0E5
:10C2E4000E94AC7828F00E943B79E181E03208F4A6
:10C2F40010C00E94BF72EC91E093420B0E94B8738D
:10C304000E94BF72EC91E093430B0E94B873E1E08A
:10C3140008950C9443660E94FA750E94B4780E94B2
:10C32400E167EF3F89F0F8010E94897AFF93EF9368
:10C334000E94B4780E94E167AF91BF910E948D740E
:10C344008F010E94B873E9CFF8011EC01A930A93B3
:10C3540010E00E94BF720C910B3311F0003208F40C
:10C3640012C0013310F0093308F007C0E02F0E9417
:10C374003D73E255FF4FE4911E2B0E94B8730E9457
:10C38400BF720C91E9CFE12F0991199108950E9490
:10C394005E7D00E010E00E94BF72AC91AD3221F4EA
:10C3A4000E94B87331E001C030E00E94817818F037
:10C3B4000E94B07908F009C0D8010E947B740E94E1
:10C3C400B4798F010E94B873F0CF303021F4F801B2
:10C3D4000E94657DC9C1F8010E94757A0E94657D3D
:10C3E400C3C124971A93E0E0E983EA83EB83EC83E7
:10C3F4000E94BF72AC91AD3221F40E94B87311E077
:10C4040001C010E00E94817818F00E94B07908F011
:10C4140022C0A981BA818B819C81EAE0F0E060E0CE
:10C4240070E00E94DB7A7F936F93FF93EF930E94F7
:10C43400BF72EC91E053AF91BF918F919F91FF2711
:10C44400662777270E946B7AE983FA836B837C8360
:10C454000E94B873D7CF103031F4E981FA816B812F
:10C464007C81188120C0E981FA816B817C810E94E2
:10C47400797A188118C00E945E7D20E030E000E0E7
:10C4840010E0EC810E940B765CF4D9010E947B746D
:10C494000E94B4799F010E94B8730F5F1F4FF1CFC0
:10C4A400F9010E94657D259608950E945E7D6FDFE7
:10C4B4008F0120E030E0EEE20E94FC7811F467DFA7
:10C4C4009F01112322F4F9010E94757A9F01A09122
:10C4D4001B0CA13030F0D8010E94CA71E20FF31F87
:10C4E4008F01F8010E94657D3FC11A9310E00E94FC
:10C4F400A878E030A1F00E94AC7858F00E94BF7296
:10C50400AC91A23231F00E94B07819F0E9811E1783
:10C5140008F005C00E9428710E94EE78ECCF0E94BA
:10C5240028710E94F7780C949F66E8810E944479F0
:10C53400E881A0915C0BEA0FE0935C0BE881A09189
:10C544005D0BEA27E0935D0B219608951A9310E0A2
:10C55400E12FA981BA810E948D74E491E03049F001
:10C56400E12FA981BA810E948D74E4910E94BA7965
:10C57400EFCF0BC01A9310E00E94F775E03029F05A
:10C584000E94F7750E94BA79F7CF1881239608950F
:10C5940064970E9411750E94BF79E88DF98D0E94FD
:10C5A400CC730E944175E6DF669608951A93ECE316
:10C5B400EA93BBDF11E0193080F40E942871E25540
:10C5C400FF4FE491A981EA2319F0E12FE05D01C056
:10C5D400E0E2EA93AADF1F5FEECFEEE3EA93A5DF82
:10C5E4000C949F6664971A930E94C4790E94BF7941
:10C5F400EA8DFB8D0E94CC730E944F750E94C47912
:10C604000E94CB681E2FED891E1720F40E94E57747
:10C614001F5FF9CF0E94C479ADDF18810EC0649703
:10C624000E9411750E94BF79E88DF98D6A8D7B8D0A
:10C634000E9419740E9411759DDF68960895E2E2C4
:10C64400EA9373DF0E948D7795DFE2E2EA936DDF70
:10C654000C94A066A881B981E4E6F0E00E94017B15
:10C664000E942379EEE2EA9360DFA881B981E4E6CF
:10C67400F0E00E94337BFA93EA93E2E0EA93B2DFBC
:10C684000C94A066A0911B0CA13020F00E948D7721
:10C69400E1DF07C00E948D777BDFE2E6F9E10E94CB
:10C6A400B1720C94A06625FE06C0E5E0F0E00E949D
:10C6B4003E6EA895F8CFEAEDFDE0E0935E0BF093B3
:10C6C4005F0BE1E00E940672E0935C0B0E94C97963
:10C6D4000E94CE6D0E9448780C940C691A930A93B8
:10C6E400E091650CE03011F00C941268E3E0EA93F9
:10C6F4001CDFE0915C0BE295EF70EA930E94F8670F
:10C704001E2FE0915C0BEF70EA930E94F8670E2FE6
:10C714001A930BDF0A9309DFE7E1EA9306DFEAEDF8
:10C72400FDE0A0915E0BB0915F0B0E949D7BEA1B24
:10C73400E093DA0E689425F80C941268EE81EA937B
:10C74400B2DFEC81FD810E94B1720E94CD7967DF76
:10C75400C5DF0C943369EB81EA93A5DF0E94237152
:10C76400F5DE0E94C979BADF24960895ED81EA9333
:10C774009ADFEB81FC810E94B172EA81EA93D5DEF3
:10C78400E981E03011F0EA93D0DEE881E03011F085
:10C794000E94C979A3DF269608950E945C7D10E06B
:10C7A400E6E6F9E1A885B985EA17FB0719F444E13F
:10C7B40050E002C048EC50E0EA85E0933809E89480
:10C7C40031F8EA93E985FA85FA93EA93EA85EA93DC
:10C7D400EA85EA93E0E0EA93C9DF0E9409689F01D1
:10C7E4000E9438150E9443760E9415680E2F31FC72
:10C7F40002C0003009F001C0F3CF31FE04C0E89458
:10C8040031F8E1E004C01F5F1230B0F2E0E00E94B2
:10C81400637D2B9608951A930A93E091400AE030C1
:10C8240011F40C941268E0E0E0933909E2E0EA9331
:10C8340027DA10E003E00E9428710E94D47961F0A5
:10C844000E9428710E94A9770E942871E05CF54F2C
:10C85400E0810E271F5FEFCFE3E0EA9311DAE02FC8
:10C86400E295EF700E94D979E02FEF700E94D97998
:10C87400E7E1EA9305DA0C9412681A930A93E091BB
:10C88400400AE03011F40C9412680E943E70E030CB
:10C8940021F0E091420AEA3209F405C00E943E7098
:10C8A400E05DE093420AE0E0E0933909EAE5EA93C7
:10C8B400E7D9E0E0EA93E4D910E00E9428710E94ED
:10C8C400D47911F01F5FF9CF1F5F012F0A93D8D9D4
:10C8D40010E00E9428710E94D47961F00E942871AE
:10C8E4000E94A9770E942871E05CF54FE0810E0F49
:10C8F4001F5FEFCFE02FE195EA93C2D9EDE0EA9311
:10C90400BFD90C9412681A930A93F894E0E0E09368
:10C914003708E091DB0EE093DA0E7894E091400A58
:10C92400E03011F40C941268EAE5EA9349DCE0E0A3
:10C93400EA9346DC10E00E9428710E94D47911F039
:10C944001F5FF9CF1F5F012F0A933ADC10E00E94AA
:10C9540028710E94D47979F00E942871E05CF54F27
:10C96400E081EA932DDC0E942871E05CF54FE081C0
:10C974000E0F1F5FECCFE02FE195EA9321DCEDE091
:10C98400EA931EDC0C941268E881EA938CDEEAE5F3
:10C99400EA93CBDDE0914009EA93C7DD0E94BF72C0
:10C9A400EC91E03031F00E94B478BFDD0E94B8739E
:10C9B400F5CF94DE0C940C691A930E94FF71E091F8
:10C9C4003B08EA93B2DDE4E4EA93AFDDE091390891
:10C9D400EA93ABDD14E00E942871E85CF74FE08134
:10C9E400E43040F00E942871E85CF74FE0810E9437
:10C9F400BA79F1CFE0E0EA9398DD3FDF3DC11A93C5
:10CA04000A936DD9E0913F09E03011F40C947E65EE
:10CA1400A0913F09AA3541F4A0913B09A33020F02D
:10CA2400E0914109E43409F04BC00E943E70E030CB
:10CA340021F0E0914209EA32C1F40E94CE6DE05D3A
:10CA4400A0914209EA1721F0E0914209EA3221F467
:10CA54000E94E15C12DF08C0E3E4F9E00E94CB72BB
:10CA6400E09142090E94DF792BC00E943E70E05D94
:10CA7400A0914209EA1721F50E94CE6D1E2FE09184
:10CA84004309ED3421F4E0914409E33209F007C08D
:10CA9400E5E4F9E00E94CB727ADC1E2FDDDB0E9414
:10CAA400CE6DE11729F0E12FE05D0E94DF7908C027
:10CAB4000E94CE6DE05DE09342090E94E15CDDDE00
:10CAC400A0913F09A53449F4A091E40BA33019F4D3
:10CAD4000E94DC2A02C00E94664EA0913F09A33442
:10CAE40011F40E94942AA0913F09AB3411F40E94DE
:10CAF4008F2AE0E0E0933F09A091E40BA33011F406
:10CB04000E94DC2AE0E00C9412683BDAA091660CE7
:10CB1400A43529F4A0E025FCA1E0A03009F03AC036
:10CB2400E0913A08E03581F4E0913B08EA93E6E0CD
:10CB3400EA930E94E842A0913B08A03820F0E091DB
:10CB44003B08E093650523C0E03721F4E0E0E0937F
:10CB540065051DC0EA3519F40E94565D18C0EA3710
:10CB640011F42ADF14C0E23519F40E9479500FC081
:10CB7400E23719F40E94AE500AC00E946030E0917E
:10CB84003908A0913809EA1711F4689431F8E0E003
:10CB9400E093660CA091660CAA3531F40E94E15C26
:10CBA400B2DEE0E0E093660C6CC0A091690CA130A9
:10CBB40050F0E091690CE150E093690CE03019F415
:10CBC400E1E0E0936A0CA0E025FCA1E0A13049F487
:10CBD400A0E026FCA1E0A03021F4A0913708A03009
:10CBE40009F001C016DBE0913708E03019F0E1509C
:10CBF400E09337080895E091D90DEF5FE093D90DE4
:10CC0400E091680CEF5FE093680CE091650CE03014
:10CC140019F0E150E093650C0895A091E40BA13064
:10CC240021F0A091E40BA23029F4E3E0E09390001A
:10CC3400E8E3E9B90895E0E00E94C16BE1B3E36081
:10CC4400E1BB85E38A95F1F7E1B3EC7FE1BBE4E472
:10CC5400E09374000E94D86B08951A9314EAE4EAEE
:10CC64000E94E67941F40E94EB79183011F01031FA
:10CC740011F4E0E001C0E2E019910895E4E9E093E1
:10CC84007400E0E008951A93E981E1600E94F0796C
:10CC940031F40E94EB79103411F4E0E04EC04CC042
:10CCA4001A93E9810E94F07931F40E94EB791831EA
:10CCB40011F4E0E042C040C01A93E9810E94F07987
:10CCC40031F40E94EB79183211F4E0E036C034C03C
:10CCD4001A93E981E03011F0E4EC01C0E4E80E9429
:10CCE400E67979F40E94EB79E0917300AA81BB8123
:10CCF400EC93103511F0183521F4E0E018810C9410
:10CD0400896BE1E018810C94896B1A93E981E093B3
:10CD1400740010E0E0917400E07811F4163908F022
:10CD240005C08BE18A95F1F71F5FF4CFE0917400A1
:10CD3400E07811F0E0E001C0E1E018812296089566
:10CD44000E945E7D3D810C8120E087DFE03011F59B
:10CD5400EE810E94EE6EF1F43A93AEDFE030D1F44E
:10CD64000E94F479B9F479DFE030A1F4EE810E94F5
:10CD7400CF6B81F4EDB7FEB7FA93EA931F930E9449
:10CD8400D46B1F91E03031F479DFE12F0E94657D8F
:10CD94000C94336950DFD9CF0E945E7D30E00E8160
:10CDA4001D815BDFE03099F4EF810E94EE6E79F42F
:10CDB4000E94F47961F41A937FDFE03041F4EC814E
:10CDC400EA937ADFE03019F459DFE0E002C033DFA0
:10CDD400E8CF0E94657D2896089522970E945C7D85
:10CDE40050E02B853A85A89538DFE03011F00C949B
:10CDF4005167EE850E94EE6E11F00C9451672A93F0
:10CE04005BDFE03011F00C9451673A9355DFE0306A
:10CE140011F00C94516721DFE03011F00C9451674C
:10CE2400EE850E94CF6BD9F5E0E0EE83EF83EC85CD
:10CE3400FD8531970E94CB7549F4EDB7FEB7FA939F
:10CE4400EA931F930E94D46B1F9109C0EDB7FEB7FC
:10CE5400FA93EA931F93E1E0EA933ADF1F910E2FCE
:10CE6400EE81FF81A885B985EA0FFB1F1083EE814F
:10CE7400FF813196EE83FF83003039F4EC85FD8524
:10CE8400AE81BF81AE17BF0708F001C0D0CFEC85DB
:10CE9400FD850E94CB7519F4F1DEE0E002C0CBDE23
:10CEA400A3CF0E94637D2F96089568970E945C7DAE
:10CEB40020E0E0E0EC8FED8F31E0A895E9A1FAA144
:10CEC400662777270E94337CEA87FB876C877D87F8
:10CED400EE8D0E94F979EE83FF8368877987AA85AE
:10CEE400BB858C859D850E94097DEA8BFB8B6C8BB1
:10CEF4007D8B0E948D7BFE017296FA93EA930E94C9
:10CF04008B6BEE8BFF8B688F798F0E94FF790E9469
:10CF1400FA7BAF010E94FF79AE8DBB278827992742
:10CF24000E94947B0E94127ADE015A960E94FA7B38
:10CF3400ED93FC930AA119A190DEE030D1F5EDA1A7
:10CF44000E94EE6EB1F50E94F47999F51A93B4DE5D
:10CF5400E03079F5303051F14F5F5F4FEC8DFD8D4E
:10CF64003196EC8FFD8FAC8DBD8D1197EBA1FCA19B
:10CF7400EA17FB0711F430E018C0EC8DFD8D3197F2
:10CF8400AF8DB8A10E94107697DEEE8DDA01F0E045
:10CF9400EA17FB0751F472DEEA8DFB8DA9A1BAA151
:10CFA400EA0FFB1FE9A3FAA389CFD4CF67DEE0E041
:10CFB40002C041DEC1CF0E94637DA6960895A88178
:10CFC400A03310F0AA3308F004C0E881E0530C94B5
:10CFD4000C69A881A13410F0A73408F004C0E881DA
:10CFE400E7530C940C69EFEF0C940C69A881AA30F8
:10CFF40020F4E881E05D0C940C69A881AA3020F04B
:10D00400E881E95C0C940C69E8E50C940C691A93CA
:10D014000A93F8940091620B1091630B7894F801D1
:10D024000991199108951A930A93F1DF8F01EA8106
:10D03400FB81AC81BD81EA0FFB1FE01BF10BDF011B
:10D044000E94527D2CF4E0E0198108810C94B76BA6
:10D05400E1E0198108810C94B76BECE9F4E1FA93EF
:10D06400EA93EAEBF0E0FA93EA93E5E0F0E0FA936E
:10D07400EA93E4E0EA93E6E2EA93EEE0EA930E94BC
:10D08400904DE4E3F5E1FA93EA93EAEAF0E00E94D2
:10D09400177AE8E0EA93E0E2EA93E1E0EA930E9497
:10D0A400904DE4E3F6E1FA93EA93E2EDF0E00E94B6
:10D0B4003D6CFA93EA93E2E0EA93E2E1EA93E1E079
:10D0C400EA930E94904D0E94016C0E944F6EEFEA19
:10D0D400F0E00E94177AE3E0EA930E94AC4BEAE0A6
:10D0E400F0E0FA93EA93E4E3F0E00E943A6EE0E0C1
:10D0F400E0931004EAE6F9E10E94686DEFE0E09342
:10D1040010040895089599818881009641F0BD81A5
:10D11400AC81FB81EA8105900D920197E1F7FD81D5
:10D12400EC810C94B76BB981A881109631F0FC8125
:10D13400EB816A8161931197E9F7EB81FC81259674
:10D144000895E991F991A991B9911D90059001145F
:10D1540021F40020D1F7EE2708951018E1F3E1E05F
:10D1640008F4E2500895E991F991A991B991CD019A
:10D1740061916D936623E1F7FC010895E991F991BA
:10D18400A991B991CD0105900D920020E1F7FC0120
:10D194000895A991B991EE27FF276D91662311F0A7
:10D1A4003196FBCF0895AA27BB27E991F991059001
:10D1B400002011F01196FBCFFD0108957991E991BA
:10D1C400F991A991B991CD01772351F07A956191A3
:10D1D4006D936623C9F7772319F07A956D93FBCF86
:10D1E400FC0108956991E991F991A991B991CD0151
:10D1F400662351F06A9505900D920020C9F76623C5
:10D2040019F06A950D92FBCFFC0108955D9BFECF4A
:10D21400E881ECB9219608951A930A93AC81BD81F3
:10D224000E947A7B3097C1F0AA81BB810E947A7BED
:10D234008F01309749F00230E0E01E0760F0F801FA
:10D2440031978F01ED93FC93AC81BD810E94636E95
:10D254003197AE81A08303C0EE81EA93D7DF1981B1
:10D264000881279608952C970E945C7D10E0E88D34
:10D27400F98D3196E88FF98F3197E4912E2FE030B4
:10D2840011F40C94F36AE12FE03039F4253211F4EF
:10D2940011E002C00E941E7AA3C1E130C1F425321C
:10D2A40019F40E941E7A9BC112E0E0E0E98B00E0D1
:10D2B4002D3211F401E094C12B3219F4EBE2E98B25
:10D2C4008FC1203219F4E0E2E98B8AC102C0E23056
:10D2D40039F450E013E0203311F4006881C102C036
:10D2E400E330A1F4203310F02A3308F009C0A52F4D
:10D2F400EAE0EA9FF0015E2FE22FE0535E0F70C177
:10D3040040E02E3211F414E06BC110C0E430A1F4FB
:10D31400203310F02A3308F009C0A42FEAE0EA9F72
:10D32400F0014E2FE22FE0534E0F5AC12C3619F460
:10D33400026015E055C104C0E53011F00C94F26AA6
:10D34400E22FE33649F40E94297AEE89FF89A48109
:10D35400AA930E942F7A43C1E33741F40E94297AA9
:10D364000E94397A0E94CB681E2F0AC0E037A1F4CC
:10D374000E94297A0E94397A0E94D5681E2F08607B
:10D384000F77403011F0411708F001C0142F40E02E
:10D39400E0E0E88B30E076C0E43611F0E93611F4D1
:10D3A400046002C0E537A1F4EAE0E88B01FF08C09D
:10D3B400E0E0FAEC6AE97BE30E941D6E1AE023C008
:10D3C400E0E1F7E260E070E00E941D6E15E01BC032
:10D3D400E83511F4086004C0E83711F00C94F16AE0
:10D3E400E0E1E88B01FF08C0E0E0F0E060E070E11C
:10D3F4000E941D6E18E007C0E0E0F0E160E070E01C
:10D404000E941D6E14E0403011F00F7701C041E01E
:10D4140001FF08C00E94297AAE89BF8914960E9430
:10D424007E7B13C002FF08C00E94297AAE89BF899F
:10D4340014960E94C16D09C00E94297AAE89BF89E1
:10D4440014960E947A7B66277727EC87FD876E8780
:10D454007F8702FF16C0AF85AA2362F4EC85FD85A1
:10D464006E857F850E94797AEC87FD876E877F873A
:10D47400EDE2E98BE989E03019F01F5F4F5F01C0ED
:10D484000B7F342F00FD14C0151710F4351708F066
:10D494000FC007FF08C002FF04C00B7F2989115089
:10D4A40001C020E301C020E20E941E7A5150ECCF5B
:10D4B4001417B0F4006102FF0AC00B7FE989EA93F4
:10D4C4000E942F7A503009F0515011504150E0E33E
:10D4D400EA930E942F7A503009F051504150E8CF1E
:10D4E400312FE889E030D1F43030B9F003FF08C0BF
:10D4F400EE81FF813196EE83FF833197E49105C07D
:10D50400AE81BF81ED91AE83BF83EA930E942F7AEF
:10D51400503009F051503150E7CF57C00E94417A42
:10D524000E94067B2E2F2A3030F003FF02C0295CB4
:10D5340001C0295A01C0205D04FD25C0213360F4D7
:10D54400A885B9858A859B85A130E0E0BE07E0E027
:10D554008E07E0E09E0709F40BC0431740F453170D
:10D5640010F000FF01C014C020E207FF0CC020E34C
:10D57400006102FF08C00B7FE989EA930E942F7AB9
:10D58400503009F051500E941E7A503009F0515029
:10D5940031500E94417A0E94417BEC87FD876E875F
:10D5A4007F87E889A885B9858A859B85FF276627B3
:10D5B40077270E94067B0E941D6EE885F9856A859F
:10D5C4007B850E944E7D09F0A9CF00FF08C0503032
:10D5D40031F05150E0E2EA930E942F7AF8CF10E044
:10D5E40046CE0E94637D6A960895FF92F82E229794
:10D5F4001A930A93DE010E94677A8D01DE01169662
:10D604000E94677A0E947A7BEA83FB83DE01149688
:10D614000E94677A0E94B3731A930A93FE013696A6
:10D624000E94426C20DEAA81BB81E0E0EC93198168
:10D6340008812496FF900895A991B991EE270024BA
:10D6440060E8E894162E169407941E2A1EF0A0157E
:10D65400B10518F0A019B109E62BB7FBAA0FBB1F3F
:10D66400669580F708957B816A81F981E88177FB6B
:10D67400770F67FD7160972F9E5781F078F098318E
:10D6840090F4AA27BB27882708948795B795A79570
:10D694009A95D1F7EA23FB23682305C0E8947727FA
:10D6A400EE27FF2766276F77769508F4606877F989
:10D6B400A991B99189919991EA17FB0768077907AC
:10D6C40097FB08950E94CD790E944A7A19F40E942A
:10D6D400517A1DC0E6F7A881B9818A819B81E0E077
:10D6E400F0E060E87FE30E94127A11C00E94CD79D5
:10D6F4000E944A7A19F40E94517A09C0E6F30E9402
:10D70400517AA0E0B0E080E89FE30E946D7C24960B
:10D7140008950E94567A0E944E7D39F4A881B981F9
:10D724000E94EF6F0E94847B20C0AA81BB818C8100
:10D734009D810E94567D34F40E94567A0E948D7B0E
:10D74400C1DF05C00E94567A0E948D7BCFDFA8817D
:10D75400B9810E94847BA881B9810E947E7BAA81C1
:10D76400BB818C819D810E94127A26960895E9914D
:10D77400F99130971AF4E095F09531960895E09375
:10D784007100E0E0E0937400E2B3E360E2BB08956B
:10D7940088EC90E00197F1F70895EA930E944566BA
:10D7A400E0300895E0E0EA930C946A6680E991E041
:10D7B4000197F1F708951A930A930C94BD46EA9FD2
:10D7C400F001F0E00895FA93EA93A02FB0E00895F1
:10D7D400ECE3F0E00E94D67A0895ECE3F0E0FA93EB
:10D7E400EA930895EAE3F3E0FA93EA930C949943F5
:10D7F400E0E0E0930F04EFE0E09310040895E0E02C
:10D80400F0E0FA93EA930895FA93EA93E8E2F0E0F9
:10D81400FA93EA93E0E0EA930C94AC4BE091590557
:10D82400F0915A05FA93EA930895E0915B05F0911B
:10D834005C05FA93EA930895FA93EA930C941643D9
:10D84400EFEEF0E0FA93EA930895FA93EA93E0E0B6
:10D85400EA930C94AC4BFA93EA930C949943E12F1A
:10D86400A0E4B2E0F0E00E948D7AEA0FFB1F089575
:10D87400A12FB0E0ADCFFA93EA93E2E3F0E008958C
:10D88400FA93EA93BCCFE0911004E0930F04089557
:10D894000E948C0D0C944549E32FF0E0E05BFD4FB2
:10D8A400E4910895EA930E94A20DFE013696FA933C
:10D8B400EA930895FF27662777270E948D7B84E0EB
:10D8C4000E94F76A28960895FE017196FA93EA93E6
:10D8D4000C94B9430E945E7D0C94BD46E8E0F0E0F0
:10D8E400FA93EA930895E4E0F0E0FA93EA93089552
:10D8F400FA93EA93E8E3F0E0FA93EA9308950E9436
:10D90400897BBECFE02FF0E00895A0913A0CB0914E
:10D914003B0CBD01A3E0B0E00E94AE7AE60FF71F16
:10D92400E491E0300895E091C005EE0FEE0FEF5F53
:10D934003E2F0895E32FF0E00895A12FB0E008955D
:10D94400A0913A0CB0913B0CBD01A3E0B0E00E9461
:10D95400AE7AE60FF71F08950E948B7AE05AFD4FC6
:10D964000895FA93EA93E22FF0E008950E945C7D13
:10D97400A09119080895E091C20BF0E00895AFE377
:10D98400B1E00E94017B089530911E08E1E0E0932C
:10D994000D04E2E0E0930E043A930E94DD18E09156
:10D9A400980BE295EF70E0930F04E091980BEF7001
:10D9B400E09310040895FA93EA93E52FF0E0FA93C4
:10D9C400EA930895E7E3F0E0FA93EA930895E22FE7
:10D9D400E450F0E0FA93EA930895FA93EA93F7CFC8
:10D9E400E32FE058EA930BCFEAE8FBE0FA93EA93DB
:10D9F4000C94B9433A930E94DD18A0918A0BAD327E
:10DA04000895E091980BE295EF70E0930F04E09194
:10DA1400980BEF700895E52FF0E00895EA0FFB1FCF
:10DA2400FA93EA930895EF5EFC4FBF01E081E0585A
:10DA3400DB01EC930895E0E0EC93AE81BF8108959F
:10DA4400E3E0F0E0FA93EA930895E52FE450F0E080
:10DA5400FA93EA930895E550F0E00895E091980B65
:10DA6400E295EF700895EA1BA2E5B7E0F0E00E94AA
:10DA74008D7A0895F0E0EE0FFF1FEA5CFD4F0895E4
:10DA8400A4E3B2E0F0E0EE0FFF1FEA0FFB1F0895DE
:10DA9400FA93EA93E12FF0E0FA93EA930895E12FE1
:10DAA400F0E0FA93EA930895E2E0F0E0FA93EA935F
:10DAB4000895EAE8FBE0FA93EA93EAE0EA930C9427
:10DAC4006046E1E0F0E0FA93EA930895FA93EA936A
:10DAD4000C944B460E94897BFA93EA930895ABE039
:10DAE400EA9FF001E252FA4F0895ED85FE85FA931C
:10DAF400EA9308951A930A933ECF1A930A93E0E0A7
:10DB0400EA930E94AC4BDDCFE1E0E0933C0C0E9431
:10DB14000968E0933D0CF0933E0C0895BD01AAE022
:10DB2400B0E00E94AE7AE60FF71F0895FA93EA93E5
:10DB3400EAE0EA930C946046E1E0E0930E045FCEE1
:10DB44000E9496460C947946E0E2EA930C9434469B
:10DB5400A3E2B7E0E881F0E0EE0FFF1FAE0FBF1FB6
:10DB64000E947A7B0895FA93EA930C944F41E881DA
:10DB7400F0E00895EE0FFF1FAE0FBF1F08950E943F
:10DB84007A7B0E94987A08950E948D7B0C94304190
:10DB9400FA93EA930C949646A9E0B0E00E94A87B1D
:10DBA4000895A7E11A9FF001EF5CF94FE081089511
:10DBB400E12FEF5FEA930C946541F0E0D4CFE8E005
:10DBC400F0E05ECEEA93E6E0EA930E941B4186CE43
:10DBD400E0916D05F0916E050895E0916905F0916D
:10DBE4006A050895AE0FBF1FE3E0F0E00E94017BD9
:10DBF4000895FA93EA931A930A930C94C512FA932C
:10DC0400EA933A932A930C94C512A0917105B091AA
:10DC140072050895A0917305B09174050895A0E06C
:10DC2400B0E00E94A47B08950E949D7BEA1BFB0B3D
:10DC34000E94987A0895E887F9876A877B87089510
:10DC4400A885B9858A859B85EFEEF0E060E070E0F9
:10DC540008950E94987A0E942B7B0895A4E0B0E076
:10DC64000E94A47B0895EC83FD836E837F830895D3
:10DC7400FA93EA930C94B146FA93EA930C945B7A80
:10DC8400A9E01A9FF001E058FC4F089537960E94CE
:10DC9400897BDF010E947A7B0895E2E3F0E0FA9346
:10DCA400EA9308950A921A92FA926A937A938A935B
:10DCB4009A93AA93BA93EA93FA93EFB7EA931A93CF
:10DCC4000895ED91FD913196FE93EE930895ADE0A4
:10DCD4001A9FF001EB5FFC4FE08108951A93E1E095
:10DCE400EA930C941F47ADE01A9FF001DF01EB5F4C
:10DCF400FC4FE081E0300895E2E0EA930C941F4782
:10DD0400FA93EA93E4E6F0E0FA93EA930E94156842
:10DD1400E0300895E1E0E0930D04E0930E040895EB
:10DD2400E0912908F0912A0860912B0870912C0841
:10DD34000895E0912108E150A3EAB6E0F0E00E94E2
:10DD44008D7AAE0FBF1F0E947E7B0895E12FEF5F97
:10DD5400F0E01ECFE0912208EA93E0911E08EA93D6
:10DD64000E94F31AA0911E0CB0911F0C10970895F5
:10DD7400A091200CB091210C8091220C9091230C45
:10DD84000E94567D0895E0911E0CF0911F0C089599
:10DD9400E091200CF091210C6091220C7091230CE5
:10DDA4000895E2E3F0E068CF1A93E0EAEA93EA81A7
:10DDB400F0E0E054F14FFA93EA930E94A2661E2F1A
:10DDC4000895E0EAEA93EA81F0E0E054F14FFA932F
:10DDD400EA931A930C94CE66EA930E945266E0305A
:10DDE4000895E0EAEA93EEE5F0E0FA93EA93E0E0DE
:10DDF400FFE0FA93EA93EEEBFBE00895FA93EA93DB
:10DE0400E0E2EA930C945767E0EAEA93E981FA8145
:10DE1400E050FE4EFA93EA930895EA81F0E0A8E216
:10DE2400B0E00E94D67A0895E0EAEA933DCEFA93F0
:10DE3400EA930C94EF66FA93EA930C94A266E0EAF0
:10DE4400EA93E8E2F0E0FA93EA931A930A93EAE891
:10DE5400FBE00895EAE8FBE0FA93EA930895EDE223
:10DE6400EA93EAE0F0E0FA93EA930E949568E0E02E
:10DE74000895EA81F0E0ABE0B0E00E94D67AE05089
:10DE8400F24F8F01AA81AA300895E0EAEA93EBE009
:10DE9400F0E0FA93EA931A930A93E2EBFBE0089515
:10DEA400E3EBFBE0FA93EA930895EA81F0E0EE0FE6
:10DEB400FF1FE050F04F8F01AA81A0380895E15070
:10DEC400F0E00895EA81F0E00E948D7AE058F14F85
:10DED4008F01AA81A5300895EFE2FCE0FA93EA935A
:10DEE400E0E0EA9300CDECE1FCE0FA93EA93E0E0B1
:10DEF400EA93F4CC0E948D7A0E94897ADF01EA8544
:10DF0400F0E0AE0FBF1FE8E0F0E00E94D67AE050E8
:10DF1400FA4E8F01E0EAEA93E1CC1A930A93ECE11A
:10DF2400FCE085CFAE81BF81888599850E946B7A9C
:10DF3400EE83FF8368877987089540931E0C50937E
:10DF44001F0CEE81FF8168857985E093200CF093A6
:10DF5400210C6093220C7093230C0895F0E0AE0F13
:10DF6400BF1F0895EA930E94DD180C94AD1FE09141
:10DF7400950BF091960B0895FA93EA930C947C1800
:10DF8400ED81EA93ED81EA930895E091AC0BF09171
:10DF9400AD0B0E94987A0895F0E0A4E6B0E00E94E8
:10DFA400D67A0895EC81F0E0EA0FFB1F0895E09122
:10DFB4002708F09128080895E093270CF093280C83
:10DFC4000C94441CE3EAF6E0FA93EA93E0E0EA9363
:10DFD4000895FA93EA930C949568E0E0F0E060E029
:10DFE40070E00895E0932908F0932A0860932B08C1
:10DFF40070932C080895E091970BA3EAB6E0F0E043
:10E004000E948D7A0895AE0FBF1F0E947E7B0895F3
:10E01400ED5EF94FE081E1300895FA93EA93E091DF
:10E024002208E05DEA930895EA930E94CF63E13009
:10E034000895ECE3F8E0E093600BF093610B08952E
:10E04400E12FA3EAB6E0F0E00E948D7A08950E94E1
:10E054008568A881AF5FEAE00E94E07AE05D0895F8
:10E06400A881AF5FEAE00E94307BE05D0895FA93F7
:10E07400EA93E0E0EA930895AAE0B0E00E94A87B66
:10E084000895E12FF0E00E948B7AE854FF4F329616
:10E094000E94897B0895E12FF0E00E948B7AE85476
:10E0A400FF4F08953696E491D901EC930895E0EA80
:10E0B400EA93E5E0F0E0FA93EA930895EA930E9484
:10E0C400351CFA93EA93E4E2FCE00895FA93EA93A8
:10E0D400EFEFEA93E5E0F0E07CCFE093250CF093DA
:10E0E400260C08950E949D7BEA1BFB0B0895A091CA
:10E0F4002A0CB0912B0C0895E0E0E093380CE093E7
:10E10400390C0895A0912C0CB0912D0C0895E09138
:10E114002C0CF0912D0CAC81BD81EA0FFB1F0895EE
:10E12400E0932C0CF0932D0C08951A930E94CF1CAD
:10E134001E2F0895E0932A0CF0932B0C0895FA9364
:10E14400EA930E941568E0300895ABE01A9FF0014D
:10E15400E452FA4F08951A930E94BB1ED3CFE09164
:10E164002A0CF0912B0C0895EA930E94BB1E0E9486
:10E17400581EE0300895EB81EA930E94F61CFA934E
:10E18400EA93E9E2FCE00895E0E0E0934D0CE093CB
:10E194004C0C08951A930A93E0911208ABE0EA9F9D
:10E1A400F001E752F84F8F01D80111960895E0E08D
:10E1B400F0E0ED93FC930895EA81D801EC93E2E159
:10E1C400F8E0FA93EA930E94913319810881089543
:10E1D400E12FACE8B0E0F0E0EE0FFF1FEA0FFB1F09
:10E1E4000E94897B0895ACE8B0E0F0E0EE0FFF1FD9
:10E1F400EA0FFB1F0E94897B0895A0911608B09135
:10E204001708EA2BFB2BE0931608F09317080895E0
:10E21400E150A7E1EA9FF0010895A7E10A9FF00108
:10E22400E15DF94FAF010895A3E21A9FF001ED55A6
:10E23400F94F0895EC93EC81E150ADE0EA9FF001D1
:10E244000895E981FA81FA93EA930895E12FF0E0C1
:10E254000895E2E0F0E00E94017B0895AAE9BBE0A2
:10E26400E0911A080895ADE9BBE0E0911A0876CE72
:10E27400A0EABBE0E0911A0871CEA3E2B7E0CBCBF1
:10E28400EE0FFF1FEA0FFB1F0895E081F0E00895F1
:10E29400A7E11A9FF001E15DF94FEE83FF83AE81A0
:10E2A400BF810895EE81FF81A481AA930C94F41F89
:10E2B4000D901C90AE81BF811296EC91F0E0E00DC0
:10E2C400F11DDB01ED93FC930895ED91FD913197E0
:10E2D400FE93EE9308950E948A210E2EAA85BB8593
:10E2E400EC91E0150895A3E20A9FF001E855F94F77
:10E2F4000895E0911208ABE0EA9FF001E752F84F6D
:10E30400EC87FD87AC85BD85119608951296EC9136
:10E31400AC85BD851696EC930895D001F0E0089580
:10E32400A885B98518960E947A7B0895AC85BD8529
:10E33400EC93E2E1F8E0FA93EA930C949133E885E4
:10E34400F985A281AA9308950A930E94E41FE030FC
:10E354000895AA85BB85EC91EA93E3E0EA930C94D3
:10E36400E842AA85BB85E0E0EC93E2E0E093240672
:10E374000895BF0100801180AE81BF811296EC9197
:10E384000895DB01ED93FC93AE81BF81129653CBCC
:10E39400E4E6F0E00E94D67A0895F0E0ED93FC9371
:10E3A4000895E2E1F8E0FA93EA930C949133E09152
:10E3B4001908A0911808EA170895F0E0E00DF11D7E
:10E3C4000895A3EABBE042CFADE9BBE0EE27A10F7D
:10E3D400BE1FEC910895A0EABBE0EE27A10FBE1F7B
:10E3E400EC910895BD01AAE0B0E00E94AE7ADB0191
:10E3F4000895E081EA930C94425EE0E4FAE0E0934D
:10E404005E0BF0935F0B0895EA930E949762E0E03D
:10E414000895EA930E9497620C940D64ADE9BBE001
:10E42400EE27A00FBE1FEC910895A0EABBE0EE27F3
:10E43400A00FBE1FEC910895AAE9BBE0EE27A00F40
:10E44400BE1FEC91E1700895A3EABBE05BCAA0EBA8
:10E45400BBE0EE27A00FBE1FEC910895A9EABBE034
:10E46400EE27A00FBE1FEC910895ADE0EA9FF001E6
:10E47400E15FFC4F0895ADE0EA9FF001EB5FFC4FD4
:10E484000895ABE00A9FF001E452FA4F0895ABE01F
:10E494000A9FF001EE51FA4F0895FA93EA930C940F
:10E4A4001C35FA93EA930E945A433A9325CCE0919F
:10E4B4002C0CF0912D0C30970895AFEFBFEFA08393
:10E4C400B18308950E940968E093520CF093530CB1
:10E4D4000895FA93EA93E0E0F0E80895E0911208D1
:10E4E400ABE0EA9FF001E752F84FFA93EA930E94F7
:10E4F400F02857CFE0911008ABE0EA9FF0010895AF
:10E50400E0E1F8E0FA93EA930C949133FA93EA93F6
:10E514000C942253E88DABE0EA9FF0010895FA933E
:10E52400EA93F0C9E0E1EA93E0912506EA930E94B8
:10E53400B0181E2F08953BDDFA93EA930895FA93D9
:10E54400EA930C94861EE0932506E0E0E0934F0CDA
:10E55400E1E3E093500C0E942F2A0C940D26FA93C9
:10E56400EA930C94A862E1E4F9E0E093600BF09381
:10E57400610BE3E0EA930C943D62A091600BB091CF
:10E58400610B08950E940968E093470CF093480CCE
:10E594000895E093600BF093610B0895E3E0EA9330
:10E5A4000C943D62E0932708F093280808950E9494
:10E5B400BD46E0E0EA930C949F0EE0E0F0E0E093C7
:10E5C4002508F0932608E2E0E0930E040895E09114
:10E5D400130441CAE0912508F0912608C4CAE091C9
:10E5E4005D05F0915E0531970895FA93EA930C94D2
:10E5F4008F45EF5CEA930C943446A3EEB6E09AC9D7
:10E60400A3EABBE0E0911A08F0E03ACE0E947A7BDC
:10E61400D001ED93FC9322CEF0E0EA0FFB1F0F0133
:10E624001DCEA3E2B7E086C9E7E0E0931808EA93B9
:10E63400E0E0EA93E4C8EA930E94C4400E94FB42EB
:10E644001E2F0895EAE2EA93E5E7F7E110CD0E9470
:10E65400DB2BE1E0EA930C94C32B1F771A930C9401
:10E66400DD18A0912508B09126080895E8EEF3E09E
:10E674000E94337B0895E053F0E00895A0E024FC69
:10E68400A1E0A0300895E0E0EA93B9C8E09133082E
:10E69400F0913408FA93EA930895FA93EA930E9466
:10E6A4001568E13008950E940968E0933308F093F7
:10E6B40034080895E0E0E0934C0C0895D2DFEA17A3
:10E6C400FB070895E0931808E0E0E093300808950C
:10E6D4000E94AD630E94442DE093240808950E9493
:10E6E400DD180C94BD46E0911908EA93E0E0EA9342
:10E6F4000E94EE2C0C94A2280E94FB421E2F1A9317
:10E704000E94742D103808951A93E091C605EA9377
:10E714000895E091890BEA930E94E817E030089588
:10E724000E940968E093540CF093550C0895D901A4
:10E7340018960E947A7B0895E4E6F0E060E070E0C9
:10E744000E942B7B08950E94DD1811CC0A93E0915E
:10E75400C605EA930895E0912F08EA930A930C946E
:10E76400121A0E947A7BFA93EA930895A0E6BBE01A
:10E77400A8CAE0913C08E053E09322080895FA9374
:10E78400EA93E0E3EA930C94AD63E0913908EA93E9
:10E794000C9455630E94987A0E948D7B08950E9480
:10E7A4001163EBE3EA930C949762E89423F8E0E0B6
:10E7B400F0E0F8DE0A93E1E0EA930C94EE2C0A937D
:10E7C400E1E0EA930E94EE2CE1E00895E091120862
:10E7D400ABE0EA9FF0010895A881B981EC91EF5F65
:10E7E400EC930895ABE00A9FF001E352FA4F0895C9
:10E7F400A083ABE00A9FF0010895ABE00A9FF0010B
:10E80400E152FA4F0895E5EAF7E1FA93EA93EA85CB
:10E81400ABE0EA9FF0010895AC81BD81EE27A00F23
:10E82400BE1F0895E02FAC81BD81F0E008950E94E1
:10E834008D7B84E00E94F76A28960895EE27A30F43
:10E84400BE1FEC91D001EC930895A2E5B7E072C825
:10E854000E948D7AEA0FFB1FAF010895E0912C0C02
:10E86400F0912D0C0895E32FA0911E08EA0F08954E
:10E87400ADE02A9FF001E35FFC4F0895A8E0B0E00B
:10E884000E94A87B0895F0E0FA93EA9308950E9409
:10E894006C420C943B42F0E00E948D7A08950E94F1
:10E8A4008D7B0E9456420C943B420E946C42E9ECE0
:10E8B400F7E1DDCB0E943B420C943B4220E030E088
:10E8C400E12FE05DEA93ECECF7E1A7CBEAE0EA9311
:10E8D4000C947762E4E4FBE0FA93EA9308951091D0
:10E8E4005D0500915F0508950E94FB423E2F0C9444
:10E8F400DD45EAE0F0E00E94D67A0895DF01EE27D4
:10E90400A30FBE1F0895FA93EA931AC9EF81F885FD
:10E91400FA93EA930895F0E0EA0FFB1F0895E02FBD
:10E92400A0E0B2E0B8CFEA0FFB1F3296E49108955D
:10E93400FA93EA93E0911B0CEA930E946338E13264
:10E944000895EA930E940938E1320895E6E0F0E080
:10E954000C94426C0E949646AAE9BBE0EE27A10FF4
:10E96400BE1FEC91E1700895EE0FFF1F0C94106D23
:10E97400EA930E946338E13208950E94B50D0C9425
:10E98400016CEAE3EA930C9434460E948D7B0C9468
:10E994004441E3E7EA930C943446EA23EA930E9461
:10E9A4006B41D2C8EA930E946B41CEC8DF01329614
:10E9B40091C80E948B7AE854FF4F0895EAE4F6E088
:10E9C400E0933A0CF0933B0C08950E94771AE0E030
:10E9D400E09321080E94C6150E94B50DE1E0E09382
:10E9E4001B0808950E94BD460E9451100E94FB42DC
:10E9F4000E2F0D330895EE81FF81FA93EA93089563
:10EA0400EAE2EA93E4E7F8E10895EA930E9416162D
:10EA14000C94B50DE093C105F093C2050895FE0171
:10EA2400FA93EA930895ECE8F8E1FA93EA93EE8511
:10EA3400FF8568897989FBCEE0E9F8E1FA93EA93E6
:10EA4400AE85BF858889998977CE0E948D7BAA89F6
:10EA5400BB898C899D89E4E6F0E060E070E00E9467
:10EA6400457B0E948D7B88E00E94F76A2C9608956E
:10EA7400E9E9F8E1FA93EA93EE85FF858BCE84E029
:10EA84000E94F76A2896CBCFFA93EA93EE85FF8526
:10EA940008950E9470630C94096884E00E94F76AE8
:10EAA40028960895EE27A10FBE1FEC910895EA93CE
:10EAB4000E94D6411F5F0895E091C405A7ECB5E01C
:10EAC400F0E00895AF5FEAE00E94307B0895E091A2
:10EAD400C305A7ECB5E0F0E0D3CBE981ADE0EA9F54
:10EAE400F001E05FFC4F0895EF73A5E1EA9FF001A8
:10EAF400E051FB4F0895EF73ABE0EA9FF001EC5E49
:10EB0400FB4F0895AC81BD81EE27A30FBE1FAC91CE
:10EB1400A0300895ABE00A9FF001EC5EFB4F08952E
:10EB2400EA0FFB1F0F01AC81BD8188CEA5E10A9FCE
:10EB3400F001E051FB4F0895EE81FF8101801280C6
:10EB4400AE81BF8115960E947A7BD0010895FE01A3
:10EB54003896FA93EA930895EAA5FBA5FA93EA9303
:10EB64000895FA93EA93FE013A96FA93EA930E947F
:10EB7400B56830E0E02F0895E091C105F091C20539
:10EB84000895A1ECB5E0ED91FD913296FE93EE93DC
:10EB94000895AE81BF81EA17FB070895E0E0E09392
:10EBA4006505E093660508951A930A933A932A93A8
:10EBB4000895FA93EA93E0910E040895A091000356
:10EBC400B09101030895E0910003F0910103FA93D9
:10EBD400EA93E0910203F0910303FA93EA93089510
:10EBE400E0930003F09301030895A981BA815ACFF9
:10EBF4001A930A9300E010E00895F801AA81BB81FA
:10EC0400EA0FFB1FE4910895AE0FBF1FAC91A03033
:10EC14000895D801F0E0AE17BF070895AE0FBF1FE7
:10EC2400EC91EA930895EFEEF0E0EA1BFB0B0895F4
:10EC3400A0910E04E4E1EA9FF0012E2F3327C3CF05
:10EC4400E0E0EA930E94AC4B0E94657D0895ECE0FD
:10EC5400EA9FF001A0910D04EA9FF00108951A9330
:10EC6400E1E0E0930E04E0930D0410E00895ED81DB
:10EC7400FE81FA93EA930895EF81F885EA1BFB0B72
:10EC840008953A932A935A934A930895EAA5FBA5C3
:10EC9400E20FF31FFA93EA930895ECA1EA930C941C
:10ECA4000F4C3A932A93EEA1FFA1E40FF51F0895A8
:10ECB400FA93EA93EBCFEAA5FBA5E40FF51FFA93C9
:10ECC400EA93EBCFE20FF31FFA93EA930895FA93D2
:10ECD400EA935A934A930895EA9FF001AEA1BFA123
:10ECE400F0E00895E2E0E0930E04E0E2F0E0EAA34D
:10ECF400FBA30895AE1BBF0BACCAEE8DF0E00895E4
:10ED0400E20FF31F3196FA93EA93ECA1FDA1E40F0D
:10ED1400F51F31960C943A6EECA1FDA1E40FF51F9A
:10ED24000C943A6EE9A1F0E0DE0116960895ED8D9B
:10ED3400EA930E94EA45E9A1EF5FE9A30895ED8B08
:10ED4400FE8BAB89BC8985CAA98DBA8DEA0FFB1FDE
:10ED5400E98FFA8FEB89FC89AF89B88DEA0FFB1F25
:10ED6400EF8BF88FED89FE89AD89BE890E94D67A32
:10ED74000E94987A0E94337CEE87FF87688B798B98
:10ED8400EB89FC89AB89BC890E94D67A0E94987A67
:10ED94000E94337CAE85BF85888999890E94097D4C
:10EDA400EA87FB876C877D8700E010E00895F8010F
:10EDB4000E94987A0E94337CEE83FF836887798768
:10EDC400AE81BF81888599850E94BB7CAA85BB855D
:10EDD4008C859D850E94BB7CAE85BF858889998979
:10EDE4000E94977B0E94667C0E94FC7BAF015A9331
:10EDF4004A930C941E6BE98DFA8DE21BF30BFA9384
:10EE0400EA930895E98DFA8DE01BF10BFA93EA93E6
:10EE14000895F901AD8DBE8D0C94106DED8DFE8DB0
:10EE2400E01BF10BFA93EA93EA8DEA930C940F4CEE
:10EE3400AD8DBE8D0C94106DEFE3F1E0EA1BFB0B7E
:10EE44000895EB81FC81AF81B8850895E00DF11D33
:10EE5400FA93EA930E94214AE5E3EA930895E09342
:10EE640065000C94D36E0E945C7DEE81EA930E944F
:10EE7400504A8F010895E985FA85AD85BE850895C8
:10EE84000E946A4AEB85FC85FA93EA930C94824AC1
:10EE9400ED85FE85A985BA85AE17BF070895EB8574
:10EEA400FC85AF81B885AE17BF070895AD85BE85D3
:10EEB400E985FA85EA1BFB0B0895FA93EA930C940F
:10EEC400B96BAB85BC85D8CEAF81B885EB85FC85A5
:10EED400EA1BFB0B0895D9010E94D67A0F0108950D
:10EEE400D0010E94017BAF01FA01AD85BE850C946F
:10EEF400106DED85FE85E21BF30BFA93EA930895FA
:10EF0400AD85BE850C94106DA985BA85ED85FE8509
:10EF1400EA1BFB0B0895E881F981FA93EA930895BB
:10EF24005A934A93EE85FF85AFCDFA93EA93EC8525
:10EF3400FD85FA93EA930E94F04CE0910E04AA85B1
:10EF4400BB85E9CCD901F0E0AE17BF070895E05CBA
:10EF5400F54F4FCAE091370CA091360CEA1708958B
:10EF6400E0911108ABE0EA9FF0010895E3E0EA9331
:10EF74000E94F462F5CFE081E05DEA930C9497621D
:10EF8400A091250CB091260C0895E2E5EA930E9425
:10EF940097620C94DD4DF096EA930E945563E2E784
:10EFA400EA930C949762EA930E949762EEE0EA93E4
:10EFB4000C949762ECEAF8E1D2CA0E94CA62EBE3CD
:10EFC400EA930C949762E0E3EA930C949762EBE380
:10EFD400EA930C9497625A934A930E947C180E2FDA
:10EFE40000340895FA93EA930C9491331A93E985C3
:10EFF400FA85FA93EA930895E552F84FA885B985FE
:10F00400A083B183E3CBE2E5EA930C9497621A936D
:10F01400E0913908E0531E2FEDE3F8E0BACAE0911D
:10F024001208A0911308EA170895E3E1F8E0DACF93
:10F03400E0911308ABE0EA9FF0010895A091740BEE
:10F0440041CDE093740BEAE2EA930E945563DBCF6F
:10F05400E091740BE05AA7CFD9011696EC9113CC2A
:10F06400F901A281B381BA93AA9308950E94CA6256
:10F07400EAE3EA930C949762D9011196E0E0EC93E9
:10F084000E947063D2CFD901EC91FDCBE05DEA938D
:10F094000C949762E05DEA930E945563B4CFEB58F9
:10F0A400F44F69CFEEE0EA930C949762EAE3EA93B3
:10F0B4000E949762F9010895E0935E0CF0935F0C4F
:10F0C400E2E0E0933608D9011196EC930895EA93AF
:10F0D4000E94556398CF0E94CA62DBCCE091190C60
:10F0E400D9CFE091190CF0E0DACFFA93EA9365CF27
:10F0F4000E94CA62ECE2EA930E9497620CCF3DDA66
:10F10400AC91A0330895A0915E0BB0915F0BE0E049
:10F11400EC930895EE81FF81E093270CF093280C83
:10F124001093240C0E94441CE1E3089541E050E054
:10F134000E94C961E887F987EAE3EA930E943E6185
:10F14400E13008951A93E985FA85C1CDE2E2EA93A4
:10F154000C943E6112DAAC91A03208950EDAAC91AF
:10F16400AB3308950ADAEC91EA930895EAE3EA935B
:10F174000C943E610E94C9613197E887F987E8855C
:10F1840008950E947A7BE40FF51FD001ED93FC9360
:10F194000895E091400BF0E0ED55F94F0895E0E05B
:10F1A400E093630CE093640C08950E94C961319765
:10F1B400E093400BE091590BA091400BEA1708959E
:10F1C4000E94CF56E091400BEA930895ECE2EA9353
:10F1D4000E943E61E0300895EC5BF44F0F01CDD9FD
:10F1E400EC91D001EC931F5FC1CAEC5BF44FA0E03B
:10F1F400A0830895EA930E943E61E1300895E0916E
:10F20400410B89CBE091410BEF5FE093410B0895F3
:10F21400A3EABBE0E091410BF0E00C944271AAE94F
:10F22400BBE0E091410B0C94B06FE091410BF0E036
:10F234000895FA93EA930C945253E091400BF0E052
:10F24400B8CBFA93EA930C94CA620E94CA62ECE2C5
:10F25400EA930C949762ECE2EA930C9497620E940E
:10F264004753E0E0E093410B0895E091410B0C9487
:10F27400B06FE091600BF091610B0895AEE5BBE0D7
:10F284000C94636EA0915E0BB0915F0BEC93F6CF80
:10F29400A0915E0BB0915F0B13970895E0E0EA93A1
:10F2A4000E94AB53E09335080895AA81BB81EC9189
:10F2B400E295E07FAE2FEC810895EA0FAA81BB812D
:10F2C400EC938ACAE091040DA091030DEA17089506
:10F2D400E0913B09F0E0E05CF64F08951083E09183
:10F2E4003B09EF5FE0933B09E12FA0913D090895AD
:10F2F400E0933D09E0913C09E150E0933C09E030A2
:10F304000895E05CF64FA0E0A0830895E091CF0D4E
:10F31400F091D00D0895A091CD0DB091CE0DEA17C6
:10F32400FB070895E12FA091D40DEA0FE093D40DCB
:10F33400E091D60D0895F0E0E85CF74F108308954E
:10F34400E091DB0EF0E0E652F24FE081E0939C00A6
:10F35400E091DB0EEF5FE093DB0E08950ED9AC91E4
:10F36400AA3308950F0109D9EC91E0530C94DF718D
:10F37400EA930E9497621F5F0895EAE5F9E1FA9320
:10F38400EA930895FE013196FA93EA930895E88189
:10F39400EA930C949762E881F9816A817B810E94E7
:10F3A4008D7B0895E05CF54FE081E0300895EA93A9
:10F3B4000E94F867EA930C94425EEA930E94C66442
:10F3C400EAE5E0933E090895EA930E948766E030F7
:10F3D4000895E0917100E87F1E2F0895E093730073
:10F3E400E4E8F2CF0A930E945E66E0300895FF27B6
:10F3F400662777270E94337C0895EE8DAE85BF85FE
:10F4040088899989F4DF0E94BB7CA9A1BAA18827C5
:10F4140099270E94947B0E94977B0E94667C0895A2
:10F424000E94977B0E94667C0895FA93EA93E2E136
:10F43400F0E0FA93EA9308952A93ED89FE89FA930A
:10F44400EA93FE017596FA93EA930C940E69EE8999
:10F45400FF893497EE8BFF8B0895ED89FE89FA932B
:10F46400EA93FE017596FA93EA930C940E69AE89B9
:10F47400BF8914960E947A7BEE83FF83BCCAE88519
:10F48400F9856A857B85AC85BD858E859F850895C4
:10F494000E94356BE883F9836A837B830895E8814E
:10F4A400F9816A817B810895EA81FB816C817D8188
:10F4B4000895E991F991309639F080EA9FE0019737
:10F4C400F1F7A8953197C9F708950024AF0DB01D41
:10F4D4000895EA0FFB1F681F791F0895EA1BFB0BB1
:10F4E400680B790B0895F195E195F0400895F09536
:10F4F40060957095E195FF4F6F4F7F4F0895EE2310
:10F504000E2EEA2F19F0EE0F0A94E9F70895EE0F84
:10F51400FF1FEE0FFF1FEE0FFF1FEE0FFF1F0895DB
:10F52400FE2FFF0FFF0B6F2F7F2F08956F2F660F96
:10F53400660B762F0895BA2FBB0FBB0B8B2F9B2F17
:10F5440008958B2F880F880B982F0895EA17FB07CF
:10F55400E1E00CF0EE270895FA9FF02DEB9FF00DFB
:10F56400EA9FE02DF10D08957A9F702D6B9F700D29
:10F57400F89F700DE99F700D6A9F602D710DFB9FC0
:10F58400600D711DE89F600D711D8827FA9FF02D95
:10F59400610D781FEB9FF00D611D781FEA9FE02D30
:10F5A400F10D681F781F089582D0D6DF0EF49BDF1B
:10F5B40008958BD0D9DF0EF49ADF0895002498E0E3
:10F5C400AA0F001C0E1A10F40E0E01C0A1609A9529
:10F5D400B9F7EA2FA02D08950024112490E1AA0F71
:10F5E400BB1F001C111C0E1A1F0A18F40E0E1F1E3E
:10F5F40001C0A1609A9599F7FD01D001089557D0F3
:10F60400EBDF0EF470DF08953F934F935F93002474
:10F6140011244427552730E2AA0FBB1F881F991FC6
:10F62400001C111C441F551F0E1A1F0A460B570BB2
:10F6340028F40E0E1F1E461F571F01C0A1603A95E5
:10F6440059F7FD01BC01D001CA015F914F913F916F
:10F6540008953BD0D9DF0EF44ADF0895AFDFEA2FD7
:10F664000895E894B7FF04C0A095B09511966894E6
:10F67400F7FD39DFB1DFFD010EF435DF0895C4DF96
:10F68400FD01BC010895E89497FF09C0A095B095C9
:10F6940080959095AF5FBF4F8F4F9F4F689477FDD4
:10F6A40026DFB2DFFD01BC010EF421DF0895E894EA
:10F6B400F7FF02C018DF6894B7FF06C0A095B095A5
:10F6C400119600F8039400FA0895E89477FF02C0B5
:10F6D4000EDF689497FF0BC00024A095B095809529
:10F6E40090951196801D901D00F8039400FA0895DA
:10F6F400ED91FC9111970895ED91FD916D917C919F
:10F7040013970895ED93FD936D937C93089505905D
:10F71400F491E02D08957A936A93FA93EA93089505
:10F72400689401C0E89401D09DD0182E862F612DD5
:10F73400192E972F712D1B2EBF2FF12D1A2EAE2FA0
:10F74400E12D0895119602D0FE2F1197E199FECF75
:10F75400FF93FFB7F894AEBBBFBBE09AEDB3FFBF16
:10F76400FF91089507D01196EF93EF2F03D0EF91F7
:10F7740011970895E19B02C0A895FCCF9FB7F89418
:10F78400AEBBBFBBE09A8DB3E81719F0EDBBE29AAC
:10F79400E19A9FBF0895552342F4503811F4E0FFD5
:10F7A40004C03196691F791F6BF050E8572711F494
:10F7B4005F93CDC05F3F31F0660F000C579567959E
:10F7C400752F08955F9300200AF0CDC0C6C050E89D
:10F7D400192E1522880F991F9527550F879550E8E4
:10F7E400072E0522660F771F7527550F6795089515
:10F7F400689401C0E8945F93F2DF703818F07F3F9B
:10F8040008F4A5C056E1571BAAF4519558300EF4DC
:10F81400593030F0EFEFFFEF6FEF7FE777F91AC061
:10F8240077275523B9F0EE0FFF1F661F771F5A95F0
:10F83400D1F710C07727583028F0EF2FF62F672F15
:10F844005850F9CF552331F076956795F795E7959C
:10F854005A95D1F700200AF44ADE5F91089568941E
:10F8640001C0E894309760407040B1F0002426F065
:10F87400772312F400943BDE172E7EE1112032F040
:10F884007A95EE0FFF1F661F111CF9CFEF2FF62F8D
:10F89400612D5F938ADF5F9108954F93AF01FD015E
:10F8A400DA01AB01BC01CA01402D012C142E4F9189
:10F8B4000895EA0FFB1F681F0895E095F095609581
:10F8C400EF5FFF4F6F4F08955F9381DF903871F1C1
:10F8D40050E8152604C05F937ADF903839F1703808
:10F8E40021F1572F591B13F112F4D7DFFACF5831F6
:10F8F40018F0AA27BB278827583028F0AB2FB82F39
:10F9040088275850F9CF552329F08695B795A795A0
:10F914005A95D9F7502D512562F0CBDF38F467950D
:10F92400F795E795739513F41EC0B7DF3EDF5F913B
:10F934000895EA1BFB0B680B51F010F40094BDDF33
:10F944006623A2F3EE0FFF1F661F7A95CBF7EE270F
:10F95400FF27662777275F910895EFEFFFEF6FE7A3
:10F964007FEF5F910895EFEFFFEF6FE77FE75F9120
:10F9740008955F932CDF703851F3903841F30124DC
:10F984000894791F23F41CF300203AF3ECCF0F9270
:10F994001F932F933F934F93112722279927689FF3
:10F9A400A0018F9F302D410D591F6B9F300D411DBC
:10F9B400591F8E9F27D0BF9F25D06A9F23D0BE9FFB
:10F9C4001DD0AF9F1BD0AE9F110D291F391F491F9A
:10F9D400591FE32FF42F652F522F4F913F912F91F1
:10F9E4001F910F9066232AF0550FEE1FFF1F661F0D
:10F9F40002C073954BF2CFDE5F910895100D211D67
:10FA0400391F02C0200D311D491F591F08955F93EE
:10FA1400DEDE703821F411200AF49FCFA4CF903891
:10FA240009F495CF01240894970B1BF4D4F3002018
:10FA3400F3CF792F1F932F933F934F9311241127C3
:10FA4400222733274427552790E2AE17BF0786079E
:10FA5400410730F0AE1BBF0B860B410B089401C06D
:10FA64008894551F221F331F111CAA1FBB1F881FF8
:10FA7400441F9A9551F7F901612D4F913F912F91B0
:10FA84001F91662332F0550FEE1FFF1F661F7A95F4
:10FA940043F281DE5F91089530976040704008958D
:10FAA40000240A160B06089500240A160B060806FD
:10FAB400090608955A934A933A932A931A930A93F8
:10FAC40008955D814C813B812A81198108810895C3
:00000001FF
